:20000000004B0020C14C0100FDC90110FDC90110FDC90110FDC90110FDC90110FDC901105D
:1C002000FDC90110FDC90110FDC90110FDC90110FDC90110FDC901103BCA0110A4
:20003C00FFFFFFFFFFFFFFFF9A100000000000000000000000000000000000000000000002
:20005C000000000000000000000000000000FAFA1400000000000000000000010000010179
:20007C00000000000000000000000000000000000000000000000000000000000000000064
:20009C00000000000000000000000000000000000000000000000000000000000000000044
:2000BC000000007800080230000800000000000000000804FA000000FFFFFF000C1100004A
:2000DC000000000000001D1100000000000000002E010F000000FA0000002F010F0000005F
:2000FC00FA000000300100000000FF000000310100000000FF000000320100000000030053
:20011C0000003301000000000300000034010000000001000000350200000000FFFF000021
:20013C00370200000000FF000000390200000000FF0000003B0200000000FFFF00003D01B8
:20015C0000000000FF0000003E0100000000010000003F01000000000100000040010000C2
:20017C0000000700000041200000000000000000610200000000FFFF00006308000000002F
:20019C00000000006B080000000000000000730800000000000000007B08000000000000D2
:2001BC000000830205000000580200008501000000001000000086010000000032000000F0
:2001DC0087010000000032000000000038C40D00C8000000810000320F01000000C50D00E3
:2001FC00900100004000009605010000952B0D00C8000000220000320F0200003600010045
:20021C000600000000000000000F000000000000000000000000000000000300FFFF0000AC
:20023C000403FFFF0000FFFF0F00F4010005401F0320000100000000FF3F0F0008000E00B0
:20025C0000000000000000000300010F000009010000000000000000000000000000000065
:20027C0000000000000000000000000000000000000000000000000000000000AD000000B5
:20029C000001363601010001020100010301000104010606080400000C0100340D01000F4E
:2002BC0010040101140100FF1608000020020000220100FF23010001240100FE2501000820
:2002DC002602000028010001290100012A0200002C01000F2E020000300100013101000881
:2002FC00320200FF3401000735010240360100003701000138010001390100FF3A01000FCE
:20031C003C0200FF3E01010F3F0100014001041F41010001420100FF4301008044080000FB
:20033C004E0100084F01000F50010001510100FF5201090A53010185540100015804000056
:20035C005C0400006004000064040000680400006C04000070040000740400007804000011
:20037C007C040000800100FF81010001000120181A18182C34041E000C0E020B040B0A0792
:20039C000800110F00000500B900B300AD00B8001C00300038000800340102000304710404
:2003BC0002046004110470040204020401040204000410046104000414046304730472042A
:2003DC0062044304000413040604000400040404120400040004000400045104640000043C
:2003FC0000040004440400040004000400046504000435048104640005040004830400045A
:20041C006604000400040804010171010101010111010101310101010101800100011001ED
:20043C0061013B001400630173017201620143010001130106013D01350004011201000155
:20045C0000010001000104010401330133013C014401320136000001000165010001350082
:20047C008101000105018201830100016601000100010801030271023001600211027002CD
:20049C0001020202020280020002100261023A0041006302730272026202430200021302B3
:2004BC0038000002000204021202000200020002000204020402370037003C0244020002C2
:2004DC00390000020002650200023502810200020502820283020002660200020002080216
:2004FC0000D940010000F13B010002A3360000006984010001A3360000006984010003798C
:20051C00E80000006984010004EF830100006984010001E383010001DD83010001698401CB
:20053C0000016984010001698401000021550100016984010001698401000169840100017C
:20055C006984010002E383010002DD8301000269840100002155010002698401000269847F
:20057C0001000289400100026984010004B7410000006984010003E383010003DD830100EA
:20059C0003A336000003A336000003698401000379E800000369840100002155010003695E
:2005BC00840100036984010004E383010004DD83010004A336000004A336000004A3360042
:2005DC000004B74100000469840100046984010004E983010000215501000104E9FA01004E
:2005FC000300000000040000EDF701008BF90100DFF90100F9F301005DF40100D5F8010088
:20061C0061FA0100C7F90100B1FA0100F9F2010019F501006DF9010001F901006DF5010035
:20063C00BDFA0100D5FA01009DFA010089FA010043FA010035FA0100D5F601006FFA010056
:20065C00ADF9010015FA01009DF60100DFFA01004D2101005D63010001F00100C1F5010080
:20067C0029F10100FDF9010099550100C5790100AD790100BDF4010061810100538101008D
:20069C0059F601000000000000000000F38201003580010015F701000000000000000000B5
:2006BC00000000000000000000010400003333333333333333333333333333333303010FD6
:2006DC0000000000000000000000000000000000FFFFFFFFFFFFFFFFFFFFFFFFFFFFFFFF0E
:2006FC00FF46485465737400000000000000000000000000000000000000000000000000B1
:20071C0000000000D106000001000000680C000008000000F605000001123456789ABCDE25
:20073C00F000000000000000000000000000000002040201010101090200A2A6A8A0A5A5BC
:20075C009F95AD96B8B2A4313117191A21241B1D1F31313331313118191A22311C1E20315F
:20077C00313431000000000002000000020000000A000000020000000200010000000000B4
:20079C000000000000000000000000000000000000000000000000000E00000003007100BB
:2007BC0030016000110070003102200350048000070010006100000014006300730072000D
:2007DC006200430000001300060000000000040012000000000000000000040004003700EA
:2007FC0037003C024400000000000000000065000000350081000000050000008300000081
:20081C0066000000000008000103710301030103010301030103220302030103000310037E
:20083C000003000300030003000300030003420300032403060300030003040312032503C5
:20085C002303250323030403040300030003000344030003000323030003650321003503BA
:20087C008103000305030003000300030003250323030803A4260020500900000000000025
:20089C00A42600205C09000001000000EC2600206809000000000000EC260020740900009A
:2008BC0001000000342700208009000000000000342700208C090000010000007C27002043
:2008DC0098090000000000007C270020A409000001000000C40B0000D4280020040D0000EE
:2008FC00C40B0000F4280020060D0000C40B000014290020080D0000C40B00003429002031
:20091C000A0D0000C40B0000542900200C0D0000C40B0000742900200E0D0000C40B0000A9
:20093C0094290020100D0000C40B0000B4290020120D0000000001401FFF00001700000040
:20095C000000014020FF0000180000000010014021FF0100190000000010014022FF010005
:20097C001A0000000020014023FF02001B0000000020014024FF02001C000000003001408E
:20099C0025FF03001D0000000030014026FF03001E0000008F0000008F0001008F00020090
:2009BC008F000300900000018F00010190000002900000038F0001048F0000058F0008047F
:2009DC008F0000048A000006510000007F0001003F0004003F0002003F0001007F000200C2
:2009FC007B756E6B6E6F776E2D696E7374616E63652D6E616D657D007B656D7074792D6943
:200A1C006E7374616E63652D6E616D657D00C0467B7374617469632D696E7374616E6365F8
:200A3C002D6E616D657D00C0000000000800000000000000200000004000000060000000C7
:200A5C00000000000600000002000000860000008200000000000000080000001000000052
:200A7C0018000000200000001404C0A00A0480A0090480A008400080FE000000060880807B
:200A9C00070880800D2007C00E2007C01400C080024000800300C080094000800840008058
:200ABC000A400080FE000000C003000080070000000F0000001E0000003C00000078000027
:200ADC0000F0000000E0010000C003000080070000000F0000001E0000003C0000007800FE
:200AFC000000F0000000F000000100020101000302010002000000000301000704010003DA
:200B1C00050800000D0101FF0E08000016080000200200002110010009330100557A010009
:200B3C00E9A50000F5BE00000D840100F929010061C8000013840100AD10010000003200F2
:200B5C000000FF0000000000010002000400100000FF080004000001000200040008000049
:200B7C0000000000FFFFFFFFFFFFFFFF00000000000000000101010100C201000300000097
:200B9C00000000007BC80110C5BC0110D9B2011033C20110BDAD0110C1B101106DBA01107B
:200BBC0065BB01101DC0011055680100E57801009F6F00000DD00000A551010031190100B1
:200BDC00B56E0100B1720100001000400600000015000000FF000000000000000302FFFF44
:200BFC000000000000000000FFFFFFFFC4090000000000000000000001003A0100000000D4
:200C1C00000000003D0C0100C1280100F5830100DF8201005DAB000001EA000001000000B5
:200C3C0040420F00010000000000000000000000000000000020004007000000110000008E
:200C5C00FF0000000000000005040000000000000000000000000000000000000000000070
:200C7C0000000000C33B3D3A5D3A713AA10A8F3A0F3BB309495E850A2F3B853B06088080B9
:200C9C00070880801808C0801D08C080FE000000001610160E18151C021203241858030223
:200CBC0010025800010000000000000000000000000001000000FF7F00000000000000002E
:200CDC0000000000000000000000000045E100005D36010001010100004002400B000000AE
:200CFC0027000000FF000000060007010C02FF03FF04FF05FF06FF07000105090004081057
:200D1C0000040810200C0000D02A0020500C0000300B000078250020E40B000041B501100B
:200D3C0095A6011015B80110010B0101020802010100004000BE040A00BE0208FFFFFFFF81
:200D5C00FFFFFFFFFFFFFFFFFFFFFFFFFFFFFFFFFFFFFFFFFFFFFFFFFFFFFFFF35452515DF
:200D7C0002030504842E0020F40C0000FF0000000000000000000000010000003D7A0100BF
:200D9C00453D0100060005000000FFFF000000000F00000005900000D1C0011061AD011046
:180DBC000A00000078180020AD680100E584010051CB0000B78301008E
:201000003C000000000000000000000034100000000000000000000001000000000000004F
:1C10200000000000000000000000000001000000000000000800000000000000AB
:20103C003400000000000000000000006810000000000000000000000100000000000000E7
:14105C00010000000000000000000000080000000000000077
:2010700030000000000000000000000098100000040000000000000001000000FFFFFFFF87
:10109000FF00000001000000080000000000000048
:2010A0002C0000000000000000000000C4100000040000000000000001000000FFFFFFFF2F
:0C10C000FFFFFFFF080000000000000020
:2010CC0038140000E410000095A1011091A70110A1C2011009B2011041B8011000000000EA
:0810EC00000000002D000000CF
:2010F400280000000000000000000000141100000000000000000000FFFFFFFF0000000093
:081114000800000000000000CB
:20111C00341400003011000065C2011069C101101BC2011091BA011000000000000000006D
:04113C002F00000080
:20114000341400005411000071C20110A5B6011099BF011045B601100000000000000000BD
:04116000300000005B
:201164002400000000000000000000008011000000000000000000000000000008000000AE
:041184000000000067
:20118800240000000000000000000000A41100000000000000000000000000000800000066
:0411A8000000000043
:2011AC00240000000000000000000000C8110000000000000100000000000000080000001D
:0411CC00000000001F
:2011D00000000000741900200400000000000000000000002000000070100000300000007E
:2011F0001C1100007C1900200400000000000000000000000C000000301300001800000092
:20121000401100008419002004000000000000000000000024000000481300001800000015
:20123000000000008C19002004000000000000000000000010000000A01000002C000000E9
:20125000CC1000009419002004000000000000000000000020000000641100002400000018
:20127000FFFFFFFF9C190020040000000000000000000000280000008811000024000000A4
:20129000FFFFFFFFA4190020040000000000000000000000580000003C1000003400000089
:2012B000FFFFFFFFAC1900200400000000000000000000001000000060130000180000009E
:2012D000FFFFFFFFB41900200400000000000000000000001C000000AC1100002400000014
:2012F000FFFFFFFFBC19002004000000000000000000000038000000F41000002800000085
:20131000FFFFFFFFC419002004000000000000000000000054000000001000003C00000020
:1813300018000000000000000000000040130000080000000000000032
:1813480018000000000000000000000058130000080000000000000002
:18136000180000000000000000000000701300000800000000000000D2
:0813780002000000980D0000C6
:041384000100000064
:0413880000000E0053
:04138C0000000F004E
:041390003200000027
:041394000100000054
:04139800D018002049
:04139C00000200004B
:0413A000FB830100CA
:0413A400FDC901106E
:0413A8000000000041
:0413AC00000000003D
:0413B0000800000031
:0413B4000000220013
:0413B800FC160020FF
:0413BC00010000002C
:0413C000E818002009
:0413C400080000001D
:0413C8000000000021
:0413CC00000000001D
:0413D0000000000019
:0413D400080000000D
:0413D8000000000011
:0413DC00000000000D
:0413E0000100000008
:0413E400F4170020DA
:0413E80006000000FB
:0413EC0001000000FC
:0413F000E0150020E4
:0413F40000000000F5
:0413F80000000000F1
:0413FC0000020000EB
:0414000000000000E8
:021406002900BB
:021408000100E1
:02140A002500BB
:02140C002F00AF
:02140E003000AC
:021410002D00AD
:021412000100D7
:0114140001D6
:0814180003000000380D000084
:081420000000000000000000C4
:0414280000000100BF
:04142C0000000300B9
:0414300083C4011060
:041434003C14000064
:041438003C14000060
:04143C0000000000AC
:041440008000000028
:041444008000000024
:0414480000000000A0
:04144C00E81800207C
:04145000937F010085
:041454002000000074
:04145800C00C0000C4
:04145C00A00B0000E1
:0414600009C30110AB
:04146400C747010075
:04146800234F01000D
:04146C0095C801100E
:0414700097C8011008
:041474000000000074
:04147800BF0C0000A5
:04147C00140A00004E
:041480002C0A000032
:04148400FC0900005F
:0214880008005A
:02148A00090057
:02148C0001005D
:02148E0000005C
:01149000015A
:041494000000000054
:041498000000000050
:04149C00000000004C
:0414A0000000000048
:0414A400DD840100E2
:0414A800515D010091
:0414AC006570010066
:0414B000396101009D
:0414B4006B62010066
:0414B8006554010076
:0414BC000524010002
:0414C000A7810100FF
:0414C400713701007B
:0414C8000DC801103A
:0414CC001DC8011026
:0414D0000800000010
:0414D40024000000F0
:0414D80018000000F8
:0414DC0028000000E4
:0414E00020000000E8
:0414E4003C000000C8
:0414E8000C000000F4
:0414EC0034000000C8
:2014F0007E482DE9F04F0C4601210170DFF8F491DFF8F481DFF8F4B1DFF8F4A178494FF04C
:20151000000C2027ADF1440D65461F4081F800C0CE490E9391F83C600D9205EA020008BF02
:2015300000287AD10D984FF0E047194662460F4002EA000008BF002843D10E9E0D9B4FF441
:201550008601B9F8B200DFF828C3CDF8289012EA060701EA030108BF002919D1C34912EA78
:20157000060701EA030108BF00296FD0374641460D9E0C8101F130034881002F83E8C000AC
:2015900004BF331CB3F1806F60D102285ED111E0374641460D9E0C8101F130034881002FC2
:2015B00083E8C00004BF331CB3F5803F4ED1B0F5505F4BD1086A6746436938682146984737
:2015D00042E046465946B6F9087091F90000BC42A0F10100087017D1728906F1300003C820
:2015F000002904BFB0F5803FB2F5505F08D0002904BFB0F1806F022A02D011F055FD03E0AD
:2016100012F0D2FF16F0C6FA524692F90000401E10706FF00101318114E041466FF0010032
:2016300001F1080210806EB1BC480078832802D0BB48812202704646316919B16046884779
:201650002146E8E7CDF82890B9F8B2000D9A0E9E02212F461140374008BF002900F09483BA
:20167000B04A43F201418142109200F06783C91C814200F06383594691F900105A464746C6
:20169000491E1170B7F908108C4205D043F60401814240F062835EE36C4890F83CC007F160
:2016B000300090E800034FF482062F4617EA090706EA080008BF00281CD10B48303003C8CC
:2016D0004FF400322F4602400F4008BF002A02D111F0EAFC41E312F067FF3EE3E819002006
:2016F0003C190020081000204014002043190020421900200020BCF1010F4FF08105884C4C
:201710000F9003D0207808B116F074FC2570BD4C0020677860810646E7702069DDF8409031
:20173000417A027A89F8006001F0070302EB0322490996B238BF361F09D304F110010A683A
:20175000167A517A01F0070106EB0126B61E457ADFF8B482B6B235F07F0540F0D782B6F528
:20177000006F80F2D3820A3031460FF0D1FFE16904F114000522083116F048FAF61EB6B22C
:201790000520E37DA57D314A6081217ECDF83090C3F3011B92F83C00617105EB0325002868
:2017B00008BFBBF1020F00F0B182BBF1020F00F3AD8260B115F0070F00F0A8825748007836
:2017D000862804D105F00700022840F09F82281300F00209B9F1020F4CDAA37805F00700D1
:2017F000022835D1D8F804A093BBE16909A801220D3116F00BFA06206081D0478146834ECA
:201810004648D8F8082037680078CDF82C80862816D127B916F0EEFB4046376882689DF9A1
:20183000240016F04BFE9DF9246078770020B8774846FE77904705F0100010F0BDFE01E052
:201850004846904716F01CF864E2C04654120020324800780022862808BF0122CDF82C800A
:201870005AB1002012F0ECFEE77805E000000C8C70170020CDF82C80A37887B17BB9012F96
:2018900000F03F82022F03D115F0070F40F03982032F04D105F00700032840F03282280939
:2018B00008D315F4405F00F02C82C7480778002F00F02782B9F1020F02DAA80A80F0218245
:2018D000C4480078C0F3810A4FEAA018BAF1010F00F01782B8F1010F00F01382BB48BBF114
:2018F000020F0CD010F80A1010F80800B8F1000F0844C7B21CD0E8091AD3BF1E0CE000EBBE
:201910000A014044097900794018C7B2E8090BD25AEA08030CD0BF1CFFB209E01831002085
:2019300014310020163100205AEA080308BF0227C5F30029A7EB09008642C0F2E281F61B22
:2019500009EB0600290980B2208124BF25210F910F994018743080B216F03EFAA678E0603D
:20197000002800F0CE810021742210F0D2F9002020711EB90C9905F0200008700C98037895
:201990000026002B65D0B9F1000F62D19048008805F0070103291BD18108324609D31B490F
:2019B00091F82E3093B90B681BB15B7E33F07F030CD15AB9800807D3D3498B68887813B102
:2019D00018468047267908B9002301D004262671D94890F83C3013B1BBF1020F39DA60793B
:2019F0000DF125010C90E92012F052FFB3469DF82560D04966B901F10800072202700822B1
:201A10000BE0C04680300020F41200209C0A002001F108000522027018224A72861C0221BB
:201A300000233170BBF1000FC37003D0317841F0100131700C990A9A01710521A2F8781082
:201A5000C2F8840015F09AFA304603210FF060FE2679E16801F174004860886523890B818D
:201A70002089A1F85C0028090ED3C9F1030082B2A1F85C20886DD84916F0C8F8E1688A6D84
:201A9000B1F85C00801888655248D34B0078C0F3011218788D81B9F1000F00F0780040EACD
:201AB000020046EA00060E744FF0FF038B730CBF6079002081F8308081F83AA081F849001B
:201AD0006089002FA0EB090085B2658100F01181E069E78029183A460831684616F096F8BF
:201AF0003C48EE19B5B26581E16800780A7C6E46C0F38103C0F3011AC0F38108002B02F0A5
:201B1000400946D0C0F301100023022801D1D0090BD29DF801209DF8000000EB0220A1F8CC
:201B300044000DF10206A1F84200AE4AB1F84400B2F85220824203D04FF6FF72824222D16B
:201B5000B8F1030F12D072783078A64B00EB022082B24A86B3F85010B61C0120914211D092
:201B70004FF6FF71914218BF00200BE0E0683146323016F05BFCE0689A493230473115F063
:201B90008DFE08360346002B00F0B6802046E168C07D831126D0BAF1020F03D0087CC00980
:201BB00003D309E059EA080206D172783078B61C00EB0220A1F84200032B0DD07078327849
:201BD00002EB00220A850DE0980C0020500D00008813002097300020E0683146283016F08A
:201BF00025FCE16888890009C0F08380886D3A46694616F00BF8E068816D79188165E66975
:201C1000B0F85C1001227F18A919A0F85C7008310DF1260015F0FAFF6F1CBDB26581E1683C
:201C30009DF82600896D0870E2689DF826609DF82630906D401C9065B2F85C00401CA2F8D1
:201C50005C0006F0070082F82400C3F3C10182F82510208992F824708046002F4CD05F4FD0
:201C70007F183E78361D8642E68045DCE06929183246083105A815F0C9FF3A789DF817C092
:201C9000111D481980B29DF81450608105EB0C60E3689DF8165000EB05409DF815500429A0
:201CB00000EB052098610BDDE06806A9521E1C3015F0ACFF3878E3686844C07D83F826003B
:201CD000986D05A9324615F0A1FFE068816D71188165B0F85C10A8EB06077118A0F85C103E
:201CF000791E89B22181B0F85C2001818918A0F85C1000F081F80DE016F0BAFA11F0D4F937
:201D100008E016F0C3F805E04819002016F0BEF8CDF82C80DDF82C80D8F804008047E16911
:201D30000A68002313710968E161D8F80810884713E0C04694170020541200204046807848
:201D500041465F46401C887097F900005946401E087011F0A9F915F023FB23480A99214FAA
:201D700000226FF0010690F83C00A1F8B2203E8110B11098007808B915F00CFF1B481B4964
:201D900090F90000401E0870194890F9000010B9134800210170154890F9000088B10D9A6E
:201DB0000E9F02214FF0E0401140384008BF00290BD00E4890F90000002806DC16F01AF94E
:201DD00003E00020014605F0F9FA0A49002011B00870BDE8F08FC04696300020140D0000E4
:201DF0003A19002040140020541200204219002043190020E81900202DE9F04FB94C0C3CAC
:201E1000E0686189E2692589806DADF13C0D0E46891808312A4615F0F9FEA81986B2E068D8
:201E3000816D6D188565E0690122311808310EA815F0ECFEE069761CB5B204226581291813
:201E5000083104A815F0E2FE9DF813109DF8100000EB0160E3689DF812102D1D00EB014087
:201E70009DF81110658100EB0120049015F0C8FFD863049815F086FCA3F84000EA2015F002
:201E900043FD0221B648E2680170117C2079084310749DF9380016F011FB82F846009DF9EB
:201EB0003800118982F84800002082F8470002F174009065B2F85C00401A51680918516056
:201ED0009089830A18D2030957D310F0070F07D000F00700032812BF081C5068401C48E0EC
:201EF0005068C17801F00703491001F0380101EB43014018001D3CE0171C02D116F07AF824
:201F1000E268B889800A2ED379684878C6112AD13E89796600204D780B7805F07F056D0034
:201F300005EBE3157E2D0DD07F2D09D003F07F031818801C5B1880B2991C8642EBDC08E08A
:201F5000002100E00121801C87F8601080B2864201DA002005E07968411879603989091AF1
:201F70003981A7F86800506E10B1B2F86800B0B1506850619089000916D292F86000002819
:201F900000F0FC80104611F0D1FFE268D06C002800F0F480B2F85000002840F0EF8016F0C5
:201FB00055F90020E06024E24FF0000B1546104605A9CDF814B007ABCDF818B095F82470CB
:201FD000CDF81CB006AA05F0F1F8002840F0CB80059A6E6968682B89311A581A1FFA80F8E7
:201FF0000AB916F007F8B5F85C0000900196CDF808800698001D03900598A969AB6D3A46F7
:2020100015300AF00BFF002840F0AD80AD4895F860302E89C15D701A288113B1284611F095
:2020300085FFAE8906F00706032E02D168680078E87395F80F90732009A914F085FD832091
:202050000DF13A0108F02CFEDFF8D082DA4651460AE0C278012A03D1002F08BFDC2027D029
:20207000001D491C0990C9B29DF83A00884279DD09988278032E07D00378B3420DD098F84B
:2020900000300BB1022E08D0032EE9D10378032BE6D103465B784B45E2D1BB10B3EBA20F78
:2020B00005DA02F0030207F003039A42D1DD50468146059895F80FC090F814E0514601E069
:2020D000491CC9B28E4549DD07694B00032E03EB070209D1FB5C032BF2D152786245EFD1E1
:2020F0000BE0C0468C3000201278B24205D098F80020002AE4D0022EE2D10698077D002FEE
:2021100008BFB9F1DC0F2DD0A869B0F1FF3F23D0712008A914F018FD5346089AA96905982E
:20213000824206D106989A4600EB8A00C068884210D85B1C2C32022BF1DB0698491CB1F1B4
:20215000FF3F00EB8A00C16002D1079801218170584608E0DB2007E0DB2004E0DC2002E0F1
:2021700014310020DD206870E26850709069577850651FB1F22015F0C7FBE2689F4DDFF8D8
:20219000849295F83C10002900F0AD8090899C4EDFF874B200F00700022858D1A078002870
:2021B00055D15078002852D1E1684FF000080CA88DF83980283116F039F906F11001E7686C
:2021D00008882B6E401C0880786E0DF139020421984704F10C0A30B94846006818B19DF877
:2021F000391080F8681015F075FC90B1E76897F8300002280ED1DAF80000594602222031E2
:20221000283014F0F1FE28B90BF116010CA816F00DF9E7680DF12E000090AD6E786E0CA9EE
:2022300042460BABA84779480078862808D1708AE768401C7082B88900F0100010F0BCF914
:2022500016F004F84046E06015F01AFBD3E0704B1A78002702B101277248026827B16F78A7
:2022700017B115F037FC28B91878002831D015F031FC70BB53782779002B40F0BA809DF8C2
:202290003800B18A02F12803002F207002F11C0201F10100B08214BF082600265D490020BB
:2022B000086015F02FFC0146009658460192263006881A460D20334604F04AFC20B914F067
:2022D0005DFE03E0180D000015F078FA1348E268017841B1D5F884702FB1394610468847BF
:2022F0000E48E26801780A9251B1907BFF287AD01046C17B042976DC40680078072872D0F9
:20231000938913F0070040D0401E56D0801E6AD1C3F30130022808D102E0C0469012002086
:202330005068007807282ED0FFE7108900285AD0104641684A1C42600F788446C7739CF839
:2023500024607EB9002F4ED00A2F4CDA0189324EF01910F8010C884209D0082F43D10829BF
:2023700005D040E0C07B00283DD00A283BDA60460189491E0181C17B0B3101700A99C87BB9
:20239000401CC8731BE0322018E0244E96F8A1000F280CD015F052FD48B9181300F002002B
:2023B000022804DA0A984D462D1D2968884796F8D7000A9A1074152000E0162010700A992B
:2023D0004D4605F1280013F095FE154E7068804795F83010491C85F83010B168884720208D
:2023F00015F068FE02E00AA812F0D4FF4FF0000828E710F059FE0FB0BDE8F08F54120020E3
:20241000541800209C0A0020600C00201831002016310020981700204C070000CC0B0020E5
:20243000F41200208C3000202DE9FE4FE54980460122A1F130000260DF480768002FFCD05B
:20245000DE4ADF4EC027E048E04B17603268920808D2324652F8042C03F14104120C42F0DD
:20247000F00222704FF0000A8346C1F800A0DFF864C3DBF80810D64D0191880E43D2480EBE
:2024900041D3802018744FF6D802A3F8512018702868C0F30464162CA8BF203C1F460F3FD6
:2024B000387800F01F001628A8BF2038844223D0624602F1980EDA4ACEF800A0261A022E5C
:2024D00005DC16F1020FB8BF6FF0010600E002263018166800F01F06844246F4F856A7F846
:2024F00066604FF001061660E8D11068374617601068CEF80060106828460068C0F3042062
:20251000162808DB06E0A5F1D0000068C0F30460162800DB203800EB2170401C162805DA59
:2025300010F10A0FB8BF6FF0090000E01520DE4F00F01F0040F4F850A3F8590038688008A9
:202550003ABFEA48C0F800A041F04061019E6246A5F13804C80E8F0E80F0010000F0010028
:20257000106087F0010000F0010090602068C0F38367C0F38F21B00C23D2304640F3072079
:2025900000280BD542425046490805D17F0806BF0127391C4FF6FF71521EF5D1002810DD19
:2025B0004FF6FF72490041F001018A4207D27F0047F001070F2F92BF01210F27111C401E04
:2025D000F0D141EA0741182013F076FC2068D24E2768C94CA6F10409C0F3870107F00300E5
:2025F00041EA0021D9F8040040F2FF3253468FB22C21466800972746A7F14000B0470C3D56
:202610002868C0F30D011C2013F056FCB84955F8080C014000F07C400143142013F04CFCB6
:2026300055F80C1C01F47C000904090C0143102013F042FC624955F8042C0968C2F303502C
:20265000C2F30345490813D2DBF800100B0510EB237003D41028A8BF0F2000E0504609048E
:2026700015EB217503D4102DA8BF0F2500E0554645EA001502F47F4002F0FF01B8F1220FC5
:2026900040EA054041EA000124BF02F0804211430C2013F011FC974DB8F1220F32BF012098
:2026B0002868C0F30070B8F1220F4FEA400040F0200084F8090126BF2868C0F34070012035
:2026D0008E4EB8F1200F40F0100084F8090138BF514606D33168C80C00F44070C1F384516F
:2026F0000143282013F0E8FBB8F1200F26BF3068C0F301505046B8F1220F4FEA400040F0E6
:20271000600084F80C0126BF2868C0F3C0605046B8F1220F4FEAC00040F0800084F80101E1
:2027300026BF2868C0F345505046B8F1200F4FEA800040F47C40A4F89C0138BF70490AD3EF
:20275000306801038A15920501F47C1100F00F00114341EA0031082013F0AEFB4FF48000CF
:20277000A5F1D0012060674A886D40F21E236FF31F40834216D90868030E13F00F0F03F03F
:202790000F01C0F3034018BF491E072805D006280EBF0720801C00F00F0041EA0011A2F155
:2027B00008000170DDF804C0CCF381477F1E13D07F1E3BD036E0C0469402224300600C4085
:2027D000B03F005040100940AC3F005015620840881300500000204328460068810C21D273
:2027F0004FF480412160D2F80210430AC0F3033703F0800321F08F010B4347EA0301C2F8DA
:202810000210D2F80130060A66F30303C2F80130116800F0E70721F0E70147EA010004E0DB
:202830002C2009404FF00040224610603B480068C0F3C0070FB94020A0624FF400702064D6
:2028500028684027C0F3C14040F0300084F8C800CCF3815050B3401E03D0401E1FD00221E5
:202870001EE0012013F0ACFF06460420314610F013FD042013F0A4FF8642FAD1224806684F
:2028900026F07F4013F0C2FDD9F81400036807214FF06022300E98474FF480602060032174
:2028B000042010F0F9FC08E0000009400420012110F0F2FC154813F0A9FD203D286814493A
:2028D00047F6180600F03F0084F8CB0F144B0E80D9F800201868D1680220884711480D4DCD
:2028F000076001212960BDE8FE8FC04694042A43FCFCFC008C13005040A00C40981300506F
:2029100000803F400A600840A83F0050BD37860070B00C4094046042A4010010B03F0050AB
:202930002C20094000600C40F0B5CB4CCB4ECC4DA088ADF1640D4108C0F090800CA808A9B3
:2029500010F01EF801287AD105F128000068D8B10769CFB1062002238DF808000022ADF83F
:202970000A300FA9ADF80C2002AB009193E803000C23B84740B9BDF83C00E085109F276312
:202990001198606315F0E2F99DF82D00012806D0022084F82800BDF8221021840BE00320BA
:2029B00009AF84F828003A6804F120010A6078684860BDF82210BDF8200009AA10F0BCFDD9
:2029D000011C02D0CDA015F016FD022013F0E0FBBDF830009DF82C7030870DA986F83A70C8
:2029F00006F1480015F0A0FCBDF8320006F13E0709A9A6F84600384615F096FCBDF8220042
:202A1000318FB087502014F0A5FFB6F84610532014F0A0FF4A20394615F0D4FA96F83A10E9
:202A3000E12014F0A3FFB18F4B2014F093FF06F10800102114F060FE0120207008E014F06F
:202A50009FFB2061012013F0A3FB002015F03CFA201D012114F042FE2046808880080DD3B5
:202A7000206B13F033FDA078271D18B109F06EFE03F08CF83846022114F030FE30894108B2
:202A900005D306F10800012114F028FE3089810805D306F10800022114F020FE30890109E2
:202AB0004CD396F8540006F1080700283ED0401E3AD0401E02D0401E34D03AE096F85010C7
:202AD000472014F053FF96F85110542014F04EFFB18F4B2014F03EFF318F502014F03AFF1C
:202AF000092396F83A008DF8593016AA8DF8580001238DF85A30BE498DF85B3018201CF099
:202B100067FBB4F85A00B4F85810884211D196F8520001280DD1B07858B13846202114F0A2
:202B3000EBFD06E0032002E0022000E0012010F093F83846082114F0D1FD3089410917D39E
:202B5000AC491820422217AB1CF042FB96F8520006F10807032818BF042802D1B06D13F0C2
:202B70009DFC12F0D3FE3846102114F0B7FD3089810907D30FF004FC06F10800202114F012
:202B9000ADFD3089C10907D30DF0B2F806F10800402114F0A3FD3089400A0DD396F85500AD
:202BB00015F092F941F2883013F0A8FC06F108004FF4807114F092FD288940086ED3687803
:202BD000002600EA500109095ED2010903D3AF782B79002F30D1410916D281090CD2C00904
:202BF00056D32879002808BF50A006D056A015F07FF909F0ABFD4BE058A015F079F909F09F
:202C1000A5FD02F0C3FF43E059A015F071F909F09DFD052702F0BAFF774815F0E9FB7F1E14
:202C3000F8D1A878012833D057A015F061F9201D012114F061FD2BE0A3B156A015F058F9AD
:202C50000720502113F0A2FC40F6AE3015F0D0FB3746162113E0C046E8100020B0110020A1
:202C7000F80D002055A015F043F90720D02113F08DFC40F6AE3015F0BBFB012776210E2089
:202C900013F084FC2F7103E056A015F031F9A6706E7005F10800012114F020FDA088002874
:202CB00042D10A200825554CADF812004FF0FF37ADF81050616A059704A88847002833D1BA
:202CD0000720ADF84850616AADF84A0012A88847149E159640BB4A499DF84E2008789042FD
:202CF00017D19DF84C004A7882420FD089684B6C7BB10021324698470BE0C04641757468C7
:202D1000204572726F723A20307800C0304601F093F8159840B1ADF818500320ADF81A0038
:202D3000616A079606A8884719B0F0BD53454E534F52205448524553484F4C442044455484
:202D5000454354454400C04653454E534F52204441544120524541445900C0465741544518
:202D700052204C45414B2044455445435445440053454E44494E472035204441544120504B
:202D900041434B45545300C05374617274696E672E2E2E00436F6E66696775726520484484
:202DB000433230313020746F20536C6F772053616D706C65204D6F646500C046436F6E6682
:202DD0006967757265204844433230313020746F20466173742053616D706C65204D6F64A2
:202DF0006500C04642555A5A4552204F464600C07F830100A1480100C8BC0200F412002022
:202E1000001900202DE9F843CC4C0F460646F80B80F0E881A07AB90F80F07581B80880F00B
:202E30006281F80A80F03B81E07910B1380980F03381206C002840F09D803809C0F09D80E3
:202E5000002501262570BE48667115F0B1F9284614F016FABB4904F170002A4615F00AFB90
:202E700004F1580090E8000314F084FFE378B0EB08004FEA103071EB09010905012B40EAB2
:202E9000010006D194F86810B0EBC12F01D8A378C3B3E670D24EA6F115010968A570090A95
:202EB00030D3606640F60900A08294F8210000F0F00040F0010084F8210094F8200000F0E1
:202ED000F00084F82000A56115F0CCFA06F6FF7211686FF0020321F00201116004F11401AC
:202EF000C6F8FB3FCE4AC6F8EB1F11688908FCD3C6F8FB3FD6F8FF1F41F00201C6F8FF1F1D
:202F100015F0A4FB2E4604F1580080E86000666612F094FB607818B9E068403015F0B8FAFF
:202F3000C7480660022013F015F811200BF0FAFFE068007C10B90E200BF0F4FF607A18B169
:202F50006572052013F006F8BE4965710878A57128B10D7004F1EC00042115F0A1FAB4F948
:202F70005000B4F95210884214BF022007200DF0E1F98EE0380980F08C80B80B77D2780B6B
:202F900029D2380CC0F0538104F13C0015F07CFAF0B1C16849680978022919D190F82700F2
:202FB000400915D2206C90F82700400910D3206C806840880028FAD0206C806840880128D7
:202FD000F5D0206C0026A0641920266415F050FA27F400472BE112F0D3FD38B1B569304697
:202FF0006FF4807100224FF00073A847964904F17000002215F03EFAB16800254FF0010881
:2030100040F602022572088884F8008082420AD0B0F5C15F07D00A8B4FF61F60104040F42C
:203030003470088306E00A8A4FF61F60104040F434700882757414F09DFED4F85421E3684D
:2030500004F5AA719A4208BFA846266E46B1864226BF301A401E801B01EB8801000B8860D8
:203070002566192015F004FA27F48057DFE004F1400015F009FA061C08D0706830B17568FB
:20309000F068B6F9241000222023A84727F40057CDE027F00807CAE00020E071F9E715F04C
:2030B000E1F9054604F13C0015F0EEF9061C15D0E06810B1783015F0CBF9F068E060284637
:2030D00015F0C4FA14F056FE2066604815F070F84FF4006104F1EC0015F0E2F9002027F48A
:2030F0008067E071A3E004F14C05284615F0CCF907F080FE284615F0C7F927F0020708B106
:2031100047F0020793E020B1042012F023FF0020A07215F0A7F9B1688046088840F6020253
:20313000824211D0B0F5C15F0ED00A8B4FF61F60104040F4347008830DE0C046A820002050
:2031500049C400007D0401000A8A4FF61F60104040F43470088204F1580090E80C00002BCA
:2031700008BF002A18D0042013F02AFBA0B1A56D14F000FE854226BF401B401E401B000BEA
:20319000F060F168708A401840F6C411F06081422CBFB0F5FA7FF160404615F057FA12F0CE
:2031B000EFFC98B1B56930466FF4807100224FF00073A84704F13C0015F066F9002808BF9C
:2031D00047F0020702D0192015F052F97569002130464FF080630A46A84727F0005726E0FA
:2031F0001500044015F03EF9014604F1440015F04BF90646B569A80814D29EB125EA0500FE
:20321000B061084615F022FA706870B16DB12A46F068B6F9241075680023A84705E0C04682
:2032300010100440084615F011FA27F4804727B104F1EC00394615F033F9BDE8F883C0464B
:20325000000004600F31002051C50000A9B000002DE9F04FADF18C0D1C911E93CC491D927D
:203270000A6806460DF156000260496841603046694612F09DFD00281F9004BF002022904B
:2032900000F0F78102200027B61CDFF84CB32090D34D2297304602A910F0C5FE5FEA000906
:2032B00000F0E48122990EA816220EF032FD9DF809707F1E00F082807F1E40F0CF81B9F16F
:2032D0000A0F40F3D681B61C316804A80160361D318805AF42F20B0039800DF1160111F0F5
:2032F000A5F8BDF81600BDF81410884200F3C181B61C16F8010B16F8017B16F8014B8DF829
:20331000380016F8011B8DF839700EAA8DF83A40304605F095FDBF4909780028064400F06E
:20333000A8811F9C012904F1020400F091814FF400500DF14E0111F079F80DF14E000DF1D6
:203350005601082213F050FE40B11C990DF14E00082213F049FE002840F07A8142F201009D
:2033700004A906F0BFF842F20B0005A906F0BAF842F205000EA906F0B5F80DF1390142F24F
:20339000060006F0AFF80DF13A0142F2070006F0A9F80DF13B0142F2090006F0A3F89DF8D2
:2033B0003B0028B1022840F0538142F2030001E042F20D000FA906F095F849E1B9F1040F40
:2033D00040F35781B61C16F8010B16F8017B16F8014B8DF8380016F8011B8DF839700EAA35
:2033F0008DF83A40304605F02BFD0028064400F040811C9806A905F0D1FE9DF836000028EE
:2034100040F00A819DF83B0000287AD195F83170002F00F0FD8095F83300874207D095F8E7
:203430008C000A2801D10AF05BFAA86B1EE0AF6B4FF400500DF15E0110F0F8FF13F0E0FEAA
:203450004FF0FF08229C2190A24695F83100A04240DCA86BB8F1FF0F08D008EB88040019C9
:20347000007912F02BFFA86B071923D195F831300746002B08BF229C19D05846229C406898
:203490001946D8467F1F7F1DFA782AB1491E04F10104F8D17F1D0AE0804795F83310491C6C
:2034B00085F83310D8F80810884795F83130A34200F094801C980CF02DFA38710120F870A5
:2034D000FC788DF8364038798DF83700229B8DF82330A1E0387911F063FB014608220DF16B
:2034F0005E0013F081FD40B138880104219814F0B5FF82453CBF8246A046641C7F1DA4B2D4
:20351000A3E795F83070002F00F0828095F83200874207D095F88C000A2801D10AF0E0F974
:20353000686B1EE06F6B4FF400500DF1660110F07DFF13F065FE4FF0FF08229C2190A24659
:2035500095F83000A0424DDC686BB8F1FF0F08D04FEA48140019C07F12F0B0FE686B0719A1
:2035700025D195F830300746002B08BF229C1CD0DBF80400229C1946D846203F2037BA7F6E
:2035900042B1491E04F10104F8D120370DE0C046600D0000804795F83210491C85F832108D
:2035B000D8F80810884795F83030A34216D02299384620220EF0ADFB1C980CF0ABF9F877A8
:2035D0000123FF2039462022BB770446787206A8FC720CF0E7FF1FE0F4120020612055E098
:2035F000000F0020F87F11F0DBFA014608220DF1660013F0F9FC38B17968219814F02EFFBE
:2036100082453CBF8246A046641C2037A4B297E764203BE0551200209DF836000EA916229F
:2036300040F004008DF8360008A80CF0BBFF1F9C9DF83B00A41C40B19DF84D700FA8394661
:2036500010F0EAF83F1A8DF8357006A80FF038FB20984844801C80B2209003E01F9C4E4423
:20367000B61CA41C209884423FF714AE2098022803DC229A6720114604E01F9A911C121A61
:203690002298921C1D9B19801E990A8023B0BDE8F08F70472DE9F04FADF1540D11F01AFF04
:2036B000032012F0CBFEC94C0025022004F11C0141F80C5F401E8D60FAD104F14000A946C0
:2036D000062701467F1E21F80C9BFBD14FF0080AC949A0F800A0C94A8160C949121D22F05B
:2036F0000303CF1A2762A361E361A66904F11C08944618460A46B14200F2A781B910E82765
:2037100000EB810121F8049C4FF6FC761F8006EA0C033746D21A00F1E80607EA020126615B
:20373000EC39A0F8E81028461BF09CFD6061C849D8F80000DFF81C8320610A6808F10C00A2
:20375000026049684160C7498346524613F04CFC28B9C54801685A46116040685060C3481E
:20377000C34FC0F8B070C0F8B850C0F8C850C14EC0F8CC50C04BC0F8B460C04AC0F8BC3057
:20379000BF4FD0F8B010C0F8C020C0F8C47009B1284688471BF0E2FD09F04EFAB94ECDF811
:2037B000389029460C2206F12C000EF0B2FAB64F0222ADF820A041F27073376340F61D0036
:2037D000ADF82220F18D7363102708430997616AF08508A8884700280CBF0A9F2F1C0120B5
:2037F000ADF82CA0616AADF82E000BA888479DF83000444620700D99616077B1D021397020
:2038100087F80190B87087F8039087F804903946BD600220FD6012F027F99C4918200122BE
:203830001BF0D6FCE220594614F0CCFB18201BF0BBFF60706068B046C8F80C000BF0B6FA2D
:203850009B4F08F18000A060D8F80C50904C4946A762F520E56014F089F88E4D05F10C0099
:2038700005F118010CF0D2FFA8600D2014F08CFA00B1CA460E2014F087FA08B94AF0100A14
:20389000162014F081FA08B94AF0200A152014F07BFA08B94AF0400A7F49A86814F0ACFCC7
:2038B0007E4905F12C00C82211F05EF87C486860BAF1100F11D1A06A78B1C2686AB1FF20FF
:2038D0004FF6FC778DF81000F81CADF8120004AEADF8140096E803009047724F07F1140030
:2038F00007F108010CF092FF7860484614F0A2FC4E46BD1E824605F8029F022068703046DD
:2039100014F017FD014678685246C9B212F000F9761C022EEFDB644907F120004FF4FA724A
:2039300011F022F8A06A002845D00769DFF87CA16FB10094514612A80A688988026012AE07
:20395000818096E8030001234A46B847A06A002831D0C26852B1514612A80B68898803608A
:2039700012AF818097E803009047A06A18B307690FB306208DF80800ADF80A0010AEADF850
:203990000C9002AD009695E803004A460223ADF84020B847A66ABDF840007769E08057B1B0
:2039B000BDF8400002AE401CADF8400096E80300022210ABB84728A014F09AFAA06A06261C
:2039D00000282FD007696FB302E0C046F41200208DF818600425ADF81A500EA8ADF81C90D4
:2039F00006AB009093E803004A462B46B84748B90E981930814615E04DF90100193100209B
:203A1000004B00208DF818604846A76AADF81A5006AE0F907C69ADF81C9096E803002A4606
:203A30000FABA047CDF8389048460EF039F8E0200C2113F09BFF13F035FE08F1040001216C
:203A500013F05AFEFEF770FFFCE726F8029B52E6C8FF01000019002054492053656E736FFB
:203A70007200C046700D0000F0120050080200206551010089560100C5560100E95A0100CE
:203A900079EE0000E810002020BF0200A5620000F80D002040150020094A0100857A0100C1
:203AB000357C010078160020F1130100A00D0000B80200202DE9F04FDFF8E0C292F808B0FA
:203AD00009AF88460646ADF1240D049338F07F05039206BF604600884FF6FF700590F08AA7
:203AF000800934BF002008203076F08AC00834BF102080207076F08A400903D260460E30E5
:203B1000007800E00020B076F08A41082CBF20240024000928BF44F010047568002108F0B3
:203B30007F08307D06916D1E02280EDB0C2808DC0C2803D1022044F40854069044F0030465
:203B500004E00D280CBF02200120044396F8880008B144F00804210900D328B1DFF8C892D1
:203B700099F8CC3013B908B1DF2051E121096DD396F88950DFF8B4A206F1240133891AF80A
:203B9000052007910AEB0001097908908918491DC9B2C918B1F5006F80F23C8100284CD05D
:203BB000049A039906F180000AF030FD0799002808603FD0806AB0F1FF3F39D07068002311
:203BD000401E8DB196F88A10524600F80119515D491EC9B241B1721892F87F20491EC9B250
:203BF000002900F80129F6D1079970660968896AB162090E00F8011996F82A1000F80119B3
:203C100096F82910089A00F8011996F8281005F0030500F8011902F0070141EAC5010170E8
:203C300071683289091AC9B270608918318105E0DB2700E0F3277770EDE00023F08A73700A
:203C5000C00828BF44F0100475686D1E336DA3B9B36D93B999F8E510012903D13089B0F5AB
:203C7000EE7F06DA200904D202290AD144F4005401E044F48054012002E044F408540220B0
:203C90000690DFF8ACA19AF8010001280FD013F021FF60B19AF83C0048B196F86B0004289F
:203CB00005D1022024F48054069044F4005444EA8834B8F1020FA4B20AD0B8F1030F10D17E
:203CD000ED1F09F1D801284614F0B0FB6D1E08E0B9F8BE00001205F8010999F8BE0005F891
:203CF0000109069802280CD0B8F1000F15D0BBF1000F0CD004990598814208D144F0400484
:203D10000BE0BBF1000F08D1B8F1000F05D00599081205F8010905F8011944EA8B24BBF128
:203D3000020FA4B209D0BBF1030F0ED10399ED1F284614F07BFB6D1E07E003990888001256
:203D500005F80109087805F80109BBF1000F05D00498011205F8011905F801093878F8B907
:203D700034480178307D0D2814D068B9306D28B999F8A800411C89F8A8100AE099F8CD00C2
:203D9000411C89F8CD1004E099F8B600411C89F8B610014605F8011904E0C046860C00208F
:203DB00044F48074201205F801092C7070683189401B7560C0B240183081200927D3B06D75
:203DD00000B130629AF83C0010B1307D0D281ED1726A12F1150002D114F00CF9726A916A89
:203DF000481C9062306A3289B162471B0092D21B019090B20290706A96F888202B461530E9
:203E100008F0FCF800281CBF7070071C07D10020707005E0E5277770F32013F075FDF8B2BE
:203E300009B0BDE8F08FC046CC0B0020140D00005412002085300020B0B50446BC480768FA
:203E5000ADF1480D002F00F0AC812078401E112800F2A781DFE810F06E0156013C012701D8
:203E70001F010801F100E300C300B2008D005D0053004200A5012A001C001200F86B0028B8
:203E900000F08F81684621460DF04EF9F96B86E1386C002800F085816846002101220DF03D
:203EB00038FF60788DF80000396C78E1F86A002800F07781684600210E220DF02AFFA11C0C
:203ED000684613F0EFFDA57BA1890022ADF80A1005B101228DF80C20F96A61E1B86B002890
:203EF00000F05F816846002102220DF012FFA5788DF8015060788DF80000B96B4FE1786B5A
:203F1000002800F04E81684621460DF00DF9796B45E1386B08B36846002114220DF0F9FE31
:203F3000A5788DF80150A3680193A289ADF80820A17B8DF80A1060788DF80000E57B8DF8EA
:203F50000B50237C8DF80C3094F911208DF80D2061690491396B684688476068002800F0C6
:203F700020810146F22008700020487011F07CFD17E1B86A002800F0148168460021242291
:203F90000DF0C7FE6078A11C8DF800000DF1020013F088FD04F10C0103A813F083FD257EDA
:203FB000E08A04F119018DF818500B22ADF816000DF119000CF0F6FAB96AF0E0786A0028A3
:203FD00000F0EF806846002102220DF0A2FEA5788DF8015060788DF80000796ADFE0386A4E
:203FF000002800F0DE806846002112220DF091FE658862796078ADF8025023798DF80520CF
:20401000E11D8DF80000A5798DF804300B220DF107008DF806500CF0C5FA396ABFE0F869CB
:20403000002800F0BE806846002101220DF071FE60788DF80000F969B1E0B86910B1204624
:204050000FF09EFFA07D002800F0AB80A07820B9A069002800F0A58003E0A069002800F019
:20407000A08013F06DF89CE07869002800F099806846002113220DF04CFE6D46A01C0168F7
:20409000406829600B22686004F10A0102A80CF089FA796983E03869002800F0828020465B
:2040B0000BF08CFB7DE0F86800287AD0684600210E220DF02EFE6078A11C8DF800000DF1FF
:2040D000020013F0EFFCA089ADF80C00F96866E0B868002865D06846002114220DF019FEC9
:2040F000A01C01686D46296040686860A07A0B2204F10B018DF808000DF109000CF052FABB
:20411000B9684CE0786800284BD06846002110220DF0FFFD60786588211D8DF800000B2270
:20413000ADF8025001A80CF03DFA796837E0C046081900203868A0B36846002119220DF063
:20415000E8FDA01C01686D46296040686860A07A410824BF01218DF80810810824BF012106
:204170008DF80910C10824BF01218DF80A10010924BF01218DF80B10C10924BF01218DF821
:204190000C1030F07F001CBF01208DF80D000B220DF10E0004F10B010CF004FA3968684643
:2041B000884712B0B0BD70472DE9F04FC54E4FF00008ADF1140DCB4DF068CDF808800028E7
:2041D0008DF80C8043D1D14CBF49843C2068814213D0BE49814210D0BD4981420DD0BD4941
:2041F00081420AD0BC49814207D0BC49814204D0BB49814201D013F0FDFE13F0E3F92168D9
:204210004FF0FF32012805D1C1F30330083806D0C01F01D0012A02D10120F07001E086F894
:20423000038012F07DFB286A00F1200120B913F0E1FE2846016A2031096806F1140088479D
:204250004FF4FA70F084A84FB7620624F462EA6992F82670DFB9A54892F8257001788F423C
:2042700015D04046342404FB002C9CF8267037B99CF82530401C9942C0B2F4D103E09CF858
:204290002500884203D1604611F0E6FEEA699849686A99C881E89900F078012814BF40466D
:2042B0000520DFF850B2944C08709BF8157127B990690068C4F8A40005E0D0690068C4F89C
:2042D000A40013F06DFA632004A910F0E1FA9BF8E720104612F072F9B4F896C082462CF072
:2042F000070C4CF0010CA4F896C0D4F8980004F18807812A40F00F00C4F8980001DB842AB0
:2043100006DB9AF80C10052914BF2421292100E0212184F89C10797D812A01F03F01797564
:2043300001DB842A19DB9AF80A306BB99DF810203F3262F305017975FA8A4FF6C07303EA97
:20435000020141F0180113E09DF8102001F0C00102F03F020A43114603E021F03F0141F05A
:2043700002017975FA8A4FF6E071114041F02001F9829AF80B209AF80C100A230CF0010C63
:20439000491D514391FBF3F1C9044CEA1141F9819AF80B101923890391FBF3F161F31C205F
:2043B000EB693861388B93F8242062F30200388393F824104FF6F77909EA000001F00801FB
:2043D00001439BF9D60039830EF0F6FF09F10801814218BFA4F8A200DAF80410DAF80030AD
:2043F000BAF80800EA69401E414303EB51004FF47A71B0FBF1F0A4F8A800106A0078A4F8F3
:204410008A8084F8AC00C4F88C80787B00F0F00040F00100787313F01FFFB0B99AF80B007C
:20443000364A9BF8E740B1FBF0F010709AF80B00022CB1FBF0F0C0B2B1FBF0F0707004D11C
:204450002F4802214170A8240470F0682C6ADFF8B89018B3404610F017FB30799BF8E7101E
:20447000884211D171799BF815212C6AF06891420CD1022142468DE80600E46C43463946B1
:2044900002AAA047EF6013E02C6AF0686168884701202B6A1B491C68087000E024681449D2
:2044B00006F1140348463A46A047F060686AA8629BF8E7009BF81571307105B07771BDE847
:2044D000F08FC0466417002000F0022000F0012000F00020008002200080012000F08200C4
:2044F0000080002040140020456F0100B30C0020D4300020CC0B002008100020B8180020C1
:2045100054180020E9190020B02B0020181300502DE9F04F09AFADF13C0D08900A9238887F
:2045300009911E46ADF81800101C08BF002000F08481002700F101094FF0FF3A4FF0010BC3
:20455000B8466CE1252940F063811078521C0A922D2818BFADF8068005D15846551CADF82B
:20457000060010780A9530281CBF4246434605D10A9908785A465B46491C0A912A28CDF869
:204590000080554616D1306804930A99CDF808A0C01C4B1C20F00300001D306050F8044C2F
:2045B0000A93002C0878009418D5ADF806B06442009413E044460AE0610001EBC4014018BB
:2045D0000A99A0F1300408780094491C0A91302801DB3A28F0DBCDF808A004932E282BD198
:2045F0000A9908782A2801F101010A9111D13068CDF80880C01C20F00300001D306050F8FC
:20461000045C002D48BF454608782B46491C0A9111E0454643460AE0690001EBC501401818
:204630000A99A0F1300508782B46491C0A91302801DB3A28F0DB02930AB1224604926C28CD
:2046500004D04C2818BFADF8048005D10A990878ADF804B0491C0A910BA9CDF80C800FABF1
:2046700007916428059300F08B80692800F08880BDF818C0752872D078286ED06F286AD0CF
:20469000702850D063283DD073281ED009980A990128A1F101010A9115D96B490C68B5F1D9
:2046B000FF3F03D0A84288BF6D1C00D8099D029508A80AA932466B46A047C7190A99039879
:2046D00001F1010974E040462AE030680A99C01C20F00300001D306050F8040CBCF1000FFF
:2046F00001F10109014608B955A00146079113F0C3FB0390B5F1FF3F5BD0A842C4BF281CBE
:20471000039056E03068C01C20F00300001D306010F8040C5D468DF82C000A990395584647
:2047300001F1010945E0082035680490E81C20F00300001D306050F8041C082210230FA8AF
:204750000DF0AAFF401E0790402101700A99079801F1010929E0082302E0102300E00A2348
:204770000A99306801F10109C01C20F00300001D306050F8041CAA42BCBF2A1C049210E0BB
:204790000A99306801F10109C01C20F00300001D306050F8041CAA42BCBF2A1C04926FF02C
:2047B00009030FA80DF078FF0790059D281A0390009C241ABDF8065000945DB906E008A87F
:2047D000202109AA12F05BF9009C7F1C641E0094F5D503980546401E039075B9BDF80600A8
:2047F000E8B10098401E009019D408A8202109AA12F045F900987F1CF4E70798411C079117
:20481000017809AA08A812F03AF903987F1CE1E708A809AA12F033F97F1C09F101094A46B9
:204830000A9812F8011C401C00290A907FF48AAE089808B14146017038460FB0BDE8F08F23
:20485000286E756C6C2900C0CC0D0000BA482DE9F84F0025B94CB749056094F8E20000281F
:2048700000F06381012800F02F81B54E02283CD0032840F05A8151F8250CD4F8B8100029E5
:20489000A0F5C060C4F8D400B8BF49420028B8BF4042814226DA4FF08057D7F8A4014568A6
:2048B000B4F8BC0030214FF47F42082300903046A847D7F8A4014568B4F8C00004214FF416
:2048D000F802122300903046A847D7F8A401B4F8D070456820214FF440620A233046009737
:2048F000A847012584F8D8501AE151F8258C13F071FC2F4600B901273946924F386800280C
:20491000FCD0B146012609F10409D9F82CA03E6009B113F065FCCAF30720C4F8BC0013F0DE
:2049300059FCAA4600B9B2463B68002BFCD0D9F800B0BAF1000F3E6001D013F051FCCBF31F
:204950008440C4F8C00013F045FCAA4600B9B2463B68002BFCD0D9F81C90BAF1000F3E60B3
:2049700001D013F03DFCC9F38120C4F8D000B8F5C061C4F8B81000F09C8094F8D80068B94E
:20499000C4F8D410D4F8C000C4F8C800D4F8BC70C4F8C470D4F8D030C4F8CC30D4F8D4103B
:2049B000D4F8BC30002954BF02206FF0010004F1C802176801EB41014018411000EB91716F
:2049D00007EBA1001060D4F8C810C4F8C43000291CDD1E293CDDD4F8CC0030B93429B4BF9D
:2049F00015391E21C4F8C81025E02A29BABFD4F8C8000B381E20C4F8C800D4F8C4003F2825
:204A1000B4BF401C3F20C4F8C4001FE0D4F8CC00032812D011F10B0FC6BFD4F8C8000B30C4
:204A3000301CC4F8C800D4F8C4000028C4BF401E051CC4F8C450032508E011F1150FC6BF51
:204A5000D4F8C8001530301CC4F8C800C4F8CC504FF08057D7F8A401B4F8C43030214FF407
:204A70007F424568364800930823A847D7F8A40104214FF400321123456831480096A847A0
:204A9000B4F8C860D7F8A40104214FF4F802122345682B480096A847D7F8A40120214FF48A
:204AB00040620A23B4F8CC60456825480096A84701E084F8D85040F2FF50404502D8801C9F
:204AD00040452DD208202EE051F8251C1E4F4BF2F5204843060A3868C0F3814001280AD110
:204AF00012F046F810F08CFD13F080FB3111C010484306EBE03694F8E50030B9134800689E
:204B100020F07F408019460801E084F8E5501048310C0660012741600E4D8760287808B9D6
:204B30000B2000E0052084F8E40004F043FFBDE8F88FC0462D400C402C500C40E40C0020DC
:204B500000A00C4000800C40B43F0050102009403C600C40F20C00002DE9F04FA54E376804
:204B70008346ADF12C0D17B913F044FA3768A248DFF89C920578002D3ED000253889796867
:204B90009E4B0795C400097818781034890906D340F6485191FBF0F1091901F5AF743B7DCD
:204BB00060438400352B0CBF2F1C4FF4FA570DF12601E8200FF06CFE9DF82600032808BF71
:204BD00044F620673068007D3C19352807D112F0E7F8014630686C300EF01EFE4443022046
:204BF0004F468DF8200007F10C000068069406A908F0D6FB8248057082490120824F087079
:204C10003978012902D0002102F0D8FB30680489456812F0A5FBDFF8FC812888000943D35A
:204C3000316840463C3890F83C70002F3CD082464A6A4F6E906AB0F1FF3F23D017B3431C34
:204C500093628862060E07F8016991F82A0007F8010991F8290007F8010991F82800387018
:204C7000086A00940190401B201A80B2029091F88820486A8B6A153019462B4607F0BEF999
:204C9000064600E0DB26DAF880706EB11FB9E4200CF01CFB05E05D4900200870E420394661
:204CB0008847002E40F0A280214628460CF030FD642009A90FF0ECFD464649463778DFF8D8
:204CD0005891087837B94846007809F051FF012805D088E009F04CFF012840F084804F4E78
:204CF000A01C87B20DF1250106F178000780E9200FF0CEFD9DF825104FF000084FF0020A66
:204D10004046012905D13C46C4F3022141F0180105E0241DA4B2C4F3022141F0080105F8CA
:204D3000011D05F8014DA6F86A009DF82470C6F88450002F0CBF3A493A497086CDF81080EC
:204D5000394C8DF814A096F83D00C6F8C01000F0F00040F0030086F83D006068C6F8801048
:204D7000804706F130052746304B254C0A90BBF1010F1CD0BBF1040F19D0BBF1000F13D04F
:204D9000BBF1050F2A460DD0BBF1030F07D148461030007811F012FC407B022808D006F157
:204DB000680205E0224B03E006F14C0200E02A46206A1749C56CC3468DE8000CC868114683
:204DD00004AAA8471B490880B968002809D41A4A92F900006836401C10700A98E6608847F4
:204DF00004E00A9888471A200CF070FA0BB0BDE8F08FC0469C0A002057180020B818002084
:204E1000401400203B190020E8190020183100206417002090120020A30C002008100020AC
:204E30004E9055550E7A5555F4120020A9A8000079DB000094170020421900202DE9F04F42
:204E5000AC4C04F128000068ADF1240D10F002F908B112F09BFBA248DFF89CA2DFF888B29A
:204E70000068A24E089011F087FF12F079F9E569A769B5F57A7F13D0C01B4FF47A72002326
:204E9000A5FB000103F09EF880464FF47A72002312F0E0FE2A46002303F094F8C01901E014
:204EB000A0EB0708A0618D488C49006820F00200086070688047DBF80010DBF804304546A7
:204ED0006918B1F57A7F0DD34FF47A72B1FBF2F2D2184FF47A73CBF804201F46B1FBF7F208
:204EF0005A43891ACBF80010B168884770688047DAF8041002466818B168CAF80400104625
:204F10008847DAF8000000285FD007464FF00009706880474FF000081FFAA5F3079083B98A
:204F30005FFA95F36BB93979E8B2884204DD79682846884209D20AE03879E9B2401A387138
:204F500008E079682846884201D3414601E07968091A7960B88878B9FB8853B9FB6843B1D0
:204F70003B8933B1B87A19460AF070FEF8687860B88808B9FB880BB13B896BB9B9F1000F67
:204F900004BF3868CAF8000003D03868C9F800003868B846074601E0B9463F68B16807987E
:204FB0008847B8F1000F0ED0B8F8043043B9B8F806302BB998F80A00B8F808100AF046FE32
:204FD000404612F0ADF8002FA2D144484349006840F002000860E06828B3804723E015F8DE
:204FF000060C2169A5F10C07032819D0E16A9DF816000978884210D115F8080C11F00EFBFB
:20501000B979012903D0022908BFA87000E02870002029460EF060FA05E012F0B7FA02E06E
:2050300009B12846884708200727ADF81000716AADF8127004A88847069D0028CFD0294806
:2050500000680088C8B1706880472649096800220D880A80B1688847089A0020294620706E
:2050700090470546FF202070706880471D4909680A8815430D80B168884711F07DFE0746B1
:20509000B7F1FF3F1CD0706807B9194F216AB94238BF0F1C80471C230546626AADF8023092
:2050B0000820ADF80000716A019268468847A16A3846491CA16210F085FAB1682846884762
:2050D00008200A27ADF808004FF0FF35ADF80A70716A039502A88847C5E6C04610E000E0BB
:2050F000B00D00000831002054190020F41200208EC2F52834170020EC3000202DE9F04F6E
:20511000A54C064600200F46ADF13C0DDFF89092ADF80C002068A44D017D252900F0108176
:205130006C3005A904F03AF8002818BFC0B240F0308120460068C18AC9080DD3007D03282B
:205150000AD09DF81F0038B99DF820004C463870B534207000201CE101A804A90AF06AFE83
:20517000A5F12F018B4691F82F30019A3468DBF808104FF47A7A504641F208155843891A23
:205190000AFB12000AFB01F1001B091B8D42C8BF002965DC854205DD002803DD346804F5AC
:2051B000915434609DF81F00002857D042F204000DF135010FF03AF912F032F804460698B1
:2051D0000DA9241A42F206000FF030F99DF834109DF81D00FF2904BF0A218DF83410FF28D8
:2051F00008BF0A209DF834206C499DF81C30D046B4FBF1F1801880B24843991008FB01F195
:20521000814298BF081C2D1805A811F0DCFD9DF81C203468B0FBF2F15143411A8BB25146B6
:205230004B4308FB02F1CA1AC91A121B091B8D4201D9002908D56942914216D2002A14D59A
:20525000B5FBF8F109B203E06900B1FBF8F189B232684FF4916303FB012405E0002004E0F1
:20527000306841F630342418346005460DF1120102A80AF0DFFD0298DBF80810B4FBFAF21F
:2052900010180290814203D99BF82F30834204D94B4603F15804267836BB9DF81C00551982
:2052B0000004A84298BF2D1A9DF81F00002808BF9DF8200016D09DF81C00B5FBF0F084B29D
:2052D0009DF833000FF06CFC9DF83120014620460FF0FEFB044611F063FD024608A92046FA
:2052F0000FF01FFA4C460DE0814204D8BDF81200401CADF812004C46BDF8120094F85B103E
:205310000DF0B2F83870244E84F8B5003068007D05287FF41FAF2348007820B112F0DAFB7D
:2053300000283FF417AF387803A9ADF80C0042F20C0004F0D7F8BDF80C00A4F8B00009E72F
:2053500068460DF10E010AF075FD3068009A2B7841F208144FF47A7101FB02020092594396
:205370008A1A944210DCA1F5FA619142BCBF00F5FA6030604C4694F85B10208F0DF074F8F8
:2053900001460020397002E039784C46652084F8B5100FB0BDE8F08F9C0A0020A086010032
:2053B000402D0020890C00202B2E00202DE9F04F002898461446ADF12C0D00F0EC8011F435
:2053D0007C1F40F0E58011F00F0F00F0E48007460591002006900A904FF0000A099055466A
:2053F00008954FF0010BCDF810B0054650460790059805990BEA000021EA0B014FEA4B0BE2
:20541000401E059100F0A480401E69D0801E56D0001F40F0B7801CB1276694F86B000690AC
:205430000720152607F8010B022301A907F8016B42F2010007F8013B0EF0F8FF684603A9F6
:205450000AF0F8FC06980EF07FFF0099019A3E4640180090824206D8801ABDF80C300090D7
:20547000581CADF80C00009B50085146814609041804030C19430004534610EB090041EB45
:205490000A0102F09FFDBF1D0090BDF80C309DF80C009DF8002006F8010B181206F8010B72
:2054B0009DF8011006F8012B9DF8023006F8011B9DF8032006F8013B0935327061E00220F6
:2054D000152607F8010B042307F8016BB8F1000F07F8013B0CBF099898F800002D1D4EE07D
:2054F0001CB1E76594F86B00069005201526049B07F8010B0DF10E0107F8016B42F204003C
:2055100007F8013B0EF092FF02A810F01FF806980EF01AFF02999DF80E209DF80E60069B39
:205530000918080200EB6200B0FBF6F002903E469DF808109DF8092006F8013B3F1D06F83D
:20555000011B9DF80A3006F8012BED1D337018E00320152607F8010BB8F1000F07F8016BF5
:20557000034607F8013B04BF0A9807F8010B05D098F8000007F8010B98F801006D1D07F89D
:20559000010BADB2059800287FF432AF2E4661E011F00F0F01D000205DE080468A460226B7
:2055B0004FF4803908F1020509EA0A002AEA090A4FEA4909B0F580301AD0B0F5803014D0B8
:2055D000B0F500300ED0B0F5802009D0B0F5002004D0B0F580102AD1072404E0062402E006
:2055F000052400E00424002704E00224012701E001242746A81C214600F030F847B104F06F
:205610000F04C0F30A0141EAC42141F4004105E004F07F0400F0FF0141EA042105F8011B6E
:2056300036180912B61C2970B6B245196D1CBAF1000FB9D1022ED8BF00260BDDB01E4FF60B
:20565000FE7708F8010BB819C0F3022040F0A00088F8000030460BB0BDE8F08FF0B504467F
:205670000846ADF16C0D401E6BD0401E0DD0801E00F00381401E00F0E980401E00F0DB806F
:20569000401E00F0A88000203CE142F2010007A90EF0CCFE42F20B0008A90EF0C7FE42F2B3
:2056B00006000DF165010EF0C1FE42F207000DF166010EF0BBFE42F2050019A90EF0B6FEAF
:2056D00004A80AF07BF905460DF1670142F209000EF0ACFE9DF86700002808BF002303D029
:2056F000022011F041F8034607A8006808A920600988271D3C46B81C218005F007079DF849
:2057100065609DF864109DF8662000F8011B9DF8674000F8016B03F0030600F8012B620753
:2057300047EA926104AC41EA8611012700F8011B9DF8672000942946019707F085F90A3021
:2057500099E042F206000DF165010EF06FFE42F207000DF166010EF069FE42F2040019A9B8
:205770000EF064FE04A80AF029F905460DF1670142F208000EF05AFE9DF86700002808BFC3
:20579000002303D0012010F0EFFF03469DF864009DF8657004F8010B9DF8666004F8017B6D
:2057B0009DF867209DF86770790704F8016B03F0030705F0070646EA916004AE40EA8710D6
:2057D000294604F8010B002700962046019707F03BF9001D4FE042F2150011A90EF026FEEB
:2057F00013AD42F2160029460EF020FE15AE42F2170031460EF01AFE17AF42F218003946D8
:205810000EF014FE11A801682160406860606A6804F108035A6028681860306803F1080134
:20583000086074684C60386801F1080528607A686A60202066E042F214000DF122010EF0A8
:20585000F5FDBDF8221002200A1258E009A8002120220CF05EFA42F2130009A90EF0E6FDA7
:2058700009A812F009FB024609A920460AF09AFE09A812F001FB80B244E042F20E0002A97D
:205890000EF0D4FD0DF10A0142F20F000EF0CEFD0DF10B0142F20A000EF0C8FD03A942F229
:2058B00010000EF0C3FD0DF10D0142F211000EF0BDFD0DF10E0142F212000EF0B7FDBDF847
:2058D00008009DF80B209DF80C709DF80D609DF80E509DF80A1004F8010B02F0010200122C
:2058F00004F8010B07F0010042EA400206F0010042EA800205F0070042EA4012042004F8EB
:20591000011B22701BB0F0BD2DE9F04F06469E48001D0068ADF1340D80470B900AA98220AF
:2059300005F0BEF99DF8280018BB00248DF828404FF6FF75ADF804509DF82800ADF80650A0
:20595000FF2108228DF8000002A812F0BBFD8DF81840D420694602F01DFD9DF82800401C5F
:20597000C0B28DF828000328E4DB82200AA902F011FD0020DFF808A2DFF808828DF828000A
:2059900081469DF828008DF8019069468DF80000D02005F085F901274D46E8B99DF80B309A
:2059B000012B07D19DF80A0020B90DF1020012F021F988B9747B002C0CBF052209224F4631
:2059D0009C4209D10DF1020006F10E0111F0F8FC002818BF012507D1002F40F0BF801DB993
:2059F000707F002800F0BA804C469DF828008DF8214008A98DF82000D12005F051F9002873
:205A100032D19DF82200FF282ED08DF800006946D42005F045F9002833D102A8311D0822EE
:205A300011F0CEFC00B330887788ADF80400ADF8067045B1307B9DF82810B7698DF8180032
:205A50000DEB81010F61D420694602F0A3FC75B1307F9DF82310884209D08DF8230008A97F
:205A7000D12002F097FC02E0641C032CBDDB032C74D14F468DF80070D420694605F010F9D8
:205A900028B1DAF808100B988847192074E002AB184612F0AFF84C4600B101242046341D61
:205AB00030B918462146082211F08AFC00284AD030887388327BADF804009DF82810ADF8BA
:205AD0000630002D8DF818200DEB810000F110000CBF4946B1690822016002A8214612F00A
:205AF00095F898F83C0030B1D8F88C201AB19DF80010204690474C469DF828008DF82140FE
:205B100008A98DF82000D12005F0CAF8E82807D09DF82200FF2803D0641C032CECDB10E079
:205B30009DF800008DF82490337F8DF8220069468DF82330D42002F02DFC08A9D12002F004
:205B500029FC032C02DB7F1C032F93DB032F05D1DAF808100B9888471A200DE09DF8280081
:205B7000401CC0B202288DF82800FFF60AAFDAF808100B98884748460DB0BDE8F08FC046F1
:205B9000F412002054120020F4120020F0B500216022ADF16C0D02A80CF0BBF8F2201AA996
:205BB00012F008FA954DBDF868001AA9A5F87400F32012F0FFF9BDF868000DF10901A5F82F
:205BD0007600E22012F0E6F9E88DADF81200410806D305F11801096805A80160BDF81200B9
:205BF000810805D3A91D098806A80180BDF81200C10807D305F11C0109680DF11A00016047
:205C1000BDF81200010908D30DF11E0005F1580128220AF0C7FCBDF81200410905D3686B9A
:205C30002F6B1390BDF812001297000B04D305F10801098819A801806D48007800280CBFD3
:205C50000121002101200CF0CBFDBDF8120041082CBF0F240B24810824BFA41CA4B2C10864
:205C700024BF241DA4B2010924BF2834A4B2410924BF0834A4B2000B24BFA41CA4B22046D2
:205C900010F03AFF071C00F0B18005260DF1090100F8016B0A68026049684160BDF81210E3
:205CB000083012F0C1FABDF81210844648080BD3BDF81410604612F0B7FABDF8161012F001
:205CD000B3FABDF812108446880807D3BDF81810604612F0A9FABDF812108446C8080BD385
:205CF000BDF81A10604612F09FFABDF81C1012F09BFA8446BDF812103E4AD388080951D343
:205D1000BDF81E10604612F08FFABDF8201012F08BFABDF8221012F087FABDF8241012F09E
:205D300083FABDF8261012F07FFABDF8281012F07BFABDF82A1012F077FABDF82C1012F0B7
:205D500073FABDF82E1012F06FFABDF8301012F06BFABDF8321012F067FABDF8341012F0B7
:205D700063FABDF8361012F05FFABDF8381012F05BFABDF83A1012F057FABDF83C1012F0B7
:205D900053FA194612F050FA117812F04DFABDF8421012F049FABDF8441012F045FABDF8DE
:205DB00012108446480909D3129960460FF007FE13990FF004FEBDF812108446080B04D32D
:205DD000BDF86410604612F02FFA05F12001224630463B4605F0B0FD0820ADF80260064D1F
:205DF00001972968ADF80000684688471BB0F0BD7A160020F80D002018130020E810002098
:205E10002DE9FE4F9B4692468946054612F02AFB02908C48353801680CAFA94208BF4168C3
:205E300001A84A4653460090284604F0DBF8834C061C13D194F8880140F0040084F8880198
:205E50000298C4F87C5112F001FC9DF8040002280CBF6FF002086FF00108ECE005F1780077
:205E700012F0F6FAB08CA4F85000B6F92480C6F808909AF80400C6F804B086F82600A6F805
:205E900024806F48F56097E80C00202106F110071940104087E80300002786F82770F068B9
:205EB00040680078022809D19AF80500012805D196F8270040F0100086F82700029812F0E2
:205ED000C5FB94F88901042807D1D4F88001B4F9841194F8862112F04EFA12F0C3FA814646
:205EF00094F8890130F004033ED104F13C000368D3B9314610F048F838B3A5F8C08096F811
:205F1000270040F0800086F8270085F8C270A07920B1207810B10120E071A771484612F0E9
:205F300095FB484800781FE004F13C00314610F02BF850B1A5F8C08096F8270040F08000AC
:205F500086F8270085F8C27048E0B4F9500000F6FF706FF31F30A4F85000484612F076FBB5
:205F70006FF00100BDE8FE8F02280ED196F8270040F0800086F8270085F8C270484612F02D
:205F900065FBB6F92400BDE8FE8F012811D104F1C80012F05DFA96F8270040F0800086F888
:205FB000270085F8C270206C0028E7D1484612F04DFB206C00282AD12078A76400BB207911
:205FD000012838D012F04EFA81466079A0B9B0680CF03EFF58B9207A012803D1484612F0B4
:205FF00035FB28E0484612F031FB04211FE004F1C80012F02BFAF1E7134901200870EDE7F4
:20601000012011F041FB192012F032FA13E0206CC0684068007802280DD1F0684068007864
:20603000022808D19AF8050028B94FF4004104F1EC0012F035FA4046BDE8FE8FA82000209F
:20605000FDEFFF9F312200200F3100202DE9FE4F0646307D01280AD196F917000DF0ACF92B
:206070004FF6FF71814208BFE82000F00681F07B834A20B91146491C0978022908DB0128CD
:2060900003D110460078022802DBF120BDE8FE8F346AB6F8289096F8347096F835B0B58B1B
:2060B0004FF000085FEA040A17D0764890F83C30002B2ED0416D00292BD004F0FF008847DC
:2060D0007049496D04B20AF47F008847001900B2001D00B2C43084B200E0C4240DB12D1DAB
:2060F000ADB269480078012809D147B16748C11991F8048010F80B002418641DA4B205EB61
:20611000090020184044801C80B210F05BFF071C02D11A20BDE8FE8F08EB09002B19388127
:20613000002D07EB030078600EBF0020E019801C00217422C7F8A00007F10C0012F0C2F9FC
:206150004C442D1907F13C00FF211022A7F84C5012F0B8F907F12C000F21102212F0B2F9B2
:2061700000243C707C707868716A328D0AF01AFA07F1800006F12C010B220AF013FA07F103
:206190008C00314611F0B3FB7089A7F89600307B87F89800707B06F10E0587F899002A68AE
:2061B00069460A60686848609DF800102046012908BF01209DF80110012908BF40F0040056
:2061D0009DF80210012908BF40F008009DF80310012908BF40F010009DF80410012908BF6C
:2061F00040F020009DF80510012908BF40F040009DF80610012908BF40F080009DF807103C
:20621000012908BF40F48070A7F89A00B07D87F89C00F07D87F89D00B28BA7F8A42022B1DC
:20623000D7F8A000B1690AF0BDF9B07F87F8A600306AC7F8A800B7F8A400C0B1D7F8A0008D
:20625000A8B17868401E7860F82101707868401E78600470B7F8A410B7F8A4607868401A5B
:20627000786039897018801C38817868B8650848007839460DF030F92046BDE8FE8FC0468F
:20629000CA0A002054120020980C0020140D00007C1300202DE9FE4FDFF82892074609F1A5
:2062B000040000688047DFF8C8A100248346002F0AF1020004703DD010F032FB6B4D214675
:2062D000FC22284612F0FEF8FF210822681D12F0F9F8FF21082205F10E00697312F0F2F852
:2062F0000227A84603224FF6FF710120AA77042329849E3505F8040F6B70AA707F1EEB70B7
:20631000F8D145464FF0050C022705F1F00606F8040F737086F802C07F1EF070F7D128464D
:2063300085F8F820AE3020F8181B20F8181B01800227AF70554695F83C0010B1286C00B111
:2063500080470CF0E3FEDFF8348108F1D60090F9000011F069FD10F0F9FA11F05BFD11F0F1
:2063700001FC11F0F3FBDFF80CA107270AF1240656F8040B00B180477F1EF9D13E48046024
:20639000446004614FF470018160C1600AF1040007680FB10EF0FEFF4B4800688AF80E403A
:2063B0004646C0B112E040460FF092FC029002A80EF0F0FF21E040460FF08AFC019001A85C
:2063D0000EF0E8FF14E068460EF0E4FF0BF018F900280090F7D12A480078012803D020466D
:2063F000014600F0EBFF2748274F047007F12408786A0028DFD108F10408B86A0028D2D143
:206410007C62BC622148A86187F82E40204BEB6187F82F401F4A2A621F49696287F8304055
:206430001E4BAB621E4AEA62214A6A601D49296320491D4FA9601D4B6F63214A6C701E4F2F
:20645000AB631E4BEF6058462B61D9F808106A61884706F1BD01522001F0B4F896F8D70090
:206470000DF0FAFE2046BDE8FE8FC046D4290020541200207C13002014190020CC0B0020E3
:20649000E8190020133100209C0A002097F3000025840100FD6E010079850000A1DA000088
:2064B00031730100A5800100D9BD0000E19C00003FC30000F1B10000413E01006501010063
:2064D00055300100F4120020083100202DE9F043071CADF1240D00F0F880F86B002800F089
:2064F000F480B7F84020002A00F0EF80007817F130014FF0000603D097F83810052902D0E0
:20651000002E00F0E280DFF8F491401E47D0801E33D0C01E1BD0801F40F0D7806CA011F07D
:20653000E7FCB7F84000012840F0CF800D2001224C4639468DF81C0007AB8DF81D20A41C9B
:20655000267005F0F9F969A011F0D2FCBDE0012A40F0BB80684C0725E0788DF81C50002852
:206570000CBF0121311C3046E1700CF039F9E07802228DF81D0028460CE0012A40F0A580E4
:206590004C46B4F860000122401CA4F8600004208DF81C00394607AB05F0CEF995E06846FD
:2065B00031460C220BF0B5FBB7F840000B2865D1FC6B14F8010B89F82C0023786078A41CC4
:2065D00003EB0023204611F097FB0546201D11F093FB8046387A4C4689F82800022806D0D7
:2065F000396804F1200001607A68426001E03888208403F00100D90828BF40F00400190999
:2066100028BF40F00800590928BF40F01000190B28BF40F40060E085834218BF0226B5F550
:206630007A7FADF8020016D33548A84213D3256311F078FB814611F075FB00EB092911F022
:2066500071FB00EB0920B0FBF5F16943401A0A300FF03CFF00E00226206BB8F57A7F0190D5
:2066700008D342F21070404504D3C4F8348011F06DFB00E00226606B029001E04C46012647
:2066900002258DF8016068468DF800500EF048F90DF10D009DF801108DF80C5011F0C4FDC7
:2066B000BDF8021011F0C0FD01990FF088F902990FF085F939460D2203AB284605F03CF91F
:2066D000B4F86600401CA4F8660009B0BDE8F08342757A7A657220436F6E74726F6C204D79
:2066F00053472052656365697665640042555A5A4552204F464600C0F80D0020E8100020CF
:20671000407E05002DE9F047DFF80CA20746AAF13500DFF8F8810068800880F0E78010F0A0
:2067300027FA814908310B6800261C17641C990D0AD2C0F13E0110F10A0F4FEAE101D8BF9B
:2067500008218C42B8BF0C1CDFF8C4C1990E0FD2590E0DD36246143A1168C1F304211629E1
:20677000A8BF20391268C2F30462162A0EDB0CE0634AD2F87C11C1F304611629A8BF203983
:206790001268C2F30442162A00DB203A61189146162905DA11F10A0FB8BF6FF0090100E0B6
:2067B0001521584C584D01F01F0242F4F85222802A6812F0030F18BF0126D20828BF46F07B
:2067D00002060FB146F00406424692F90740041B052C04DA9479B44208BF918866D00F28C9
:2067F000A0F10F0827DB08EB0014A4F1F0084FEA282EBEF1070F88BF4FF0070E7546062D6E
:2068100088BF06255CF82570042404EB850465462C59E41B04F0FF05F70824BFC4F307277F
:206830003D44B70824BFC4F307473D44770828BF05EB146501E00025AE465CF82EC0F70895
:206850000CF0FF0424BFCCF307273C44B70824BFCCF307473C44770828BF04EB1C64ADB276
:20687000A9EB0101A8EB0E277D43002905F1800504EB1524D8BF012103F0FF0334254D4387
:20689000A9B259434FF6FF73B1FBF4F18B4238BF191C802889B2918005DA10F1800FB8BFD6
:2068B0006FF07F0000E07F20D0719671194800681F2910604FF0000008D340F2FF128A4279
:2068D00006D24908401C8A42FBD301E01F219180124F0F39090940EAC10047EA0001CAF8BD
:2068F000FB1F0026CAF8FF6FBDE8F0870C490D4F424608200F60921D1070BDE8F087C046DB
:206910003C1100506E62084024220840FC3000209C130050082009403500094000E7A480DF
:2069300030100940FDFDA400AC3F0050804A2DE9F04F13680546ADF13C0D0DF12A0003608E
:20695000526842607B4C94F8B30005F1280105F12807002800F0E8806878002840F0E48065
:2069700011F0B8F8DFF8D091DFF8D48100B3042046466A68A873301D12780068042A00F045
:20699000958095F83000022812D14846007801280ED06A4905F1280002220E46203110F061
:2069B00023FB28B906F1160105A811F03FFD05AF686E002800F0B880012102AA0AF00EFA26
:2069D000002840F0B1809DF80800A873E86C40B139460DF11E0208ABFCF73AFC002840F050
:2069F000A38008A80090686E39460DF11E0306F065FC002840F0988048460078012851D099
:206A10004FF400500DF122010DF010FD0DF122000DF12A01082210F0E7FA38B10DF122004B
:206A30003946082210F0E0FA00283BD194F85900002837D0A66CB4F8445042F2010004A947
:206A50000DF0F4FC049A4FF000410020E2FB0610061C206D11F056FA86190498B04202D801
:206A70006D1C361AADB24746786880475FFA80F8206CB04204D1208FA84208BF002608D018
:206A900026642587002084F8350010F0C9FB0126E064B968404688470EB10BF0DBFA01208A
:206AB00084F85800002084F859003DE08B468047264C0D9095F8307022480A264FF000092A
:206AD000804610F807A0207AB84206D152462046594610F075FC012804D0761E04F10C0422
:206AF000F1D100E0A1465FEA09070FD198F80601164F461C810088F8066101EBC001F0B2AF
:206B10007F180A2804BF002088F80601384659460A2211F07BF80C48094900788968B8723C
:206B30000D9888470420A8730FB0BDE8F08FC046580D0000402D002055120020600C0020A4
:206B5000F4120020000F0020641700208E0F00202DE9FE4F0CAF89469A4604467D680292E8
:206B7000294604F0BBFD061C00F0EE803888F082DFF8F481347598F83C0018B1012C04BFBE
:206B90001520307506F1800029460B2211F03EF8012C04D00D2C1CBF7068401C00D17068CF
:206BB0003062002598F83C0035650028B5654CD0052C18BF012C43D14FF0040B86F86BB01A
:206BD000F08A86F86950C00932BF6148674816300078029986F86A000A6806F16C073A602B
:206BF0004B687B600889388110F074FF40BB06F16C0011F01BFC574F07EB8407386810F4FD
:206C10007F0F0CD086F82CB0386806F12C01012200F47F003063304603F020F9386810F091
:206C3000FF0F4FF003090BD02A2086F83C00386806F13C0100F0FF003064304607F04CFDFF
:206C500098F83C0008B10D2C13D00095029A534630464946FCF72EFF071C76D1E41F012CFA
:206C700003D8707E40F020007076304607F05EFE6BE010F02FFF294600B1012135483430A0
:206C900009B94FF00309052186F86B10016811F0F70F12D02A2186F83C1098F80120006838
:206CB00006F13C01012A00F0FF0030641CBF20F008003064304607F00FFD0095029A534618
:206CD00030464946FCF7F6FE5FEA00083AD1224806603489756801A964200DF0D9FD1F4E84
:206CF000A01C0DF1050187B206F178000780E9200DF0CEFD9DF80500012806D13C46C4F3F1
:206D10000220022140F0180006E0241D0421A4B2C4F3022040F0080005F8010D671A05F89A
:206D3000014DB9B2C6F88450AD1C28460AF0F0FC9DF8040000280CBF09480A48C6F8C0002E
:206D5000C6F88000474600E01A27F8B2BDE8FE8F850C00208007000098170020081000201C
:206D70004E9055550E7A555554120020980C00202DE9F043002B08BF002A10D10029BCBF15
:206D900000204FF0004106DB50EA01071CBF6FF000006FF0004109F0CCFABDE8F0835FEA26
:206DB000530898EA610803D50026404266EB01015FF0000913F0004E03D00026524266EB23
:206DD00003031C461546002C08BF8D429CBF2C1C0025070C47EA01470E0CB44208BFBD42F4
:206DF0009EBF240444EA15442D04070A47EA01670E0AB44208BFBD429EBF240244EA15649E
:206E10002D02470847EAC1774E08B44208BFBD4200F29280870847EA81778E08B44208BF5A
:206E3000BD427BD8C70847EA4177CE08B44208BFBD4265D8070947EA01770E09B44208BFDC
:206E5000BD424FD8470947EAC1674E09B44208BFBD4239D8870947EA81678E09B44208BF32
:206E7000BD4223D8C70947EA4167CE09B44208BFBD420DD8E60146EA5566EF01B14208BF6B
:206E9000B84201D3C01BB14159EB09094EEB0E0EA60146EA9566AF01B14208BFB84201D392
:206EB000C01BB14159EB09094EEB0E0E660146EAD5666F01B14208BFB84201D3C01BB141B3
:206ED00059EB09094EEB0E0E260146EA15762F01B14208BFB84201D3C01BB14159EB09093A
:206EF0004EEB0E0EE60046EA5576EF00B14208BFB84201D3C01BB14159EB09094EEB0E0E5D
:206F1000A60046EA9576AF00B14208BFB84201D3C01BB14159EB09094EEB0E0E660046EA3B
:206F3000D5766F00B14208BFB84201D3C01BB14159EB09094EEB0E0EA14208BFA84201D31F
:206F5000401BA14159EB09094EEB0E0EA34208BFAA423EBF2D0A45EA0465240A8AD3734691
:206F70004A465FEA080803D50026404266EB01015FEA480803D50026524266EB03031E465F
:206F900017460B46024631463846BDE8F083704701282DE9FE4F40F0EB80DFF80CB2DBF898
:206FB000DC00012840F0E1800220CBF8DC0010F087F901200DF048FF5FEA000805D001203E
:206FD000CBF8DC0010F08CF9D4E011F065FA6B4902900020086001200FF0F2FB012818BF8E
:206FF000002003D100200BF001FF0120644900900020644F08603868112011F009F90028DD
:207010000CBF00240124102011F002F908B144F002040F2011F0FCF808B144F004040B20E9
:2070300011F0F6F828B158480068584E016B308888470A2011F0ECF8002600B101264FF08B
:20705000805A0AF5DC75301C04D02868504E016B308888474F48012606602868816944F0E3
:20707000200088474C48066011F0CCF800F001010191400814D2494811F071F88146B9F134
:20709000040FF8D0B9F1010F05D1DAF8D80142684248032190474249086820F00300086025
:2070B0000020FFF72FFB2B683868986B8047019801280DD0B9F1010F05D1DAF8D8014268FF
:2070D0003648314690473649086840F0030008602B48066028684169204688470B2011F0D6
:2070F00097F820B12868294BC16A188888470A2011F08EF820B12868254BC16A1888884766
:207110002448032206602449CBF8DC2000230B602868416B204688470128F9D13868042086
:207130000DF092FE044615481E490660386808688009FCD30098012802D130460BF056FE7D
:2071500011F04EF808200DF07FFE07460298CBF8DC6011F077FA0CF01DFA10F0C1F857EAD1
:20717000040018BF4FF0FF3804E06FF0040801E06FF001084046BDE8FE8FC0460C400940C3
:20719000000222432C200940B8010010DE090000DA09000028200860800104430040034055
:2071B0002422084014100940E40C00202DE9F043044694F830900F46984615468B20ADF1FE
:2071D000340D0DF10A0103F06BFD8A20694603F067FD94F8250000283ED1B9F1000F19D1BF
:2071F000BDF80A104FF6FE70884205DCBDF80A1088422FD1694615E0B4F844009DF80A6026
:207210008DF80C0000128DF80D00BDF80A008DF80E601BE0B9F1020F09D0B9F1030F19D142
:2072300004F1280103A811F001F9092612E0207CC00934BFB4F84200B4F844008DF80C0092
:2072500000128DF80D00208D8DF80E00001205268DF80F00002013E002280CBF0526092607
:20727000012818BF04F11C0104D1892006A903F017FD06A9324603A810F0C8FC94F8260070
:2072900006EB0D01C8723A4603A831460AF0A6FE002840F08E80B9F1000F19D1BDF80A108D
:2072B0004FF6FE70884205DCBDF80A1088422FD1694615E0B4F844009DF80A608DF820008F
:2072D00000128DF82100BDF80A008DF822601BE0B9F1020F09D0B9F1030F19D104F12801CD
:2072F00008A811F0A3F8082012E0207CC00934BFB4F84200B4F844008DF8200000128DF8A6
:207310002100208D8DF8220000128DF8230004203E6881460BA9822003F0C2FC9DF82C10C5
:20733000307B8142D8BF9DF82C00002841D007460024722029460FF007FCB0689DF82C10E1
:207350002018C8F80000007881422EDD2B68C10001EB0011D8F80000C91829604278012A6F
:207370001FD0807828BBB9F1040F06D0091D08A810F094FA012816D017E008884B888DF84E
:207390002800042208A98DF82A3000128DF8290018128DF82B000AA810F012F8012802D0AE
:2073B00003E0807828B9002004E07F1E04F10304BFD1F3200DB0BDE8F08370472DE9F047E8
:2073D0007E4C804660680F46ADF1180D8047A246714E724D6F4C8146B8F1010F64D010F091
:2073F000E5FB00285BD063480078002857D162480078002853D16148007800284FD1604858
:20741000007800284BD15F480078002847D15E480078002843D15D48007800283FD15C48EE
:20743000007800283BD100200AF070FF002836D12078002833D1286A436CF068022104AAAA
:2074500098479DF8100050B3012FA0461ED0544C2A6AF06894F9001011F1020F05D0926B83
:2074700094F900109047F0682A6A4E4F97F9001011F1020F05D0926B97F900109047F068AB
:207490002A6A6FF001013970217001E0F0682A6A012188F80010D169884700206870DAF85B
:2074B00008104846884761E001200AF02FFFDAF80810484688473C4800780F2845D1207895
:2074D000012845D1DFF8E48098F8C2000028FBD1286A436CF068022105AA98479DF81400E9
:2074F000B14660B198F8C20048B9207801282FD10020012F20702BD010F064FB28E0DAF84C
:207510000400804700230222029380468DF80C20274E2270286A7381C76C8DE80C00254B8C
:20753000D9F80C000836314602AAB847002C01D510F060FD224991F90000401C0870DAF804
:207550000810EE604046884702E0384606F020FD2078194D022803D1287808B110F04AFD51
:207570002878012802D020780228FCD006B0BDE8F087C046143100201631002018310020C5
:2075900015310020173100203A1900203B1900203C190020E9190020641700204014002080
:2075B00038190020391900206D0C0020B02B002008100020953E0100E8190020F4120020F1
:2075D000421900202DE9FE437B4E80460F46B8F1450F06D13046342210F018FBC6F89C6078
:2075F000E7E00FF08AFF3B2808BFF42000F0E280724C04EB8004A07810B9E178002938D000
:20761000E178814208BFFB2000F0D480B8F1580F25D0B8F1600F1BD0B8F1E00F0FD0B8F1F0
:20763000E80F05D03A78904220DC91421EDB20E006F1E7003978007881421AD1B9E097F944
:2076500000000BF0B9FE4FF6FF7181420ED010E038880A280ADBB0F5804F07DA09E038884D
:207670008F2803DB46F2B041814202DAE820BDE8FE83544D6868804781462078627839467F
:207690008019943010F0C2FAA968484688474046503800F08C80801E73D0401E00F0848016
:2076B0008D387CD0401E63D0401E75D0801F1BD00D387ED10E2096F815718DF8000017B1C8
:2076D0001B208DF8000096F9D6109DF90000884203D0E0206946FFF775FF10F061F896F832
:2076F0001501002841D164E0032096F8E7108DF8010081294FF005008DF8020006DB8429B5
:2077100004DA8DF8010008208DF802009DF8010096F8B910884204D04F200DF10101FFF756
:2077300051FF9DF8020096F8C510884204D057200DF10201FFF746FF214C94F83C00A0B118
:2077500010F0C8F988B1226F7AB1022000278DF803000DF103018DF8047042F21B00904771
:20777000226F42F21C0001A990470CF0D9F820E096F8D7000CF070FD01281AD01A20BDE80A
:20779000FE8396F8BD0018B902200EF029F810E0022010F087FC0CE010F0D8F909E096F931
:2077B000D60010F041FB04E010F0DCF901E010F031FB0020BDE8FE83CC0B00209C02000006
:2077D00054120020F41200202DE9F04705461F461646ADF1380DD1B16C480C7802684FF04E
:2077F000010808FA04F0024211D069607EB13046002106F0E1F8AE6010F034FE644C814640
:20781000601C0078022804DB484610F01FFF0020B8E0002870D103F0F9FF5E49086840F05C
:20783000020008600AA810F00DFCDFF86CA15B499AF802000AAA0C9004F1EC000DF094FF36
:207850000AA810F0DFFB002619210AAB8DF830609AF80000524A0B9004F170000DF09AFBA2
:207870000AA810F0EFFB9AF803004E490AAA0C9004F590700DF078FF0AA810F0C3FB9AF871
:2078900001008DF830801A210AAB474A0B9004F18C000DF07FFB4549324604F1C800134672
:2078B0000CF0AEFF424810F083FC424A3346042104F128000FF084F94FF6FF70A4F8C4002F
:2078D00084F8C760E67026716671A671E67126720523667204F15802A672314684F8683039
:2078F000304682E803004FF4FA71C4F85C11324AC4F860116078167004EB8001401CC1F832
:207910005451C0B26070484610F0A0FE44461FB903AF384610F04CFA386828607868E8601C
:20793000387C2874B8696C742862788A6882234EAE61EE616E61F86800B1A861786900B126
:20795000E861B86800B168610021A02205F128000AF0DFF905F1400000210EF089FF6846D6
:2079700010F025FD1649029505F1780000226B460CF046FF134905F19C0000226B460CF0A0
:207990003FFF28460EB0BDE8F087C046D4210840A820002000200940A60D00007D7C010010
:2079B0007D04010051060100993D01003D65010049C400006D4501000E310020CB73000006
:2079D00025770100198401002DE9FF4707467878002840F0E78097F8961002291CBF03299D
:2079F000E82097F88B108029C8BFE82097F88C10092901DB0A2900DDE82097F88D1009B1D6
:207A1000042905DB8029C0F2CC80862980F2C980002840F0C780684C04F1E70000788842C7
:207A300004D007F18D01E820FFF7CCFD07F18C01E720FFF7C7FD07F18B01E120FFF7C2FD95
:207A500007F198015020FFF7BDFD97F8960002280CD04FF6FE70A4F8B40007F18E0104F1BB
:207A7000AA0010F0E3FC07F18E0504E007F18E052888A4F8B400514807F180010B2210F034
:207A9000C5F84FF001080220A7F816802946387501A80FF02CFF97F89A60B7F8989078684B
:207AB00007F19A01002EA0F1010078600CBF002040464E780EB140F002008E780EB140F06E
:207AD0000400CE780EB140F008000E790EB140F040004E790EB140F0800079684A1E7A6046
:207AF000374B08703E7D7968481C3862701E0026087038893E65801C38811878BE65002822
:207B100040D04FF0040A87F86960F88A87F86BA0C00934BF94F8B90094F8E20087F86A004C
:207B3000296807F16C0001602B8903816C6844600FF0D0FF30BB07F16C0007F18E0110F08B
:207B500075FC204C206810F47F0F0CD087F82CA0206807F12C01424600F47F003863384636
:207B700002F07CF9206810F0FF0F0BD02A2087F83C00206807F13C0100F0FF003864384652
:207B900006F0AAFD00963846832101AA4B46FBF791FF061C02D1384606F0C8FE301C01D175
:207BB00006E0E82078701820387038460BF068FF0090BDE8FF87C046CC0B0020382F0020E0
:207BD00090120020880700002DE9FE4F724C074694F83D00002800F0DC80784EB7F84210D2
:207BF000BD3EB6F8BA00884240F0D38007F128000FF05EF8002800F0CC80B046002598F841
:207C1000BD0084F83D5010B102200FF0B9FB6348007810B101200FF0B3FB387C400905D371
:207C300010200FF0ADFB802010F044FA20200DF0D7FD634B1E4606F120000CF035FB7A6837
:207C500051781078334600EB0120C0F30321C0F3003684F8391000F00F0184F83A60C0F3F0
:207C7000031684F83E1098F8E30088F8C0600F2804D0884202DDD67806B9014688F8A110C5
:207C900098F8A1A083F84050BAF10F0F09D194F83B0002287DD10EF0C5F907F075FBBDE84E
:207CB000FE8F3F480078012803D001202946FFF785FB3C484068804700900FF021F83A4809
:207CD000DFF80091DFF8E4B0066898F8A12099F80030D9F80400311A980091FBF0F05BF8CA
:207CF00022100DF097FBC9F804605BF82A0001912F4EB060F0600CF0EFF8019831680EF08F
:207D1000C5F909F039FC274900988968884794F83B0002280DD128480CF0C6FA98F8A12053
:207D300034F812004FF470719140091A22480EF0FBFF98F8C060388929460BF00DFB206315
:207D50000F2E14D098F8A11094F83900B14208D0401C6FF00F05B0408101A1EB80016D184E
:207D700005E0401CB0408501A5EB8005A03D6563022004F1200584F8380028460CF094FA9A
:207D90000C48A062616B28460EF0CEFF102010F091F9BDE8FE8FC046BC160020432F002002
:207DB000E8190020F412002080140020C40A00001419002029180100F82F0020890C00205F
:207DD000E82F0020B81800202DE9F047064637680C465FEA0208ADF1180D14BF00214FF099
:207DF000FF3107F14800814610F0B0F8002818BF0B2040F0DF80002565707148FC60B8F123
:207E1000010F057004D065700220FC600EF016FB2078012840F29080801E012857D9801EFF
:207E300001282CD9801E012800F2B88010F01AFB8246A078009021782846062908BF012070
:207E5000019001200290A068228A6368E16806F011FB0746504610F0F9FB002F40F0A080AE
:207E7000B8F1000F02D00FF029FE02E030460EF0E3FE002800F0878010F004FB21E010F0EC
:207E9000F1FA012782460097A168A278606824782B46042C08BF3B1C07F0E2FD0746504661
:207EB00010F0D4FB002F7BD1B8F1000F02D00FF005FE02E030460EF0BFFE002863D00EF070
:207ED0005DFA3E49C1F8B0510D60074668E010F0C9FA8246E08A0090E0680190208B02905D
:207EF000A0780390207D04900121059122782846022A08BF081CA368E178626802F0F2F9B4
:207F10000746504610F0A2FB002F49D1B8F1000F02D00FF0D3FD02E030460EF08DFE002826
:207F300031D00EF05BFA071C3AD1E078A168E28A236909F0F3FDC8E710F094FA8246E08AFE
:207F50000090E0680190208B0290A0780390207D049001200590277807B90546E17862680C
:207F7000A368284602F07CFA0746504610F06EFBB7B9B8F1000F02D00FF0A0FD02E03046D6
:207F90000EF05AFE08B9142014E00EF00FFA071C06D1E07821690CF0BFF896E74FF0FF370A
:207FB000B8F1010F02D002200DF0D4FF484610F06FFA384606B0BDE8F087C0465045024010
:207FD000123100202DE9F0411C4615468C4208BF854282BF00230022E5E0002C08BF002D63
:207FF0000AD100290EBF00286FF000006FF0000100F0E1F8BDE8F0815FF000085FF0000E26
:20801000002C08BF8D429CBF2C1C0025070C47EA01470E0CB44208BFBD429EBF5FEA044476
:2080300044EA15445FEA0545070A47EA01670E0AB44208BFBD429EBF5FEA042444EA156423
:208050005FEA0525470847EAC1774E08B44208BFBD4200F29380870847EA81778E08B4428A
:2080700008BFBD427CD8C70847EA4177CE08B44208BFBD4266D8070947EA01770E09B44288
:2080900008BFBD4250D8470947EAC1674E09B44208BFBD423AD8870947EA81678E09B442DE
:2080B00008BFBD4224D8C70947EA4167CE09B44208BFBD420DD8E60146EA5566EF01B14218
:2080D00008BFB84201D3C01BB14158EB08085EEB0E0EA60146EA95664FEA8517B14208BF15
:2080F000B84201D3C01BB14158EB08084EEB0E0E660146EAD5666F01B14208BFB84201D363
:20811000C01BB14158EB08084EEB0E0E260146EA15762F01B14208BFB84201D3C01BB14173
:2081300058EB08085EEB0E0EE60046EA5576EF00B14208BFB84201D3C01BB14158EB0808FF
:208150004EEB0E0EA60046EA9576AF00B14208BFB84201D3C01BB14158EB08084EEB0E0E2D
:20817000660046EAD5766F00B14208BFB84201D3C01BB14158EB08085EEB0E0EA14208BFE8
:20819000A84201D3401BA14158EB08085EEB0E0EA34208BFAA423EBF2D0A45EA0465240A8A
:2081B00089D3734642461E4617460B46024631463846BDE8F0817047F0B542F20400ADF17B
:2081D0001C0D0DF115010CF031F942F2050005A90CF02CF9654C66489DF81510A066642081
:2081F000414321666349C4F884109DF814104843E0676148C4F8A0006048007880B942F24B
:20821000020069460CF012F968460EF069FF04F15C000BF03BFD04F134000BF055FF27E07F
:2082300042F2030069460CF001F90EF0B9FD0546684629460BF0F0FA2D1A04F1780084F821
:208250005B500BF023FD04F134000BF0C9FC012742F20200694684F854700CF0E7F8684689
:208270000EF03EFF04F15C000BF010FD84F85870434800780EF0A2F9407B022804BF0120B1
:2082900084F8B40094F8B80000286DD13D4D0021302205F10C0009F03CFD204600213322E7
:2082B00009F037FD38482862384FAF6105F114000BF0ECFC42F21B000DF116010CF0B6F8E5
:2082D0009DF816000DF1160185F8300042F21C000CF0ACF89DF816109DF8160085F831100D
:2082F00095F83010012641B148010EF031FD686308B910F0B1F895F8310040B100EB8000C4
:2083100080B20EF025FDA86308B910F0A5F8204905F13C000A270A684B6802607F1E4360FF
:2083300000F10800F7D1002195F8307085F88C1047B1686BFF220346C2777F1E997703F1F6
:208350002000F8D195F8317047B1A86BFF22034602717F1ED97003F10500F8D1281D0622F9
:2083700009F0D7FC84F8B86007B0F0BD402D0020A5430100A5FD0000D7830100551200202F
:20839000B30C0020000F002075BA0000002A7515680D00002DE9F041704B714ADFF8B8819A
:2083B0000C46D128014610DCD12878D0713800F0B080401E00F0A980401E00F0A2801138F5
:2083D00010D04C3800F0868007E0D23853D0401E40D0401E33D0401E28D008460FF0BFFDF1
:2083F0000B2802D1F420BDE8F0815A4D05EB8005A97809B9E87850B1E878884208BFFB20D1
:2084100000F0A6802278914269DC904267DB554E7068804729786A78074640464018214619
:208430000FF0F4FBB1683846884790E02178022955DA1846641C042200EB810084E0207809
:2084500003284CDA1746C100241D182201EB0011781879E026783046022840DA2C2505FB93
:208470000680611C102239300FF0D0FB616905FB0680C1646BE022786178022A2FDA0229F1
:208490002DDA40462C2301EB42064F1C03FB0205022285F8387000EB4600A23018E022786E
:2084B0006178022A1BDA032919DA2C23404603FB020595F830309942A4BF4B1C85F830304A
:2084D00002EB4202891801EB4101032240189030A41C39E020786778022800DA17B1E8202B
:2084F000BDE8F08141462C22C5197E1C02FB00136A0083F8286002EBC50288180A227C3060
:20851000E6E724B3184608221EE004B3104648221AE0B4B9404600F17C04A0F1080200F1C0
:20853000900300F1A201022042F82C4F9360401E116104F10A0403F1090301F10401F3D1AC
:2085500005E040465822243021460FF05FFB0020BDE8F081040B0000D4290020C82A00209E
:20857000802A0020F41200202DE9BC4305466D4800880021820804D2B5F89A20D20828BFB5
:20859000E82110F0600F04D1B5F89A00800828BFE8212889B0F5006FA8BFE82195F8980065
:2085B00030B995F89400002808BFF52100F0B580002940F0B280DFF87091D5F8A800DFF8C8
:2085D000708199F83C1010B9012903D02BE0002900F0A2800FF07EFA68B9D5F8A81040460E
:2085F000BD3041F002010078C5F8A81018B141F00801C5F8A810D5F8A81011F0FF0F05D07C
:208610002A2085F83C0001F0FF072F6411F47F0F07D00420D5F8A87085F82C0007F47F0027
:20863000286399F83C10002069B3404995F894700B6804226FB925232B750968C98AC9092D
:2086500034BF98F8B91098F8E21085F86A10891C08E015212975D98AC90934BF98F8B91063
:2086700098F8E21085F86A1085F86B2005F18C0785F869003B6805F16C010B607C684C60F9
:208690003B890B8101E00121297595F89C70EF760446AC65B5F89A102C6595F89D30E982D3
:2086B0006A682B7795F82C702A620F2F09D00246B5F8A40005F12C0100B90122284601F073
:2086D000CDFB28BB95F83C10FF2901D1AF6D27B105F13C01284605F0FFFFC8B9009495F8E2
:2086F0009810B5F8963005F18C022846FBF7E2F9071C0CD12889B0F5006F03DA284606F08A
:2087100015F904E0E520687028460AF037FC3846011C02D1BDE8BC831821284608F0F2F903
:20873000BDE8BC8388130020541200209C0A0020CC0B00202DE9F043894614460546ADF1EC
:208750002C0D69460DF034FB5FEA000800F0C480AD1C0226284602A90BF065FC071C00F0F7
:20877000BB809DF80900814509D0F6197D1908F10200B61CAD1CB6B2B042EBDCACE0401E2B
:2087900005F1020500F08B80401E52D0801E38D0401E2BD0401E24D0401E18BF622040F019
:2087B000AB80202F40F0988028686F6805F10801206004F10806676001F108050A684B6813
:2087D000326004F1100773602A6868683A6005F108067860306804F11801086073684B60AC
:2087F00089E0022F78D12888208084E0202F73DC20460021202209F08CFA3A462046294697
:2088100077E0042F68D12888AD1C208015F8010BA070287800F00100E0702878C0F34000CF
:2088300020712878C0F38000607128784011A07161E00A2F50DD0DF112000021162209F0E8
:2088500068FA28682D1D20602988271D42F20B00398004A90BF0EAFDBDF81000A188884218
:208870003ADCA81C10F8011BA17110F8011BE17110F8011B217210F8011B0123C1F3C202EB
:20889000A2720DF1120200F0DBFA28B39DF82700A0819DF81670E78104F1100026E0042F64
:2088B0001ADD0DF112000021162209F032FA15F8010B207015F8010B607015F8010BA07068
:2088D00015F8011B0DF112020023C1F3C2002071284600F0B5FA08B967200DE09DF8270025
:2088F000E0809DF81670278104F10A000DF11601112207F057FE00200BB0BDE8F083704708
:208910002DE9F84F4FF0000B6A4C8DF800B00FF015FD2279684DDFF88C81012191404FF638
:20893000FF725218024095F83C00628120B36A6F12B342F21A00694690475948677906781A
:20895000A6B19FB99DF8006086B1D5F8980068B18047454659492A78097830B1678908318D
:208970004A43B0FBF2F0C019608167799DF80010608907FB01006081A078002840F08B8046
:20899000494E306AC06B80470746484D648998F80010336A687808304443D86B8E00804761
:2089B000D8F80410464B401AD91C0A78B0FBF6F03C2303FA02F1B0FBF1F24A436978801AEB
:2089D00001F10803B0FBF3F25A43821A01F108038A1AA21802F10809B0FBF3F25A436B7852
:2089F000801A091A6418083406FB0471304C04F15807387894F87420616500F0F00040F006
:208A10000200387003F1080080B206FB001104F13C063078A16300F0F00040F002003070C7
:208A300002F0F00084F874000FF060F8AA46454630B16868A16B88423CBF0120031C00D3ED
:208A50005B469AF80100297823B91C2008F03EFCBDE8F88F3A7802F0F0023A705B46636512
:208A7000327808308D0002F0F00242F00302327082B205FB02F0A063307940F018003071FF
:208A90004FF4FA57A76401FB09F0A4F84E300DF089FFBDE8F88F04F039FABDE8F88FC0460E
:208AB00010310020B818002040140020641700200810002054180020541200206517002060
:208AD000890C00202DE9F04F684C2068ADF12C0D002840F0C78004F124063068002800F0FB
:208AF000C18063480078022800F0BC80624D281D006880470A90606AB046074678B35D4E0C
:208B10004FF0000A4FF01D093B7D0820711E11F8012F9A421ED0401EF9D140463946524660
:208B30000CF0B8FE787E30F07F0005D194F82F00401E84F82F0004E094F82E00401E84F8CC
:208B50002E0087F8019057F80CBC38460AF016FA5F4602E0BA4657F80C7C002FD4D13520A1
:208B700007F008FE454EA968002849D1452007F001FEA96800283DD1D8F8000038B1017D29
:208B9000252904D050F80C0C0028F8D110E078B196F8580050B3684601A907F04BF938483D
:208BB00000990078001F884213D8012086F85500152007F0DFFDA96848B10A9888472068C1
:208BD0000DF106016C3000F0E9FA58B10FE00A9847E0252007F0CEFDA9680A9888470020A7
:208BF00086F85500042000F0ABFB3BE0192000F015FE37E00A98884708200BF025FE31E0A2
:208C10000A98884796F8B400B8B10EF0D9FA317800290EBF0921491EC9B201EB81017118B5
:208C3000D1F802100FF01AFC42F21071814292BF00206431081AC0B200E000206968002829
:208C500008BF0620D9D0C6F8980088470446D6F8A010D6F8980006F1A8020DF013F9A96860
:208C7000204688470BB0BDE8F08FC0469C0A002097150020780D0000F4120020402D002000
:208C90002B2E00202DE9F843664C002605466676687D0628A4BFE8216176A97D0E2903DD68
:208CB00003281CBFE8216176032805D15E48008840083CBFE820607695F8280008B1E820F8
:208CD0006076E87D092801DB0A2801DDE8206076287E08B1042805DB802801DB862801DBD5
:208CF000E820607604F11807294638460DF09CFA291D112207F12C0007F054FC95F8280059
:208D100004F11809002804BF84F86060A87D04D095F8290084F86000688DA4F85600687EAE
:208D300084F85800A87EDFF8048184F85900E87E822784F85A00287F98F8D76084F85B00CE
:208D500098F8E63084F85C70394F84F85D6005F11D01E763042684F8406098F8E72084F89D
:208D70005E3009F1490084F85F200B220EF04EFF607E00284ED1687800284BD1287EA77E8B
:208D90008DF800000FB1EA20607605F11701E720FEF718FC94F8600028B1287E022808BF24
:208DB00001208DF8000098F8E7009DF80010884203D0E8206946FEF705FCA77E1E4C601C8C
:208DD000007808B10FF016F9B8F8BA0019490880C7B1032F12D0052F05D0012F03D0022F27
:208DF00001D00FF007F9022060700BF0E9FF4FF6FF70A8F8BA001149088005E00BF0E0FF0F
:208E1000032000E0012060702720287030460EF0B7FA01E02A20287028460AF031FEBDE84B
:208E3000F883C0467C2F002088130020CC0B0020C58001006E1700208030002092140020A3
:208E50002DE9F04F154601F00708C1F3C2074FEAA119044683460C22ADF1240D0021684603
:208E700008F057FF6248B8F1000F36D0B8F1010F7ED1228801A9A6780A80E41C8E7014F81E
:208E9000011B01F00F018DF8081022880DF10A031A80BDF80A30A41C4FF0000C6B75019E40
:208EB000CDF818C04168B14207D1017A9DF80820914202D14189994208D006990C30491CF6
:208ED00006290691EED96046614601E0017840788DF800108DF8010022E014F8013B14F825
:208EF000016B8DF8003000228DF801600C38079210F80C1F994202D14178B14207D0079958
:208F1000491C06290791F3D91046014603E04168027A4089687501918DF80820ADF80A0010
:208F300003A806F04BFD9DF800109DF80100B8F1000F11D0B8F1010F1AD1019904989DF8F5
:208F500008209DF81460484086EA02010918BDF80A20BDF8160004E09DF80C2051409DF83F
:208F70000D205040401803D1EF701FB1022F05D0002039E02188281DA41C0180B9F1010FA1
:208F900027D0B9F1020F2CD1BDF80A10281DC91DCA10214607F006FBBDF80A00C11D04EB53
:208FB000E104F0B1401E811000EB5171C910C9B26D182B798710012600EB577121F0070178
:208FD000401AC0B2401C06FA00F0FF301840287107E0291D20460AF0FDFF207804EB8004B5
:208FF000641CA4EB0B04A0B209B0BDE8F08FC046981400202DE9FE43654C664D0E46B0097A
:2090100059D3624800F1280980464DE00178D0290EDBD02909D181783970C17879700179E9
:20903000B97085687D60C168B9600EF0A1FF47E004F1080528600AF023FD28460CF0AAF975
:209050003EE0884798F83010491E88F83010A9688847009801788DF80410A0604778CFB153
:20907000DC2F0DD0DD2F0BD0E42F09D0F32F07D0DE2F05D0DF2F03D0E82F18BFDB2F0BD195
:2090900004F006FD9DF80400162805D168460CF081F901E00AF0F4FC9DF80400162803D083
:2090B00004F108000CF076F948460CF011FE002869680090C5D1F00BA846C00305D0364F7A
:2090D00008F09EFA00280090A0D1700905D32E208DF8040001A80AF0D3FC700805D3252098
:2090F0008DF8040001A80AF0CBFCB00805D326208DF8040001A80AF0C3FCF00805D3272095
:209110008DF8040001A80AF0BBFC300905D329208DF8040001A80AF0B3FCF00908D3002033
:209130008DF805002D278DF8047001A80AF0A8FC300A08D300208DF8050030278DF80470F2
:2091500001A80AF09DFC700A08D300208DF8050035278DF8047001A80AF092FC6068D8F8A6
:20917000041080B18847616800270091D8F8081067608847009804F1080630600AF080FC2B
:2091900030460CF007F90020BDE8FE839C0A00207C130020F4120020481900202DE9F04F96
:2091B0000546824660480E460178ADF1140D0EF091FC5F4C00283FD0DFF8808108F1040016
:2091D0000068012914D0287A022835D15749504602220F4620310DF007FF38B903208DF89B
:2091F000080007F1160168460FF020F9EA4623E095F8089014F809A080470A274FF0640BCF
:209210008E340390207A484506D15246204629460EF0D6F8012804D07F1E04F10C04F1D151
:2092300004E00027F772A07ABB463073D8F80810039888475F4672E021464FF0000864276A
:209250008B468D6B91F8310086F81E804446D9460AE099F800106D1C2034ADB234E099F84A
:209270003100641C6D1DA4B2A04217DDE8780028F5D028790BF094FC514608220DF0B4FE8E
:209290000028ECD1E878B077288800047060287986F80B80F077A87847463073DBF8344026
:2092B000002F08BFBB46C5D086F81E8042F219000DF10A010BF0BAF80DF0A2FF83461D4827
:2092D0000178642745468146A94228DDA07F0028BFD0E07F0BF064FC514608220DF084FE68
:2092F0000028B6D1E07A022803D0E07A58B1612710E0616858460FF0B1F8BDF80A200E4938
:209310005143814201D9474604E0A07F6C2740F00800A07730462146202207F043F93846CA
:2093300005B0BDE8F08FC04655120020600C0020000F0020300F0020808D5B00F41200200F
:209350002DE9F8435B4C0746207808B10EF052FEA0465A49624D584C0120012F88F800006C
:209370000E682868A77024D9BF1E47D0544A7F1E11D07F1E34D07F1E2FD10021C08A617138
:20939000C0093ABF101C2938101C0078207108460EF0A8FE59E01046401D00780DF00EF9DF
:2093B000407B022802D1002007F04AFF0CF088FE4BE0C68A002143486171F10934BF90F895
:2093D000B91090F8E210217197B990F897707FB10229C4BF022020710AE00EF00BFE34E033
:2093F00090F86910617190F86A0020710027A771FFF786FA286848BBBDE8F883DFF8C89070
:2094100099F800008700F06B8047D9F804103C22401AB0FBF7F0B0FBF2F151436278401A7D
:209430009101A1EB8201091AF06B3C311FFA81F98047264907FB0900086791F8740000F060
:20945000F00040F0020081F8740028682049097879B910B90EF0CEFD28684168087800F006
:209470002000E0708878E0710878800901D20EF0F9FEA078032818BF022819D1154D6868EA
:209490008047A17802290CD013490F7817B913490F7837B1022188F80010A9688847BDE81F
:2094B000F883832188F80010A968884709F062F9BDE8F88318310020541800206014002010
:2094D000AE0C0020CC0B0020B81800200810002010310020F4120020143100201631002030
:2094F0009C0A00202DE9F84F884605460EF040F801464FF6FF70884210D042F21C0BAB45FA
:2095100009D0ABF10100A84205D01A38A84202D0001DA84205D10EF0DDFA10B16820BDE858
:20953000F88F534C480000EBC1002418D4F8027017B9D4F8066016B3D4F80610B94208BF18
:20955000692000F093806078401E12D0401E09D0801E14D1D8F80000874200F2818081424E
:209570007ED30CE0B8F80000874279D8814277D305E098F80000874272D8814270D33D4FAD
:2095900078688047ABF11A0A2B463B4E0090A3EB0A03012B25D90A3B012B14D9DB1F3DD19F
:2095B000207862780021301808F0B3FB637840460EF062FC834298BF181C02D940460EF0AE
:2095D0005BFC02462BE00DF0EBFBBF68B8F80010884243DD207862784146301806F0E2FF05
:2095F00023E00DF0DDFB8146404649460AF014F9BF68A9EB00005FFA80F9B9F1000F2DD05D
:20961000207862784146301806F0CCFF1B485146A94218BF401C80F8009006E062782078C0
:209630004146301806F0BEFFBF680AF11900A84204BF002086F887005846A84213D196F891
:20965000870096F886104218322A01DC08430AD1022086F88600302586F887500098B8472F
:209670006A20BDE8F88F0098B8470020BDE8F88FC4000000F4120020FC2D00209A2D002027
:209690002DE9F04F0746880FADF1140DC0F0B98000200AF0C9F960485B4E4FF0000900F173
:2096B0001408C8F80090012048F81C6C0DF0E8FD56480EF07DFD564DBC68CB4640F60A062F
:2096D00005F1140095F82010EA7895F82130A5F816908246C5F818B001F0F0010680012A50
:2096F00085F8201003F0F000A4F8029040F0010085F8210001D17B7CABB1B8680088A6F169
:209710000801814208D0B0F5C15F05D0218B4FF60F400840208304E0218A4FF60F40084065
:20973000208287F81190B868694604F05DFB68460EF080FC3346D91F4A1C00E03446666815
:2097500036B13088834203D0814218BF8242F5D1C4F804A0607B00F0F000607305F13C007E
:209770000EF092FE8068008881421FD082421DD03E8D06B397F8340097F83560C7F82CB072
:2097900000F0F00087F8340006F0F00040F0010087F8350007F12803AB619AF80D00A7F8EE
:2097B0002A9000F0F0008AF80D0004E0DA4605F1580080E80006B9680A8A4FF6FF30104037
:2097D0000882D8F800000028FBD0687AC8F8009070B901200CF0F4FF01280FD0607B00F0EE
:2097F000F00040F0010060730A480EF0E1FC05E00BF07EFF0028FBD00BF098FFB86848F8F6
:209810001C0C05B0BDE8F08F01010E04152E0000A8200020312B0100081004402DE9F843EE
:209830005E4D804695F83C00002798B16A6F8AB1D5F8940070B142F21A0069469047D5F837
:209850009400804730B19DF8000018B1B8F1E10F08BF0127524A02F1E70000780CF0AEFE40
:20987000407B02280CBF05260126514C2068002800F09280B8F1000F914675D0B8F11B0FE0
:2098900002D1017D05296FD1B8F1E90F2CD05FBBB8F1E10F16D10EF063FA90B12068C18A53
:2098B000C9080FD299F8C810817699F8B6104A1C89F8B620406881703046FFF741FDBDE88A
:2098D000F8832068B8F11C0F1DD1216A002950D08847344900200978206001295CD00146D5
:2098F000FDF76CFDBDE8F883F1200EF00DF82768B87E50B90EF034FA20B12068C18AC90858
:2099100001D2CFE7206847462FE07868398907F0FFFE78680088000905D395F83C0010B121
:209930000BF09AFF2768F88AC00811D3387E00F07F003876387D032803D1787E40F0040015
:209950007876F0200DF0E0FFE168206888470FE015490126B87E0E70401EB876F0200DF0BC
:20997000D3FF12480078A8E70027477009F006FB2068C08A000A0AD395F83C0018B999F8E8
:20999000D7000AF069FC99F9D6000EF04DFA0020206010200EF08EFBBDE8F88354120020D7
:2099B000CC0B0020E819002010310020561800209C0A00202DE9F843614C5A4D5A4EDFF8A6
:2099D00070815E4F94F8E4100846401E0B2864D8DFE800F07B2C43062343062343067664E5
:2099F000042907D001220A2945F8212C14BF0220032004E0202045F8210C0120024684F8E8
:209A1000E200002045F8390C0827C5F8FF7FC5F8F37F45F8392CBDE8F883052914BF09202D
:209A30000620002784F8E400376075E094F8E170383D0120002FC5F81B0004BF06200021F9
:209A500002D00021F160032084F8E400032045F8010C3160306880085ED294F8E4103348E6
:209A7000012703290ED00068456800216022052300914046A84794F8E400062814BF0A2023
:209A90000720CFE700684568002160220523022000904046A8470420C4E7FEE72548264F3C
:209AB0000026012506600E203D6005F03BFA02200CF050FA84F8E45084F8E360BDE8F883F8
:209AD000002038600C25786024E04FF08059D9F8A0010168202088472C3D0F2045F8010CCD
:209AF00041F61D56C5F80360D9F8A401466800214FF4C0720723022540460095B047D9F89E
:209B1000A401C66800214FF4C07207234046B0470120386084F8E45004F178000EF096FCBF
:209B3000BDE8F88339400C4038600C40A401001000A00C402C500C4004800C4034600C4033
:209B5000E40C00202DE9F04F8146ADF11C0D01F05DFE0DF037FD0026012804D10DF042FF23
:209B7000022808BF012651490868C0F38150012806D151F80C0C0127010E07FA01F006435C
:209B90004B4800780DF07CF94A4D2C46286038B1FF2204F1400107467F1E01F8012BFBD18C
:209BB000D9F800104FF0000801F0FF02FE2A1CD0CC4601F0FF0342460127FF2B0ED09842D0
:209BD00003D907FA03F31E4201D002206AE001F0FF0143EA0808611881F840205CF8041F0E
:209BF000521C01F0FF03FE2BE7D1092005F084FCC4F8049004F1240001210CF039FE23682C
:209C10003BB3002794354FF0040BBA460120B840064218D118EA000F04BF07F0FF0141F4BE
:209C3000C04104D0E01990F8400059F82010224803F07AFDF8B24FF0FF310DF0EDFC23689F
:209C5000C5F800A001E0C5F800B07F1C2D1D9F42DCD304A80EF0D6F9184D194A28781021C2
:209C700004AB059004F108000BF094F968460EF0E9F900276A46686803971249029004F15A
:209C900060000BF071FD104951F80D0C012620F4F85040F4005041F80D0C0C4DC1F8FF6F57
:209CB00038462E6007B0BDE8F08FC046B43F005011310020C4270020007FC767880D0000B5
:209CD00045760100F54B01000D3009400800094056482DE9F04F0068ADF1140D08B90EF0C7
:209CF00089F9534C2078012803D000200146FDF765FB574F07F13C004E4CDFF83CB1DFF8D5
:209D10003CA1DFF83C810078A8B9606880478446584607784FB95046A168077837B98322B8
:209D3000404602706046884767E0A16802224046027060466DE04748463000780CF03EFC94
:209D5000407B022804D14448C01C007807F078FA0CF0B6F93B4D286A3B4E016CF06888470E
:209D7000039060688047B946029058460778002F46D150460078002842D1D9F888100020EB
:209D90008847F42001A90AF083FD304F9DF904000399884219DCB879B8B9A1680298884724
:209DB000B878042801D00EF025F904214046BE790170D9F88810701CB87109B1032088472D
:209DD0000320788103F0A2F824E0832140462A6A0170536CF0686A4600219847B5F906001C
:209DF000BDF90010884214BF002001200AF04CFEA16802988847387A307008F0BBFC09E00F
:209E1000022140460170A16802988847D9F888100420884706480078012803D00020014621
:209E3000FDF7CCFA05B0BDE8F08FC0469C0A0020E8190020F41200201431002016310020A0
:209E500018310020401400206417002054180020541200206D0C0020561800202DE9FE4FDE
:209E700007461046002F00910CBF4FF0E80B4FF0000B002900F0AC80BBF1000F40F0AA80CE
:209E900060B17868401E7860F82101707868401E7860002606703889801C3881009C4FF05E
:209EB00000094FF0020ADFF83881CDF80490083C14F8080F00F00F010F2900F08680012897
:209ED00021D004287BD1454890F83C00002876D0424D6068696D8847061C26D03889B7F8C6
:209EF0004C103018801C81421FDB7868AD6D6168019B3A46801BA847B8B178683D89801B42
:209F1000786076195AE00098019E042309EB0001C91C11F8010FFF2841D021283DD13889EF
:209F3000B7F84C200B30824202DA1A20BDE8FE8F7868B8F8D020401E786012120270786883
:209F5000401E786098F8D02002707868401E7860019D057098F8D2007A68107098F8CE205E
:209F700078681201401E786042F00F02027098F8C0C098F8A1207868401E786042EA0C1232
:209F900002707868401E7860212505707868F61DB6B2401E7860052505705B1EB9D178685B
:209FB000C6F30121401E786041F0880101707868401E7860067038893618B61C3E81BAF17E
:209FD000010A09F108097FF473AF7868B86501E04FF0E80B5846BDE8FE8FC046541200205A
:209FF000CC0B00202DE9F04F5D4C054600208A46ADF12C0D80461746B4F952100A93DDF8A6
:20A0100050B084F88901B4F950008BF80080401A40F6F87101400829A8BF012080F29280B3
:20A03000B4F95000401CC0F30B030CF04DFF0646D4F87C01B384854207D194F888014108E5
:20A0500024BF00F0FE0084F888010A98006800B940463062387B00F00F00022814BF40460A
:20A07000B868BAF1000FF06175D00AF19C000DF0B9FF002865D128460BF066FD051C1AD1DE
:20A09000E36BC3B109F02CFE236C08902BB1216CE26B304605F06EFF38B9236C5BB9E26B35
:20A0B0003046694605F066FF28B1012384F88931E06B3060E66394F88991B9F1000F4AD140
:20A0D0000DB9E56B95B12A683046294605F052FF18B92D68002DF6D108E00223286884F8E4
:20A0F00089312246306092F889912E60B9F1000F31D10A980179504604F022FA014601297E
:20A1100026D094F88901002825D1012923D0E16B09B10868D0B9387B00F00F02022A1AD11E
:20A13000C01118D141B9206CA8B1216C3046424605F020FF28B10EE03046424605F01AFF04
:20A1500048B902208BF80000464604E00968E0E7042084F8890130460BB0BDE8F08FC0461C
:20A17000A82000202DE9F04F5D4E7068ADF11C0D80474E4A924611784D4D04919AF80020A7
:20A19000B168012A0BD001248AF8004088472878012805D020460021FDF710F900E0884709
:20A1B000454C444FDFF81491E06807F1B001814206D1494691F90000002818BF002762D1F2
:20A1D00070688047002205903E4BA7F8B22003F13C000778002F07BF4FF48600111C384805
:20A1F00020219046384A9B461378CDF808809B0904D21278120938BF012200D302228DF848
:20A210000C20226AD76C8DE8030034492F4A304B106802AAB8470028B768A08030D449462D
:20A2300091F900009BF801302A4A401C08702B49002B92F90000E16000F1010010700CBFD0
:20A2500042468022B4F84400234B4FF67F7101400A431043A4F84400B3F8BA00B3F8BE1092
:20A27000A4F852000822A4F8501003F1D80104F1470318460DF0CAFC0598B847012702E0E7
:20A290000598B847474670688047B16817B9049A8AF8002088472878012803D000200146EB
:20A2B000FDF78CF8384607B0BDE8F08F3A190020E819002008100020401400204319002001
:20A2D00000004F8C541200201531002070170020F114000042190020CC0B0020B8100020A1
:20A2F000F41200202DE9F04F8A4609AF4FF08051ADF11C0D90463D69059001F5D870049091
:20A31000D1F8B001D7F808B04169069327208847524C4FF00309143CC4F884970126C4F8E0
:20A330007C67C4F880970220C4F8FC06F868C4F8080430460EF05CF8D4F808040008F8D2DD
:20A35000D4F88C07800F28BFB14655D2681E41460C238DF800000DF1010011F8012B5B1E8C
:20A3700000F8012BF9D1022D19BF0020011C98F80C1000208DF80D108DF80E008DF80F0006
:20A390000099C4F83C15019BC4F84035029AC4F84425039BC4F848353968BAF1020F4FEA0C
:20A3B000C542A1EB0A08A2F5002106D34FEA4A52A2F580026FF315021143264A0A43C4F823
:20A3D0004C258246C4F85085BBF1000FC4F854A5214DC4F858B511D02E6078682060C4F871
:20A3F00008B030460EF004F8D4F88C078008F8D3D4F88C07000801D3CA4627E0C4F884974A
:20A41000D4F88C0710F0030FFAD1D4F8800720F00200C4F880073F7D47B1049F3868016AE6
:20A43000272088473868016927208847C4F87C670598C4F8806748B12E6006982060C4F896
:20A450000880C5F800642062C4F82880504607B0BDE8F08FC80104200000484218400240DB
:20A470002DE9F04F894609AF4FF08051ADF1240D9246059038683D69079001F5D8700490F5
:20A49000D1F8B001D7F808B04169069327208847504C4FF00308143CC4F884870126C4F872
:20A4B0007C67C4F880870220C4F8FC06F868C4F8080430460DF09CFFD4F808040008F8D226
:20A4D000D4F88C07800F28BFB04653D2681E51460C238DF800000DF1010011F8012B5B1EFE
:20A4F00000F8012BF9D1022D19BF0020011C9AF80C1000208DF80D10019B8DF80E000099E2
:20A510008DF80F00029AC4F83C15B9F1020FC4F84035039BC4F844254FEAC542C4F84835C6
:20A53000A2F5002106D34FEA4952A2F580026FF315021143254A079D0A43C4F84C2581466C
:20A55000C4F85055BBF1000FC4F85495204DC4F858B511D02E6078682060C4F808B030463B
:20A570000DF046FFD4F88C078008F8D3D4F88C07000801D3C14624E0C4F88487D4F88C076B
:20A5900010F0030FFAD1D4F8800720F00200C4F880073F7D47B1049F3868016A27208847AE
:20A5B00038680169272088470598C4F8806740B12E6006982060C5F800642062079FA7603E
:20A5D000A762484609B0BDE8F08FC046CC01042000004842184002402DE9FF41044666686E
:20A5F000A7680D460DF03EFF3178012903D10EF02DF8002091E0012131700EF027F82878D4
:20A6100070706878B07068687060A868B060E868F06028693061287D3075687D7075A87D8F
:20A63000B075A869B061287F3077687F7077A87FB0774FF00008C6F82080C6F830804546BB
:20A6500075627563B562B56386F82C50102386F83C3086F82D5086F83D50786804F04CFFD0
:20A67000204604F0BDFC204606F01CF970B92C480068C16838688847786804F053FC0DF089
:20A69000F1FE35700DF0E2FF2C4645E068460DF0B9FC0094387B234A0190B9686B4606F133
:20A6B00080000AF077FC68460DF0CCFC00941E4938696A46029006F19C000BF055F8B07849
:20A6D00030B906F1D00029460CF0D2F817483061707830B906F1EC0029460CF0C9F8144859
:20A6F000F06068460DF063FE01958DF800501149029406F584700A226B460AF081F8B96932
:20A71000FA6906F140000DF018FC0B4A06F16C00042123460CF054FA20460090BDE8FF81D3
:20A73000D001001035C20000C95B0100AF830100A7830100A90B0100058101002DE9F04329
:20A750004E4CDFF83C8194F83F600027ADF1140D002E57D198F89660002E53D0C768007AD4
:20A77000454600F00701C0F3021900E0BF1C0E46701EC1B24EB17A783878B5F8BE6000EB11
:20A790000220B042F2D1022710E005F19406443600E008374846411E5FFA81F9A0B3304607
:20A7B00039460DF07BF80028F3D0032794F83F0040F0040084F83F0002A80CF08DFA01207D
:20A7D0000CF0DEFD04F13401872000F069FA04F13C01852000F064FA04F13D01862000F080
:20A7F0005FFA04F13E01882000F05AFA0120009004F134060196B5F8BA30394602AA052072
:20A81000FCF7A6F9002F35D198F8A1100F2931D0404690F8C0208A422CD090F8BD000028C4
:20A8300028D11848007828BB17480078012803D001200021FCF7C2FD16490C46606880474D
:20A850002146124C94F83B20022A11D194F83820FF2A0DD00E4A176857B9576A47B98968AB
:20A87000884704F1200009F01FFD06F0D5FF01E08968884705B0BDE8F083C046042F00203E
:20A89000CC0B00208A130020E8190020BC1600209C0A0020F41200202DE9F8434D4E84463F
:20A8B0000120002430704C484E4D04704B48DFF83081047005F14E000088B14614EA0307A6
:20A8D0004FF0020606EA020608BF002E13D120464FF0E04710401F4008BF002803D11D20D5
:20A8F00006F0F4FC4FE0454695F90000401E28700DF074F947E0424692F900303A4E5B1E4F
:20A91000137043F20842824207D06F8E931C834203D0BA4218BFBB4216D130460830006879
:20A93000826C60469047008843F6030181420AD004F0B4FB98F9000000283ED098F900003F
:20A95000002837DD41E06F8EB5F86A1043F60400884220D0B8421ED0B5F84E2090421AD0B0
:20A97000B1F5505F05D0080B0BD31D2006F0AEFC07E01E480168304601F5C071016004F027
:20A9900057F90DF007F998F90000B0B198F9000000280FDD19E016480078022812D00328BD
:20A9B00010D004F07BFB98F9000030B198F9000000280ADC0DF01EFB07E020460146FCF78F
:20A9D000FDFC02E0204606F081FC89F80040BDE8F883C046E81900203C1900203B190020C2
:20A9F0004219002008100020581400200C010021561800202DE9F84F994692468B4606461B
:20AA10000DF030FD4E4C0090B4F95210B4F950000AAF401A40F6F871014008297CDAB4F99F
:20AA30005000401C6FF31F30A4F85000B4F950800CF04AFA054606F178000DF009FDC5F886
:20AA500008B085F826A0C5F80490A5F824803D48EE6097E80C00202100271940104005F1F4
:20AA7000100383E8030004F13C0085F827700368002B43D129460BF087FA002844D0A6F891
:20AA9000C08095F8270040F0800085F8270086F8C270A07920B1207810B1A7710120E071E1
:20AAB00000980DF0D3FD206C002845D12078F0B92079012840D00DF0D5FC0646607988B910
:20AAD000A86808F0C5F940B930460DF0BFFD04F1EC0004210DF0E4FC2EE004F1C8000DF0CD
:20AAF000B5FC02E0184901200870304622E001200CF0CAFD19200DF0BBFC1DE004F13C0042
:20AB100029460BF041FA50B9B4F9500000F6FF706FF31F30A4F850006FF0010809E0A6F889
:20AB3000C08095F8270040F0800085F8270086F8C27000980DF08AFD4046BDE8F88FC04639
:20AB5000A8200020FDEFFF9F0F3100202DE9F04704466568A6680F46ADF1200D0DF082FC06
:20AB700095F8DC10012903D10DF070FD002085E04FF0010A85F8DCA00DF068FD3878287072
:20AB900078686860387AE860706804F0B5FC204609F098FCF868676828B9A06890F814904F
:20ABB00090F8158003E090F8009090F80180B9F1FF0F15D0B8F1FF0F12D0324840EA090180
:20ABD0000491FE23069340EA080004A9059007F1980005F01BFEC7F8A400D7F8A40070B905
:20ABF000294800240460294F3C60706804F09AF90DF038FC85F8DC400DF028FD3DE0494641
:20AC10000D220BF009FED7F8A40041460E220BF003FE68460DF0F6F9307B00946B46B1682A
:20AC30001B4A019005F110000AF0B4F968460DF009FA306900946A461649029005F12C00C3
:20AC50000AF092FD05F1600051460BF011FE287830B905F17C0000210BF00AFE0E48686027
:20AC700000202872C5F8BC000C4AC5F8C0000421234605F1C8000BF0A3FF204608B0BDE812
:20AC9000F087C04600200084042800401004054225C10000D93801006F83010075800100DB
:20ACB0002DE9F0410C4601467138022840F29780133825D04D4F4C387BD0401E62D0401EEF
:20ACD0004AD0401E38D04A4D401E2AD0401E1AD008460DF044F906460B2E11D0414D686861
:20ACF000804780464048B100425CBF1840184278394620460CF08AFFA968404688470DE03A
:20AD1000F420BDE8F0812278022A68DA2946601C483101EB820104220CF078FF0020BDE8C0
:20AD3000F0812278032A5ADAD3002946201D03EB02131822C918EFE72678022E4FDA2C25DC
:20AD5000601C05FB0671102239310CF05FFF05FB0670C06C6061E1E7207802283FDA2C21A7
:20AD700001FB0070667890F83800B04237DD23786278394602EB430201EB42010222A23167
:20AD9000A01CC9E72078022829DA2C2101FB0070667890F83000B04221DD20786278394642
:20ADB00000EB4000121802EB4202891803229031E6E72078022812DA2C2101FB0070667864
:20ADD00090F82800B0420ADD6278207839468018420002EBC00289180A227C31D0E7E82027
:20ADF000BDE8F081F4120020040B0000D4290020802A0020F8B5071C00F0A180B86840F6DA
:20AE1000030120264A1C02E04068761EF6B260B15EB10388994218BF9A42F5D1F9681CC868
:20AE300028311CC149C881E849007868BA690026BE6168B3F96848680078022818BF42F0EA
:20AE5000020297F82700002300F00700401E09D0401E04D0801E08D14FF0805304E04FF0F9
:20AE7000804301E04FF00053324697F82700000908D397F8270010F0070F03D04FF08070AC
:20AE900032430343B7F92440084621467C68A0470DF0E8FA2A4C0546B4F95200401C6FF3F6
:20AEB0001F30A4F8520004F14C00016881F827600CF017FF28460DF0C9FBB4F95000B4F9B0
:20AED000521088423BD1F86890F8C20000280CBF0520072005F02EFA04F5AA742568F86820
:20AEF000854208BF656890F8C240002C0CBF0468341C80F8C2604DB195F8C23023B9286827
:20AF1000A04228BF041C01E085F8C260A4B10D480068B4F1FF3F12D0B4FBF0F101298CBFDC
:20AF3000B4FBF0F10121F86878300DF08DFAF86878300DF08BFAF8BD012009F075FEF8BD42
:20AF5000A8200020043100202DE9FE4F514C814604F13C0A50460DF097FA90468B4607468A
:20AF700008F0010000900DF07DFA0325BBF1FF3F019015D1266C2EB1206CC068814508BF89
:20AF9000206C0BD00DF06EFADAF8006074E0F168894570D10DF05AFB301C71D0B0F924B08B
:20AFB00058460BF0A7FC00286AD0216C814248D0B84217D104F1C8000DF04AFAE06B0068E8
:20AFD000E06397F82700394640F0040087F827000AF110000AF0D8FF5FEA980022D3E76B0B
:20AFF00001221BE017B9832D20D01CE03968884225D104F1C8000DF02BFA396808683860CE
:20B0100091F8270040F0040081F827000AF110000AF0BAFF5FEA980004D3002248463946F7
:20B0300007F04AFD832501980DF010FB2079012829D004F1EC0002210DF032FA23E03F68E7
:20B05000D0E7009F90F82720012505FA07F13E1C41EA020180F8271014BF0C480C480BF0F1
:20B070009BFD5FEA980004D3E16B48462A4607F023FD832504E03668002E88D10DF0E6FA81
:20B0900001980DF0E3FA2846BDE8FE8F0100020401000104A82000202DE9FF410646080BE3
:20B0B000C0F08E80484C00250127E0682570016A2772C90803D3C36904212A46984743492D
:20B0D000A0462A4608F170000DF0D4F940480DF06FF8D8F80C0041683F4C886808B9C868FA
:20B0F00020B1A4F11C00C5613A490160384608F09BFC2560394844F81C0CB1684D80B0683F
:20B11000028840F60200904208D0B2F5C15F05D00B8B4FF60F421A400A8304E00B8A4FF646
:20B130000F421A400A8200F1080C7774ACF10702531C00E039464F6837B13888844503D069
:20B15000824218BF8342F5D12F464F60487B00F0F00040F00100487308F13C000DF094F947
:20B170008068008882421BD0834219D0308DC8B196F83400758596F83530F76200F0F000D4
:20B1900086F8340003F0F00040F0010086F8350006F128024A60487B00F0F000487301E01C
:20B1B000C8F86050B068694602F01EFE68460CF041FF20680028FCD02560B06844F81C0CD3
:20B1D0000090BDE8FF81C046A82000205D770100152E0000510007061C10044001010E04C2
:20B1F0002DE9F04106467478ADF1180D002C40F089804948B6F896100088884218BFE8247E
:20B2100006F18C0101A80D460CF071FB01A80BF04FFD424B40B996F8990040B1A3F13C00D8
:20B23000007820B9E8246DE0002086F89900002C68D196F8990000280CBF0120052004272D
:20B2500037752946F0820DF10E000CF050FB706896F89840401E7060411E7160B6F896809E
:20B270000470327D71680024481C3062501E0870308934651A78B465801C3081A2B386F8A5
:20B290006B70296806F16C0001606B6843602A8902810CF01FFC06F16C0228BB06F18C01DF
:20B2B00010460DF0C3F81E4D286810F47F0F0CD086F82C70286806F12C01012200F47F00A3
:20B2D00030633046FEF7CAFD286810F0FF0F0BD02A2086F83C00286806F13C0100F0FF0069
:20B2F0003064304603F0F8F90094304603210DF10E024346F8F7DEFB041C02D1304603F067
:20B3100015FB2CB174701A203070304608F0B8FB06B0BDE8F081C046860C0020901200200B
:20B33000900700002DE9F04706464FF00108ADF1600D0922B07D8DF84C8006F117018DF83D
:20B350004D000DF14E000CF061FC464D68688047814616A98120FFF7A3FC707D002854D0CC
:20B370009DF85800022817DA042000238DF80300347D8DF802809DF858708DF8013069466C
:20B390008DF80040781C8DF85800D220FDF702F8812016A9FCF7FEFF00274FF0FF0A3C4646
:20B3B000307D8DF8217008A980F001008DF82000D120FFF775FCC0B99DF82200FF2814D060
:20B3D0008DF800006946D420FFF76AFC20B1A96848468847192042E0307D69460DEB80006B
:20B3F0000461D420FCF7D6FF01E08DF822A08DF82440307D8DF8234008A98DF82000D1202F
:20B41000FCF7C8FF7F1C032FCADB307D00279DF84D208DF840000DF14E018DF841700DF1D4
:20B4300042000CF0F3FB8DF84B80D02010A9FCF7B1FF071C0FD1307D314610228DF828002E
:20B450000DF129000CF0E2FB30690AA90F90D320FCF7A0FF0746A96848468847F8B218B03F
:20B47000BDE8F087F41200202DE9F04FFF25ADF1140D8DF800504FF6FF79ADF80290ADF8D4
:20B4900004900AF09BFDDFF81CB104900BF1020000880027001F84B2082C64DB4E46B0463F
:20B4B000C246201F02A9082280B20AF037FFBDF80800814508D1BDF80A10894506D1BDF879
:20B4D0000C20924502D107E0BDF80A1051EA000317D1BDF80C30A3B9BDF80E1008466FF3DA
:20B4F0000E0060B908460830844206DA0CF082FD04980CF01DF900204FE008462EE0241FD2
:20B510002EE0C20BD30327D1BDF80C20854203D18E4208BF90451FD0C5B28DF800500E46FB
:20B53000ADF802609046ADF804809DE80600384607F0C0FC80B9BDF80E20A01A07F1885192
:20B55000001F083280B292B20AF0E8FEBDF80E003F180837BFB201E0BDF80E00241A083C3C
:20B57000A4B2082C9DDA09F0C5FB3FB10C484FF088513A460CF0A6FE0CF09CFC04980CF059
:20B59000D7F85A46507800281CBF0020011C03D1C7F58054391DA0B2518005B0BDE8F08F6E
:20B5B00004E001005C1900202DE9F84F064630798028D4BF0020E82071790027092901DB2D
:20B5D0000A2900DDE820B17909B1042903DB802975DB862973DA002871D1DFF8FC8098F812
:20B5F000A1000F286BD0B8F8BA104FF6FF70884265D0B8F8B410884261D0F079314C01287D
:20B610000BD040B1FF285AD194F83B00002856D101252F4602E0012500E00225DFF8A8A01D
:20B630000AF12000834608F03FFE0AF1100008F03BFE04F1200008F037FEDFF8949009F16E
:20B65000040000688047214B84F83B500246FF21002060631D6884F83810002D0CBF012186
:20B67000011C012F84F83D10554684F83C7008BF032085F840004846816810468847B11DD0
:20B69000E820FBF79FFF711DE720FBF79BFF311DE120FBF797FF94F83D00012802D1202005
:20B6B0000CF000FD0B4898F8A1104FF47077A86207FA01F000F2636158460CF0A9F8BDE831
:20B6D000F88FC046BC160020E82F00209C0A0020F4120020012C0100CC0B00202DE9F84F36
:20B6F00005464448DFF8109183462E18093699F83C0034788846B0B1D9F8541099B10BEB80
:20B710008507786B00F0FF0088478246D9F85410786B00F47F008847504480B218B1317892
:20B730004018001DC4B23548007801280CD198F808704FB1324898F80930C1190E79C05C4B
:20B750000019401DC4B200E000260D2D09D106EB0408B8F1F80FD8BF2A4F1CDD0CF04AFCDB
:20B7700005E030198046801C0BF02CFC074697B902200BF027FC011C0AD00BEB050090F8AF
:20B7900025001A270870204E4F70307807F0A4FE0020BDE8F88F08F10202384600210CF069
:20B7B00091FE07F10C00002174220CF08BFE07F13C00FF2110220CF085FE07F12C000F2151
:20B7D00010220CF07FFEE0197860022D3E810BDB0B2D09DA7868401E78606D1E0570388917
:20B7F000641EE4B2401C3881A7F84C403846BDE8F88FC0464C07000054120020980C002094
:20B81000140D0000D00A00207C1300202DE9FF47484D95F8E700002877D101243D4F85F84B
:20B83000E740387B85F8E6007E68C5F8106101A80CF0BDFD002605F10C00029601AB8DF857
:20B85000046035490396324608F0DAFF334905F1300001AB324608F0D3FF314905F15400C0
:20B8700001AB8146324608F0CBFFB96820468847DFF8BC802B4808F104037A7B0078186842
:20B89000C0F3815A22B1BAF1030F04D185F8E140BAF1030F1ED0BAF1020F1BD0BAF1010FFA
:20B8B0002CD14FF08059D9F8A4011F4F456831464FF040521C23032000903846A847D9F85A
:20B8D000A40131464FF400720923456800943846A84713E002200AF0B1FDBAF1030F0CBF68
:20B8F0004FF47A7142F2107110480068B1FBF0F148460CF0A9FD48460CF0A8FD40460068BB
:20B91000C00802D230460AF099FD00200090BDE8FF87C046E40C00000F890000AD18010046
:20B93000791401001131002000A00C4004310020B03F0050E40C00202DE9F04F0C469246F8
:20B950008046994600213822ADF13C0D684606F0E0F920686D4628606068686020892881AE
:20B97000207A032804D0022003268DF80C0002E003268DF80C603A4C207818B104F1380032
:20B990000CF010FB208FADF80A0060781F28B4BF411C00210027B8F1050F617040F08000BD
:20B9B0000BD0B8F1040F05D0B8F1020F08BF40F0600004E040F0200001E040F040008DF8F0
:20B9D0000D00ADF828A04FF0010BCDF8249022498DF80EB00A680BA80260496841608DF80D
:20B9F000356005238DF83660B8F1050F8DF8343012D0B4F86200B8F1040F08D0B8F1020F7B
:20BA100012D1B4F86800401CA4F868000CE0401C80B2A4F8620007E00BF0B2FB6061B4F84B
:20BA30005C00401CA4F85C000C4918206A4613F0CFFBC0B258B1B8F1050F09D1206B0AF0A5
:20BA500045FDB4F85C00401CA4F85C0000E05F4638460FB0BDE8F08FD10600005D600000BE
:20BA7000E81000202DE9FE4F0BF0CAFB434C04F10C020290116820614FF40050491C1160F4
:20BA9000694608F0D3FCDFF8FCA0DFF8FC9094F8330000285FD0A66B94F8310000254FF002
:20BAB000FF0BA0462F4654E0B07F800821D3F07F09F076F80146082268460BF095FAC0B142
:20BAD000716802980CF0CAFC2D49814211D8F07FB7770AF0F3FB86F81FB0DAF80000804794
:20BAF00094F8323013B15B1E84F83230D9F80810884798F830006D1C2036ADB236E0F078F9
:20BB1000800822D3307909F04BF80146082268460BF06AFAC8B13088010402980CF09EFCCF
:20BB30001749814211D83079F7700AF0C7FB86F804B0DAF80000804794F8333013B15B1E26
:20BB500084F83330D9F80810884798F831006D1CADB2A842D3DC94F8320048B1A046666B8E
:20BB700098F8300000254FF0FF0B2F46A8429BDC04F1140008F08AF8BDE8FE8F000F0020CD
:20BB900000A493D6F8120020F41200202DE9F041414C0746206800287BD0DFF80081002F95
:20BBB00018BFE92F17D10BF0FBFA4546297801EB81016918C1F8020095F8B560287800EBAB
:20BBD000800029184E702878401C2870C0B20A28A4BF00202870324D68681C2F32D0314E68
:20BBF0004FB1F079032806D1E12F04D0002088F8B200072000E0052008F026FE2468F07957
:20BC100003280ED06CB1002084F86900E18A2648C90938BF2938007884F86A003846FDF716
:20BC3000FDFD98F85700012833D168688047044606F00AFEA96820468847002088F85700CA
:20BC5000BDE8F08180470646A96894F82F0002281ADA216804F124000BF0C2FB94F82F00AC
:20BC7000A968401C84F82F00304688472068007D252819BF012088F85600012088F8550040
:20BC900000202060BDE8F08130468847F120FDF7C5FDBDE8F081C0469C0A0020402D002063
:20BCB000F412002090150020AE0C0020F8B5454C05466078002800F08380B4F95200B4F987
:20BCD0005010884213D0284609F03EFF38B9216C21B1216CC9688D4208BF206C38B1B0F9E1
:20BCF000241002224FF0E043284605F04BF90CF0B9FB074604F5AA700168A94219BF002671
:20BD10004660002606606078E168401EC0B26070002843D12078E56088B1012008F084FF32
:20BD3000022008F081FF38460CF090FC05F140004FF0FF310CF00AF90CF094FB074604F1E2
:20BD5000EC000CF0A7FB04F170000CF089FB04F590700CF09FFB04F18C000CF081FB04F1E7
:20BD7000C8000CF06BFBE66038460CF06FFC05F140000CF08BFB05F178000CF05FFB05F1EC
:20BD90009C000CF05BFB04F128000BF0B9FA287C012815D10E2003F0C5F8F8BD8D4208BFFE
:20BDB000E66038460CF052FC05F140000CF06EFB05F178000CF042FB05F19C000CF03EFB5C
:20BDD000F8BDC046A82000204549B0B5044601F13C00007800287FD094F88B00002871D1D5
:20BDF0003520207504F18D01112204F16C000BF00DFF04F13C00FF2110220CF063FB04F159
:20BE10002C000F2110220CF05DFB94F88C0004F13C0500283ED0401E29D0401E14D0401EB5
:20BE300058D12A20287002272764042305F8103C4FF410222263032184F86B10204607F051
:20BE5000C9F9071C3BD137E02A200A272870042327644FF44C1205F8103C0221226320460D
:20BE700084F86B1007F0B6F9071C28D124E02A2002272870042327644FF4102205F8103C7A
:20BE900001212263204684F86B1007F0A3F9071C15D111E02A2002272870042327644FF401
:20BEB000502205F8103C00212263204684F86B1007F090F9071C02D1204602F037FD381C5E
:20BED0000BD1B0BD01280AD1C86C8047002808BF002002D0192000E018200BF0B9FFB0BDB8
:20BEF000541200202DE9FC410746BE6833687D68986B20F4FA609863AC6B44B13168886B62
:20BF100040F4FA6088634FF0FF30BDE8FC81AA6329630024EC776C630CE09DF80000296B04
:20BF300008706B6B286BAA6B401C2863581C6863501EA863A86B90B93168886B40F4FA60E6
:20BF500088636A6B6878296B0128A1EB0201296303D1EB68384698476A6B144646E005F18A
:20BF70004000694609F096FA0028D6D50CF07AFA204F8046387820B902200AF05FFA0120A2
:20BF9000387040460CF062FB1B49086840F4007008603168886B40F4FA6088636878D8B9B4
:20BFB000696805F1EC000BF0D1FF90B1AC630CF059FA0646387818B1022009F0CBFF3C70FE
:20BFD00030460CF043FB1027696B286BEF77401A2863686BBDE8FC8195F82D0030B1686B55
:20BFF00020B1AC6305F19C000CF05CFA2046BDE8FC81C0460C310020301000402DE9F04FAD
:20C0100009AF9A4616460D46ADF1440D3C89D7F80480109000203F888DF83C00BC4201DAA1
:20C03000C24501D30BF0E6FF002E69D0364810F80690042EA4EB09044FF00000A4B2B8BFD8
:20C0500001205FEA000B0EBF3F1BA04400242F49082307A8A7EB0907BFB211F801295B1E1B
:20C0700000F8012BF9D1290E00F8011B2B0C00F8013B2A0A00F8012B9DF83C1000F8015B7F
:20C09000234D06702868109A4369686898470646B6F1FF3F24D001208DF801009DF83C6018
:20C0B0008DF802600BAA04928DF800B08DF80390CDF80880CDF80CA002218DF81410ADF8C2
:20C0D000164007ABADF818702E686868326A01936946904706462868826968680FA99047D9
:20C0F000002E18BFE4200CD1B9F1000F08D0444448460BA911F8012B401E04F8012BF9D16A
:20C11000002011B0BDE8F08F180D0000AB0C0020F4300020B0B53F49446809688068496827
:20C13000006888473E4D012205F118031A6050B1217AFF2907D0FF214009217264D204208E
:20C1500043F8180C45E0207A00285DD0324B3349401E1AD0401E02D0FD3855D051E01D68DB
:20C17000D4F8B4000570D4F8B870D4F8B400401CC4F8B400781EC4F8B800D4F8B87027B3A2
:20C19000012F3BD9092202201BE0D4F8B000401EC4F8B000D4F8B070EFB9D4F8B870A7B1DD
:20C1B0000220D4F8A8202072127C2D1F012F4FEA420242F001022A609CBF0321696001D9BF
:20C1D0000B220A600CF014F9B0BD0020207204220A600220F6E7D4F8AC0000781860D4F8CD
:20C1F000AC00022F00F10100C4F8AC00F0D2D4F8B870002FECD100202072052243F8042C12
:20C21000E7E7FF202072B0BD04F12C000CF04AF9B0BDC046AC0100100828004004280040B6
:20C23000042800402DE9F8438146D9F808703868066CD9F8045046646A6CAB6CA86B16F436
:20C25000F06F0146A2EB03082AD1F00911D270095DD301B395F83C40641EA14298BF0C1C6F
:20C270004846214609F050FDA86B001BA8630DD04DE081B1484609F047FD95F82D10A8635E
:20C2900011B9002843D101E00020A86305F19C000CF008F93BE0484641460AF0D7F936E0DD
:20C2B000F20A19D24FF00008444602E0A86B401EA86340B34846012109F026FD386844684D
:20C2D00014F00F04C0F80480F0D0286B401E2863686B401E686316E0386844680022202916
:20C2F00004F00F044260CCBF20270F1C4846394609F00AFDC7F12007B845C8BFB84648468C
:20C3100041460AF0A3F9EC77484606F06DFBB0090BD3A96A49B10F46484609F02DFDA862ED
:20C3300018B94846391D07F0E7FFBDE8F88370472DE9F04105463E4804780F46002DADF1D0
:20C35000280D42D03B48866A002F3ED08046D6B17069C0B10123ADF8223006208DF8200059
:20C3700029460C2200236846ADF8243004F01AF903A839460E2204F015F9766908A803C889
:20C390001A226B46B047787B012668B9002C14BF0FA013A06988102208F00EFA397B13A083
:20C3B0000A2208F009FA08E0002C14BF12A017A00BF09EFD19A00BF09BFD88F80260002012
:20C3D000314606F00DFA88F803600AB0BDE8F0815265737461727465643A20307800C04670
:20C3F000537461727465643A203078004368616E6E656C3A2000C046446576696365205279
:20C41000657374617274656400C046C0446576696365205374617274656400C04672657155
:20C4300075656E637920486F7070696E6700C046E8100020F80D0020F8B53A4C0D46A8085A
:20C450004ED2E8086DD301250420A57209F0F6FF0BF090FC04F1580282E8030004F13C00B9
:20C470000CF012F8E16868B1C068064641B18E4206D0316AC90803D3C369042100229847A4
:20C490003146E1604868284900780860022009F0D5FF112003F030F8E1682571087C10B174
:20C4B000E078012803D00E2003F026F8E16849681E488F680FB9CF681FB10021C1611C4F05
:20C4D00007601C4A40F2FF711160002787611A4941611A480BF06CFE19200BF0C7FFF8BDE2
:20C4F00004F14C0630460BF0CFFFFEF783FC30460BF0CAFF25F0020504F13C0158B9E808A9
:20C5100003D208460BF0C0FF58B104F1C8000BF09FFF042101E045F0020104F1EC000BF0B5
:20C53000BFFFF8BDA8200020D02108400010044051000706000004600A00004091960000D0
:20C550002DE9F0410BF066FA3D4C276C002F6CD010F00A0F16D107F1100292E8600000219D
:20C5700005400E4008BF002D5FD03969BE690840676430434FF48041B86104F1EC000BF0AD
:20C590008FFF52E039692F4DBB69002641F00A0126640840103D1843B86105F108033A69F0
:20C5B0001868904307F11002186092E803002868091C88433946286004F14C00804609F092
:20C5D000E3FC04F1EC0002210BF06AFFA06C60B3F86840680078022827D197F82700400845
:20C5F00018D297F8270080080ED2A06C2064A968A06C00690843A860A06C2F68103003C80C
:20C61000081C384328600FE0A06C2730017841F0020104E0A06C2730017841F00101017080
:20C63000A16C404609F0B0FCA664206C30B904F13C000BF029FF08B103F064FABDE8F081BF
:20C65000A82000201C10044070B53F4C0646A07EADF1200DF0B994F85C0082281AD0394BE4
:20C6700040F2016046F25C05ADF8080034491868ADF80A50426A086802A99047812814BFBB
:20C690006FF07F009DF90C000AF0B0FB94F85C10226B505494F85C00822814BF401C00205B
:20C6B00004F1180584F85C0094F85C0005EBE00292F82C00411082F82C10400807D294F85C
:20C6D0005C00401C84F85C00C0B28128ECDB94F85C0081282CDA05F14401E120FAF772FFA3
:20C6F00002204FF6FF738DF81800A17EADF8103031F0020018D0012919BF072083210820B0
:20C71000802100224935009204AA0195FAF720FADB2807D0E52805D0F32803D0DF2818BF5F
:20C73000E8280AD1607603E0304605F0DFFB04E02A203070304607F0A3F908B070BDC0463E
:20C7500070170020601400207C2F002070B53D4C012504F108000026A06304F130016563DB
:20C770000420E063402084F8400060680E600BF0B3FD2070617A207A3346282240EA012032
:20C79000A52181FB0001000C0E0430430914801A04F11002994182E80300A37AE27A42EA0B
:20C7B0000322192383FB02231834920B9E049B13324384E80C00244C04F1180686E803004B
:20C7D000203484E80C00214C60832083E28316200BF0DAFA0A22618B20810BA007F0ECFFDA
:20C7F000E18B0EA00A2207F0E7FF218910A00A2207F0E2FF2089012801D0A07810B1A57017
:20C8100004F034FB70BDC04653656E736F722054656D70202843293A2000C04653656E73D5
:20C830006F722048756D69646974793A2000C0465761746572204C65616B20537461743AA4
:20C850002000C046F014002030300020E81000202DE9F04707467D68D7F8089090460E46D6
:20C870000BF000FE8246A86A002864D105F584700BF0EEFD0024EC772E6250466C620BF02E
:20C89000E5FE0BF0EFFD2F4E3378824623B9022009F0D4FD0120307050460BF0D7FE2A496C
:20C8B000086840F4807008603846414609F064FAA862C0B93846414607F01EFDA878D0B9CD
:20C8D000A96805F1D0000BF041FBE8B1AC621020E8774946284605F045FB0BF0C3FD82464F
:20C8F000307840B323E0D9F80010886B40F020008863A87810B12046BDE8F087A96805F111
:20C91000D0000BF023FB10B9686ABDE8F0873846414607F0F1FC1020AC624946E8772846E4
:20C9300005F020FB0BF09EFD8246307818B1022009F010FB347050460BF088FE4FF0FF30B9
:20C95000BDE8F0870D31002030100040FEB506463B4C3178B4F86C00E1292FD0B4F86E0063
:20C97000E92926D0B4F87000D9B9364D3069AF6A02903FB37F692FB3E96A1931814221D815
:20C9900006208DF800000422ADF802200023ADF804309DE8030002ABB84708B90298E8621A
:20C9B00010E0401C80B2A4F8700022A00BF023FD08E0401C80B2A4F86E0003E0401C80B20F
:20C9D000A4F86C00717831F07F0031D001F06000402819D13078B8B965690AF0D1FBB4F8B9
:20C9F0005E10B4F87E706422401B60614B1C4D1CB0FBF2F001FB0702AFB2A4F85E70B2FBA3
:20CA1000F3F0A4F87E00717801F06001202906D1307820B9B4F86400401CA4F86400602938
:20CA300006D1307820B9B4F86A00401CA4F86A00FEBDC04664617461436E663A2000C04644
:20CA5000E8100020F80D00202DE9F04106AF3D793E68984604460B1CADF1180D074611D0F1
:20CA7000012B15D130797379641C3870B17904F8013B337A04F8011BB17A04F8013B738951
:20CA9000181201E03178707804F8011B04F8010B8AB9002D0CBF42F20C0042F20D0069465F
:20CAB00007F0C4FC9DF80000BDF8003004F8010B181204F8010BB8F1010F34D0B8F1020F84
:20CAD00039D1002D0CBF42F2020042F203000DF1020107F0ABFC7589CDB1681E01468B1054
:20CAF0000DF1020201EB5371C910CBB2811000EB517121F00701401AC0B20121401C01FA82
:20CB100000F0D15CFF3080F0FF000843D054E81D0DF10201C210204603F044FD7089C01D93
:20CB300004EBE00407E0002D14BF02210121204602F09AFE0419E41B06B0A0B2BDE8F081BC
:20CB50002DE9F04390460A68D8F800401678814600271D463846ADF1140D531C242E0B60DC
:20CB700053D112F8016F5B1C4C2E0B600ED1AA68E41C24F00304241D54F8040C494606F07D
:20CB90001DFE2968EF600127091A2960462E1AD1E41C24F00304241D54F8040CE41C02900D
:20CBB00024F00304241D54F8040C002749460390AA68ADF8047001A803F06CFB2968EF6056
:20CBD0000127091A2960532E1FD1E41C24F00304241D54F8040CE861C8F80040288B0090BC
:20CBF000A968EA69D9F800004346F7F791FCD9F80040002714B10119C9F80010D8F80040F4
:20CC10002968EF60091A01272960662E0AD12B8B23B9E41D24F00704083403E0E41C24F0FC
:20CC30000304241D1FB9E9690E700127EF60C8F8004005B0BDE8F0833748F0B538C8ADF1EE
:20CC5000140D6A4638C209C882E80900334E00231C4606F1200080E818007471B4710127E6
:20CC7000F771347106F1180080E818002C482D4A07604FF480501060694642F8100C06F137
:20CC9000080003F0C3FD0028306041D008F0A2F9254E06F1200528460BF0BCF920462946EB
:20CCB00086F8284008F0B6F9706080B30B20652109F06CFC40F6AE300BF09AFB0D20E621EA
:20CCD00009F064FC40F6AE300BF092FB0720502109F05CFC40F6AE300BF08AFB0E2016216D
:20CCF00009F054FC751CB7700F20F4630223707006F1080273634027B26306F1300186F89F
:20CD1000407070680D600BF0E7FA307001E0FEE7FEE705B0F0BDC046980C0000303000205B
:20CD3000301A4442A0200240F01400202C4870B50568B5F1FF3F08BF00250AF043FC0128B5
:20CD50004DD108F0E7F9142849DB26482649002601230660254A0B60254C13602068002872
:20CD7000FCD1264A131D2349186820F00300014321480068C0080CD2106810F0030F0AD018
:20CD900041F003001860106800F003000328FAD101E041F001011A481960006820B11948ED
:20CDB00000682846F5F740FB174818490660184D0A686FF35B4245EA020008601549086803
:20CDD000C0F30130012806D10A681348104040F400320A60086020680028FCD170BDFEE77B
:20CDF0001C130050840460425C600C40082204430C00684204000020B03F00500040034065
:20CE100080012843000120438C210840482003400000390104000940FFFFFCFC2DE9F04F40
:20CE300009AF3C897D6816464FF0000A0246002EADF1440DA04610933C888DF83CA05CD09C
:20CE5000304810F80690042E03DAA8EB0900C8462D18F868A4EB080407AB0827A4B2C01D9F
:20CE700010F801C97F1E03F801CBF9D1080E264F03F8010B080C03F8010B080A03F8010BDC
:20CE9000386803F8011B9DF83C101E704369786898478346BBF1FF3F2AD0042E04DA032011
:20CEB0008DF80000022002E002208DF800008DF8140002959DF83C608DF8026001218DF843
:20CED000011038688DF8039007ABADF816800BADADF81840026A0193109E04956946786801
:20CEF0000396904783463868826978680FA99047BBF1000F18BFE42000D1504611B0BDE88C
:20CF1000F08FC046180D0000F43000203349F8B501F13C02107800F0F000364D107091F8C6
:20CF3000740000F0F00081F8740091F84000002640F0180081F840004FF4FA508864688946
:20CF50008E6308B901206881274C254F254994F83C300978083148433978002B01FB00F0AB
:20CF7000009037D0E26F002A34D0D4F88000002830D005F1080168469047074669792B79C0
:20CF90001D481B4D0268652F1AD0A7B9117D052920D116490F78EFB90146006890F82C00CE
:20CFB000042817D10968A46D906D096B3346A04780B91A2001E02E703846FCF72FFCF8BDB7
:20CFD00082F8691082F86A30D4F880102E701C208847F8BD009809F0E5FCF8BD0810002021
:20CFF000B81800206517002054120020890C002018310020541800209C0A00202DE9FF4743
:20D010008046D8F80870D8F804400D460BF02AFA217819B10BF01AFB00205BE001212170EB
:20D030000BF014FB68460BF0C9F800268DF8046004208DF8000040F61A23ADF8023078787A
:20D05000694601F055FE254982460868BAF1000F3ED0894640B9FE20029002A909F104003E
:20D0700003F0D4FBC9F80000297C012914BF1C4A4FF000421B4B39780A4343EA020102916D
:20D0900005F082FE08BB2878607068686060287A2073E8682061287C2076C4F81CA06168C7
:20D0B000404604F03DFC58B9207B012806D02169084303D0404608F06DF808B9464608E042
:20D0D000D9F80000397806F057FC504602F002FF267030460090BDE8FF87C04628190020BE
:20D0F00000004080000880A12DE9FE4F83460020374E00907068019180472E4C0290E06851
:20D1100004216A4600F0DAFE2B4DDFF8B0A0DFF8B090DFF8B4802B4E2BF0010725F00105EA
:20D13000BD4213D0504620F00100B8421CD1494691F9000010F1020F18D03068826B91F94D
:20D150000010E068904781280ED10FE0414691F9000010F1020F09D03068826B91F90010FE
:20D17000E0689047812801D00AF044FF3068C66A1649019AE0685B46B047061C01D50AF035
:20D1900039FFBD4207D0504620F00100B84204BF49460E7001E041460E7001200090E06821
:20D1B00004216A4600F08AFE0949029889688847BDE8FE8F64170020E5E2000019050100B3
:20D1D00039190020601400203819002008100020F41200202DE9F84F07463248DFF8C89017
:20D1F00000EB4706183699F83C00348890468B46B8B1D9F85410A1B12C4D05EB8705686BB1
:20D2100000F0FF0088478246D9F85410686B00F47F008847504480B218B131884018001D71
:20D2300084B225481230007801280CD198F808604EB11F4898F8093081190D79C05C2418DC
:20D25000641DA4B200E00025281980B209F0BAFE0646184890F80090D6B130460021224674
:20D270000BF030F94FF00008A41937700D4986F8018006F180007460CA5D358159460AF0B9
:20D29000C5FC4846314606F027F94046BDE8F88F8DF8007068461A2103F034FC1A20BDE810
:20D2B000F88FC04688030000541200204C070000140D00007C130020860C00202DE9F04F96
:20D2D000364E0025ADF1340D07464FF0010AA846A9460C93DDF858B00B914AE017F8020FE0
:20D2F000AD1CADB2401E1BD0401E09D0401E04D0401E36D1022C34D138E0032C31D135E04E
:20D31000072C2ED1B9787878FB1C40EA0120A6F84400186806F14802106086F859A025E0B9
:20D33000052C1ED1CDF80890B91C0A8802A80280897881700B9803A9FBF730FF9DF82A00AC
:20D35000A0B1029B40F0020000F0F7008DF82A0006F1500203931068049003A805F0B0FCD0
:20D3700004E008EB0400801C1FFA80F8E7196419A5B23846694608F025FF041CAED1022DAA
:20D3900003DC4D466720A84600E048460C990D800DB0ABF80080BDE8F08FC046402D00205F
:20D3B0002DE9F84F0D46064628684FEA900A3248504502D3287A022802D00320BDE8F88F2D
:20D3D0000BF050F8DFF8B4800090D8F8580108F5AA79B04214BF00240124A00080F00400F4
:20D3F00059F8007006F19C0083460AF0FBFD68B957B107F19C000AF0F5FD38B938460221D3
:20D4100001F09EF8074602E0022700E000271C4800686FB998F8880140F0020088F88801CE
:20D430000098C8F87C610BF011F90020BDE8F88F2A68A10001EBC40149440A612E7A0E764E
:20D45000BAFBF0F1012998BF012158460AF0FCFF58460AF0FBFF00980BF0F8F8012F07D1D3
:20D47000D8F88001B8F9841198F886210AF083FF8320BDE8F88FC04640420F00A820002004
:20D49000043100207CB5354C054694F8A1000F285ED03348697E0078890959D2297E002832
:20D4B00041F00201297639D069684A1C1078801010F0030F32D000F0030002280ED1B4F875
:20D4D000B4304FF6FE70984208DD56791179002001EB0621994208BF012004E004F1AA0014
:20D4F000491D0AF0DBF9C8B9687E696840F0010068764A78C2F38102022A2DD1491D4A7855
:20D5100009784FF6FF7601EB02218E4224D1297E00F0EF0041F0200129761CE0687E114E34
:20D5300040F0030068763078B0B994F8D7008DF80000FF238DF8033094F8E6608DF801603F
:20D5500094F8E7508DF8025068460AF010FF7CBD687E40F0010068767CBDC046CC0B002006
:20D5700054120020F716002070B50546344C2878ADF1200D00284FD1208F04F148066B8860
:20D59000ADF800003146ADF81030E2200AF002FD0DF1120031460AF0C7FE698853200AF0DB
:20D5B000D9F9208F04F13E063146ADF80E004A200AF0F0FC01A831460AF0B6FE00268DF8AE
:20D5D0000D60A08FADF8020094F83A308DF80C30304608F093FF522031460AF0AFF994F82A
:20D5F00050000F281CBF01206070E06828B102681AB10DF10E0069469047032008F0C8FD00
:20D6100094F85200032818BF042813D104F1080010210AF071F80DE0002060700AF054FC52
:20D6300041F2883008F06AFF0649B1F85A00401CA1F85A00216E09B12846884708B070BD82
:20D65000B0110020E81000202DE9F0432A4A2B491778ADF1140D002F44D02E48077837F0E3
:20D670007F073FD1C88A2C4F254E264D401C0024C88207F16808012097F87410307001F05A
:20D69000F00187F8741029783C67012902D02146F9F794FE09F064FE1D4E301D006880471B
:20D6B0001E4F022381460294203F8DF80C30386A1B4AC56C8DE81800134B1068414602AA7D
:20D6D000A84718490028A1F12001088006D40F4991F90000C7F80C80401C0870B168484605
:20D6F000884706E0088B401C0883002010700AF065F805B0BDE8F083163100205418002034
:20D710003B190020E8190020A91B010042190020F4120020183100200810002060140020C9
:20D7300070170020B41700202DE9F0470D4606465FFA85FA280824BF2E4845402E494FEAC5
:20D750008A03C85885EA00023240C2F300672B4A06EA0504B043224006F4E0240243B4F55E
:20D77000E02F01D1500E14D306F4E020074310D002F4E027B7F5A02707D0B7F5803704BFE2
:20D7900022F4003242F4A02203E022F4803242F4C022DFF86C80CA5008F1D0073968012205
:20D7B000002002FA0AF40C4218BF101C5FEA000906D1F00D04D34146C5F3805001F80A00DF
:20D7D000300E0BD30AF04EFE290E34BF0021211C3A68A243114339600AF038FFB9F1000FF1
:20D7F00006D0F00D04D34046C5F3805100F80A10BDE8F087006000A000100840007F077FD5
:20D81000002002402DE9F04117460D460AF02AFE324C8046207883266DB16D1E04D06D1EF0
:20D8300055D0681E11D00EE0B4F8C4004FF6FF71814202D005E0206C08B9802648E0206C18
:20D85000808C388044E0032642E0386800215022054604F05EFA022704F5AA7C04F5B27256
:20D87000A5F110015CF8040B41F8100F137A0B735068486052F80C3B7F1E18448860F1D197
:20D89000206C002808BF02200ED0206CC068276C286297F82600236C85F82C00D869226C70
:20D8B0006862106AA8620320E76B8FB105280FDAFA6801016A5097F826204C192273FA69EF
:20D8D00062603A6AA2603F68401C40B2EDE7387040460AF0BBFE3046BDE8F081A8200020B2
:20D8F0002DE9FC47314CA11D0888401C088009F087FC0026B046354681462846694604F025
:20D91000E3FB8246BAF1FF0F4CD09DF80030606B23B900EB4A104068010402E000EB4A10F7
:20D93000416848460AF09AFD864203D29DF800700646D0466D1C0A2DDFDB1E4D281D006879
:20D95000804794F833106FB9A26B08EB88030026FF27491ED218D67013791771C9B284F880
:20D9700033100CE0616B0022FF2701EB48118A77CB7FCF7794F83210491E84F832100C4A35
:20D99000643BD9B2136804EBC1013C310B6052684A6094F88C10491E84F88C10A96888475E
:20D9B000BDE8FC870AF058FDBDE8FC87000F0020680D0000F4120020E0B501880025A1F614
:20D9D000020159B143F20402891A04D0491E19D190F8246000E00226C76901E0C67B476911
:20D9F00087B13F1F052044F2380357F8041F0A04120C934203D0401EF7D13F1D01E0C1F38E
:20DA100003450DB90120E0BD1F4B3046401F18D01C4A401E10D0001F0CD0801E0DD0C01E0B
:20DA300006D00F3819BF1A1C6032184A443204E0121D02E0121F00E0083A1068C0F383400B
:20DA500003E01A461068C0F303200F2806D0A84216D921F4702141EA004110E0761F0AD0CE
:20DA7000761F08D0761F06D00F3E1CBF21F4702141F4802103D121F4002141F4E021396041
:20DA90000020E0BD0011005020130050C4100050F0B5064600210B22ADF1240D0DF119008C
:20DAB0000AF010FD2E4F2F4C3078C01E14D0801E04D0143810D0801F01282DD801208DF8DC
:20DAD000180006F18B0103A80AF0B0FC032538788DF8145068B112E000208DF8180006F1CA
:20DAF0008B0103A80AF0A2FC032538788DF8145028B9B4F8BE000225ADF8020005E00DF18A
:20DB1000020004F1D8010AF091FC8DF80A50B4F8BA00ADF8160017E002208DF8180006F1F1
:20DB3000320103A80AF0BCF90DF1020006F128010AF0B6F9BA34208806F11C01ADF816001A
:20DB50000DF119000AF06FFC0B208DF8000077788DF80170684600F085FA09B0F0BDC0461B
:20DB700090120020CC0B00202DE9F843334D0120002428702B48DFF8B080DFF8B490047025
:20DB90002A4800F16A010F8814EA03064FF0020101EA020108BF00290FD120464FF0E0473D
:20DBB00010401F4008BF002827D0424692F90000401E10700AF012F81FE0424692F90010A9
:20DBD000491E117067B901F069FA46464846047096F90000F0B196F90000002817DD1DE073
:20DBF000B7F5505F07D114481249006800F5C070086001F01DF809F0CDFF484642460470E1
:20DC100092F9000030B192F90000002806DC0AF0F1F903E020460146F9F7D0FB2C70BDE883
:20DC3000F883C0463C19002042190020081000203B190020581400200C010021E8190020DC
:20DC50002DE9F043DFF8BC808946054617464FF0FF31ADF1140D40460AF078F92A4C04EB5D
:20DC7000C504666825680AF0FDFB2168096800290BD42968002905DCB9F1000F09D04FF010
:20DC9000FF3108E0B9F1000F03D00AF0DFFC002430E02968491C29600AF0D8FC28680228C0
:20DCB00028DA1FB903A80AF04EFB03AF38686860B76868460AF0A6F9307B144A00946B46BE
:20DCD0003946019005F12C0007F064F905F16400002108F0CDFD05F14800012108F0C8FD54
:20DCF000706801F009FC0A4A05F118002346042108F066FF40460AF0CBFB204605B0BDE8F3
:20DD1000F083C046A4300020800D0000256E01009F8301002DE9F84F8A463149044601F15F
:20DD3000B400007828B920465146F7F7E7F9BDE8F88F0A25884642F2107B20465146F7F728
:20DD5000DDF998F8B410002848D19AF80060D4F80090002937D023480168C88AC20832D2D6
:20DD700080094FF0000702D3087D15282BD009F027FA98F800308446002B0EBF09235B1EF1
:20DD9000DBB20A2003EB830208EB0201491C0A78964207D0002B0EBF09235B1EDBB2401E35
:20DDB000F0D110E0D1F8011060460AF057FB642101FB09018B4505D942F242706426401AD3
:20DDD000B0FBF6F717B90020BDE8F88F20686D1E07442760B1D10AF03FFB6120BDE8F88F37
:20DDF000402D00209C0A002080B50288A2F602073FB143F20502BF1A14BF002090F82400BC
:20DE100000E0C07B2C4AD2F88832401F0B6048D0401E3CD0001F30D0801E24D0C01E18D01A
:20DE30000F380CD0D2F890024860D2F894028860D2F8BC0220F0784040F080503AE0506940
:20DE50004860D06A8860506C20F0784040F0704030E010694860906A8860106C20F078402D
:20DE700040F0F04026E0D0684860506A8860D06B20F0784040F0C0401CE090684860106A61
:20DE90008860906B20F0784040F0A04012E050684860D0698860506B20F0784040F0405001
:20DEB00008E01068486090698860106B20F0784040F02050C86080BDC41000502DE9F041B6
:20DED00016460C4607460AF0CDFA304D80462A7929786879002C4FD0641E46D0641E41D098
:20DEF000641E3BD0641E2BD0641E15D0641E33D111430843012821D005F13C000AF0C4FA78
:20DF1000E0B9316805F1EC000AF0CEFA316805F590700AF0C9FA31E01143084301280DD015
:20DF300005F13C000AF0B0FA40B9316819200AF0A3FA31681A200AF09FFA1FE000241EE012
:20DF5000306828B1012807D1802006F06DFE15E0802009F099FB11E0032410E0307885F8EF
:20DF700068000BE03088788208E00120FE68787406F16000F86001E0306838608324404644
:20DF90000AF064FB2046BDE8F081C046A82000202DE9F04F2B4F04463878ADF12C0D0128E5
:20DFB0004DD1DFF8A8A0DAF82000274E436CF068022108AA98479DF82000002836D1DFF837
:20DFD000A08008F10400006880470024B146022509901F48059404A90490D9F80C008DF867
:20DFF0001850FFF7DDF93D70564602941949306A8DF80C50C76C4C812B468DE81800164BC2
:20E01000D9F80C0002AA08318B46B847002801D509F0F0FF114991F900004746401C087033
:20E030000998B968C6F80CB0884708E03878012805D10020012C387001D009F0C3FD0BB0F4
:20E05000BDE8F08FE9190020641700204014002000093D0008100020953E0100421900208E
:20E07000F412002070B50646304930780D5C401F1CD0083851D0401F4FD0284608F0A2FF3E
:20E09000041C0DD130780C2808D1706830B1301D07F080F9284608F095FF0446002C43D0C4
:20E0B0002A462046314609F0B1FD37E0B07810BB327A307C51005410401901F00E010918CB
:20E0D00004F0380040182430C0B208F07BFF041C2AD03146182209F099FD04F1180060604D
:20E0F0007168242209F092FD6068243060617169327C0E46D6E7012816D12435E8B208F0F8
:20E1100061FF041C10D03146182209F07FFD04F11800606071682422EBE7344624B1044810
:20E130000078214605F0D8F970BDC046AC0C000048190020F8B50AF04DF804F0EDFB0AF0FC
:20E1500061F8044604F00C000C284BD0E0081ED208F06AFC264E376805460120014609F0C8
:20E17000BDF931686943884211D2224CF020B0FBF7F0291A20460AF061FA20460AF05AFA25
:20E190000120F8F705FF204609F06AF92CE0200928D2194809F0E3FF0428FAD0174A61096D
:20E1B00005D220B11168104621F0010103E01046016841F001010160983210684FF0805539
:20E1D00040F003001060D5F8B8018169202088470B4CD5F8B8712068B86B804701202060AD
:20E1F000206801E00AF028F909F0FAFFF8BDC046BC0D0000F00C0020004003408C21084081
:20E210002C200940F8B5324D6868804706462E4CA9682068002854D160698047676A40F059
:20E230001000002F4CD00022797E0140884205D03A4657F80C7C002FF6D141E004F12400F3
:20E25000394607F027FB002F3AD02760787E30F07F0005D194F82F00401E84F82F0004E043
:20E2700094F82E00401E84F82E00A9683046884721680889C98A05F06FF8A08513480078B5
:20E2900008F09CF905462068C18A090A08D3C07E05F0E2FF206890F91C0009F0C5FD206851
:20E2B000697B012903D002290DD1052005E0007E401080F0010000F00100FBF741F8F8BD4A
:20E2D000A96830468847F8BD9C0A0020B30C0020F41200202DE9F0412A4D0120014628709A
:20E2F000F9F76CF828496FF0010008702B480068C06B8047254C074621786068A2688B00F0
:20E310003E1AB6FBF3F05843361A8800204902FB03F8B1FBF0F0904201D209F06BFEB91BC6
:20E330001C4861604144FEF7DFFE1D4C083CA06867682168404207F0A9FE002F08BFA16825
:20E3500008D0A16878688142DCBF401A78603F68002FF7D1E068884202D0A06005F0BCFD2C
:20E3700003F00AF90C4C60688047064600F01AF8A1683046884709F03DFA00202870BDE887
:20E39000F081C046E819002038190020B8180020FFF6C2FFE5E20000F4120020601400203D
:20E3B0001C1900202DE9FF412E482D4F00683E78C06B80477968401AB100B0FBF1F4B86804
:20E3D000FF680025A8464146BC4271EB080101DAB84206D82946424684428A413CDA07462B
:20E3F00000E0294638463246F317001BA94109F031FC272704464FF47A7200230D46ADF8B1
:20E4100002700820ADF800002046F8F7B1FC01901548016868468847029843464FF0000174
:20E4300000F6FC02A41A9D416042A94111DA0F48026829462046F8F79BFC0D4604464FF0CD
:20E4500000016042A94104DA204606F023FE002000E00120064908700090BDE8FF81C04621
:20E47000B8180020601400201813002050170020173100202DE9F84F2E4C012683461D46A4
:20E4900090468946C4F87C670320C4F880670AAFC4F88407D4F88C0710F0030FFAD1387A74
:20E4B00058B14FF0805ADAF8B001016A27208847DAF8B0010169272088470220C4F8FC0643
:20E4D0003868C4F80804304609F092FFD4F808040008F8D2D4F88C07800F28BF301C26D201
:20E4F0002868C4F83C056868C4F84005A868C4F84405E8681049C4F848053879002814BF3B
:20E51000081D081CC4F84C05C4F850850020C4F85405C4F8580509490E60C4F800B0C4F8CE
:20E530000880C1F80064C4F82090C4F82880BDE8F88FC046044002402800002000004842CC
:20E55000314A2DE9F0410446106C002301261F4687420CD0106CC068844208D1106C90F888
:20E57000260009F0E1FC3E46031C18BF176CD56BDDB1D56B17E0C868844205D191F8270011
:20E5900040F0080081F82700096826E0E868844208D195F8260009F0C7FC002608B10BB91B
:20E5B0002F4603462D68002DF0D1002E18BF022027D1002B14BF002F002022D0106CC06808
:20E5D0003946844209D1106C884206D1106C2730017841F008010170D16B0029CBD1C2F83D
:20E5F0007C4192F8880140F0010082F88801BE8CC2F8804103F00103A2F88461012082F831
:20E610008631BDE8F081C046A8200020F0B506460F4600251446ADF1240D8B200DF10E01E3
:20E630000095FCF73DFB8A2001A9FCF739FB707A00282ED1387AA0B9BDF80E104FF6FE70ED
:20E65000884205DCBDF80E10884220D101A90DE020489DF80E700488BDF80E008DF8127009
:20E670000CE0022807D0032811D1394604A809F0DDFE09240BE038888DF812008DF810404D
:20E69000211200128DF8111005248DF81300284611E002280CBF05240924012818BF311CC7
:20E6B00004D1892007A9FCF7FBFA07A9224604A809F0ACFAB07A04EB0D01C8736A4604A813
:20E6D000214603F08BFC002814BF281C009809B0F0BDC046860C00202DE9F84F07460E1C80
:20E6F00014BF4FF000094FF0E809002F4FD0B9F1000F4ED17868401E78603F210170BD6D88
:20E71000002D0CBF802000207968DFF890A00224083E491E7960DFF880B008703889A7F8BE
:20E730005440801C388116F8080FFF282CD02A2828D1706830B35546696D884780467868AC
:20E750009BF80020A0EB08007860716829B9AD6D3A460023A84748B10BE0AD6D786871686D
:20E770008DF800206B463A46A84710B9EB20BDE8F88F3889B7F854504044388108EB05007B
:20E79000A7F85400641ECED17868386501E04FF0E8094846BDE8F88F8030002054120020B7
:20E7B000F0B52F4C0546A07EADF13C0D022806D0012804D005281CBFE820607649D194F850
:20E7D000600000284AD1002109A81822617609F079FECDF828D009A8294600F031FE94F8AB
:20E7F0002E0094F85810814220DD266B70B10746BDF80A007189884204D13046694608F0B3
:20E81000FDF898B97F1E06F12406F1D194F82E00276B8100242201EB40117818694609F09A
:20E83000F5F994F82E00401C84F82E000D48007828B19DF8340010B994F8580028B909A86C
:20E85000FFF710FC94F8580040B194F82E10884204D12A202870284605F012F90FB0F0BDAC
:20E870007C2F0020620C00202DE9B841804608F097FAC01DC51098F82300002849D198F89A
:20E890007E4008F08DFAA04243DD264A1368E010191891F86C1004F007042141CFB207E04F
:20E8B000401CC0B21918C40091F86C7088F87E4047B9691E8142F3DC1068002188F87E1022
:20E8D000417029E098F97E10C0000830884226DD401A79080BD298F87E10401E4FEA6707AF
:20E8F00001F1010188F87E10F3D1BDE8B88198F87E000D49087098F87E0088F8810098F8E9
:20E910007E00401C88F87E000320FAF719FDBDE8B881002088F87E00072005F095FFBDE894
:20E93000B881C0469C0A0020641700202DE9F041054609F05BFA287E000904D2287D0128F4
:20E9500008BF022700D00527DFF89C80464670688047264C04F124010B68002B08BF0D603F
:20E970000CD07F1E0026FFB202E07F1E1346FFB253F80C2C22B92FB143F80C5C012601E0C5
:20E99000002FF2D1D8F8081088471EB3216928468847E88AA168C00818D2D8F8040080475E
:20E9B00094F82F10491C84F82F10D8F8081088470C4991F83C0028B10846006D10B180476F
:20E9D000BDE8F081FFF71EFCBDE8F08128468847BDE8F081F1206870284604F0CFFABDE8DF
:20E9F000F081C04654120020F41200209C0A00202DE9F8430D46064668687468B7684FF024
:20EA1000000810B9E86800284FD02078012814D109F028FDD4F8BC1049B1D4F8C0108D619E
:20EA3000C4F8C05009F012FE0120BDE8F883C4F8BC50C4F8C05009F009FE022007F0FEFC09
:20EA500004F160004FF0FF31814609F07FFAB86809F00AFD3046294602F04EFA0546B868FF
:20EA700009F004FD207888B9B5F1FF3F08D004F17C004FF0FF3109F069FA207A48B111E037
:20EA900003202072022007F065FA0BE0B5F1FF3F02D04FF0010805E00320207204F12C0095
:20EAB00009F000FD484609F0F3FC4046BDE8F8831A481B4901641B4941641B4981641B4953
:20EAD000C1641B490165022280F8202019494165194981651949C1651949016619494166B1
:20EAF000194981661949C16619490167194941671949016019494160194981601949C160D4
:20EB100019490161002180F83C1080F83F101749C161C162012180F830107047042F0020EC
:20EB3000D9790000ED3D0100514A010079410100292F0100395C0100216F01008D4D010096
:20EB5000E93A010065530100457B0100A5170100154E0100E97701008580010051730100BA
:20EB70004D090100F12F0100C9840100C58001002DE9F04FDFF898A001270446DFF89490A8
:20EB90008AF8007099F80000ADF1140D012803D038460021F8F712FC204606F03FFEDFF81B
:20EBB0008C80D8F804008047049000248DF80C701B4D02941849286A184AC66C4C8302236C
:20EBD0008DE81800174B106818318B4602AAB047D8F80810E88000280AD4134A92F90000C3
:20EBF000401C10700498C5F80CB088473C460BE0504604700498884748460078012803D061
:20EC100020460146F8F7DAFB204605B0BDE8F08F3C190020E81900200810002070170020BF
:20EC3000401400201942010042190020F4120020F8B5264C236813B909F0DCF92368244818
:20EC50000068044609F0DCF8D860204608F09AFD264C18826068804706461E48A168027828
:20EC7000832A30D11C4DEF782FB386210170082008F086FB688B1B4F1949401C6883174806
:20EC90003A7881621849812A09DB0978842A07DA40F6485292FBF1F101F6B83106E0097849
:20ECB00040F6485292FBF1F101F2A321203008F0AFFDA16807E085220270304688470020EC
:20ECD00002F004FBF8BD30468847F8BD9C0A00205814002018310020541800209417002072
:20ECF00051460100B30C0020B8180020F41200202DE9F0410F46810001EBC000DFF8A880AF
:20ED100028490C180D58666807B94746387830B97888312818BF322814D1207A90B909F0EA
:20ED3000A1FB8446387830B96978AA7800230A4318BF012302E0217A69184B782BB1604613
:20ED500009F084FC0020BDE8F08118B901206870A87003E0207A012128184170604609F0E3
:20ED700075FC38782870B07900F0C6FB2168606809780268267A11607D88036841468A1D05
:20ED90003101A1EB4601505AB0F57F4F14BF1B1D08331D603979204607F0A8FA2046BDE8C2
:20EDB000F081C04690080000580B000070B5214E002086F85400012186F85500E82008F056
:20EDD000D5FD5220012108F0B9FD1B4D482205F1800406F15C00214601F0E4FB1748C5F81D
:20EDF0008400383CF4601648C5F88C001548C5F8B0001548C5F8A4001448C5F8880014488B
:20EE1000164CC5F8900013481549C5F89800124847F23052C5F8A00004F19C0005F0A4FD8C
:20EE30004EF660220F49E06104F1C00005F09CFD206270BDB0110020E810002079D500002A
:20EE5000015C01005925010069F100006D650100E103010099160100251C0100F80D00209C
:20EE7000597801001174010003B42DE9F0472C4C4FF0000908AF84F801903968ADF1100D46
:20EE900002A80160B988818002A803C89A46164602F02EFBA046051C14D04C4686B1284627
:20EEB0006946012207F03AFA1AF804009DF80010884205D1641C6D1CE4B2ADB2A642EEDC3A
:20EED000A64227D0B8F80200F61C4FF6FC7440F6F87134402018814203DA09F0F3F8FCF708
:20EEF000C3FA396802A8BE88016002AD868095E803002246534601F07DF998F80100B8F875
:20EF10000210002818BF814604D10919083188B2A8F80200484604B0BDE8F04702B0704776
:20EF30005C1900202DE9B043044609F09BFA81462748021992F8EE10491ECFB2002F82F8E1
:20EF5000EE703FD1254901EB84014A880C78904634F07F0718D1E1090FD24FF0805000F5C6
:20EF7000DC75D0F8B8018169104688472868416B404688470228F9D11EE000EB8800D0F8E2
:20EF900004110020884717E04FF08055D5F8B801016A10468847D5F8B801816A4046884776
:20EFB000D5F8B801016B404688470A4901200860094908688008FCD304F03F003F2801D09A
:20EFD000FFF7B0FF484609F041FB0020BDE8B083E40C00202820086028200840B0090000B8
:20EFF000F0B52B4D05F12C0158C9ADF11C0D02AA58C20AC94FF0805682E80A00476884681C
:20F01000D6F8D001C16820688847216821488A6B10408863206840F2F271416497F83C0012
:20F0300097F83D10C0100DEB80008068084321684863684609F004FAD6F8D001397F46688B
:20F0500005EB8101BA698B68797F206855F821101943BB7F05EB8305AB690B430199B04719
:20F070000D490A1F106840F010001060086840F001000860A07D0027FF2802D0E07DFF280F
:20F0900000D11FB1086840F44040086007B0F0BD440A00000DF8FFFF30100040F8B52A4CDB
:20F0B000A07830F0010708D0042806D0032804D0052802D008F09EFFA07804222349244D78
:20F0D00067790A70E73D95F8B820791CC9B261718A4233DB032831D005F08CFAA078194E5B
:20F0F000042809D131463C3991F83C0020B1D1F8881009B102208847207995F8C510421C13
:20F110009142C4BF401CC1B21248217105686868298902F0FDFA68680088000904D3314647
:20F13000087808B106F098FBA078052803D1607908F0D8FFF8BDF9F7E3FBF8BDE12002F011
:20F15000C5F8F8BD901200205418002018310020B30C00209C0A002070B505462B4C28784A
:20F17000ADF1200DEB2829D040B3E92806D0E12843D14FF4FA7007F091F93EE004F1560119
:20F190000878401C087094F85200032818BF042803D14FF4FA7007F081F994F85600032800
:20F1B00009D094F85200022827D104F10800102108F0A2FA21E007F053FD1EE094F8520080
:20F1D000022817D104AE6946304606F003F95220002108F0B3FBE06820B1026812B130464F
:20F1F00069469047042006F0D3FF04F10800102108F082FA002084F8560005482A300168E9
:20F2100009B12846884708B070BDC046B01100200612002030B50446ADF12C0D08F00EFED9
:20F23000002818BFFC2050D168462146112201F0B9F9A57C617D8DF81250607C8DF815102B
:20F25000E37C8DF81100227D8DF81330A57D8DF81420002105B10121257E8DF8161094F894
:20F2700025208DF81850E07D8DF8252094F824308DF81700E58C8DF8243004F119010B2223
:20F290000DF11900ADF8265008F0C0FC607C1A2550B9812007F05CFD04460A94A4B1FF2106
:20F2B000812209F00FF909E09DF81510880000EB411080B207F04CFD04460A9424B10720DD
:20F2D000694603F061FC002528460BB030BD10B5401EADF1380D28D0401E09D0801E4FD0F2
:20F2F000401E43D0401E3FD0401E3BD0002048E001A800F063FB04460CA942F2090005F047
:20F3100095F89DF83000002808BF002203D0022007F02AFA024601209DF83010009001ABF0
:20F33000204605F0F8FB0A3028E001A800F046FB04460CA942F2080005F078F89DF83000EE
:20F35000002808BF002203D0012007F00DFA024600209DF83010009001AB204605F0DBFBF0
:20F37000001D0BE020200CE002200AE042F2130004A905F05BF804A808F07EFD80B200E0D0
:20F3900004200EB010BD704728482DE9B0410025DFF89C80294C0570ADF1140D88F83B50B4
:20F3B000012088F83800201D006888F83D50804720490F686FB1797E8A0806D341F0010156
:20F3D0007976397E01F0FD01397657F80C7C002FF1D1A1688847102008F06CFE082008F087
:20F3F00069FE98F83C00E0B90920134C8DF80000B4F8BA108DF80F50E027ADF8021094F880
:20F41000D7308DF8017094F8E6208DF8043094F8E7108DF8052068468DF80610FEF722FE09
:20F4300001E088F83C5005B0BDE8B08154120020BC160020C00A0020CC0B0020F4120020C5
:20F45000F8B505460E460520287096F849006968E870F06B4861686806F1280108F020FD8A
:20F47000B6F842006968488196F84600696848746868002404761F4869680078C873686868
:20F4900006F11C01193008F0CEFF307C69688873706810F8011B6A68918110F8013B6A68CC
:20F4B000918941EA0321918107786A68F91117F007071174214607EB470218BF0121891890
:20F4D0004018401C10F8011B297201F00702E860491001F0380101EB4201401872683189C9
:20F4F00068618B18834239BF2C72211C801A091A2974F8BDB20C0020F8B5064608F0B2FF69
:20F51000264D0746A91991F8EE00421C002881F8EE203ED1224C04EB8604267806F03F000C
:20F530003F2801D0FFF7E8FF648836F07F0018D1F0090FD24FF0805000F5DC75D0F8B8017C
:20F550004169204688472868416B204688470128F9D11EE005EB8405D5F80411012088470F
:20F5700017E04FF08055D5F8B801C16920468847D5F8B801416A20468847D5F8B801C16A74
:20F5900020468847074901200860074908688008FCD3384609F05AF80020F8BDE40C002088
:20F5B000B009000028200860282008402DE9F84F294C8A468346211D08880A254FF0FF0993
:20F5D000002604F13C084746401C088038465946082207F009FD30B16D1E07F1080706F19D
:20F5F0000106F3D100E0B146B9F1FF0F05D1207A401C2072FF20BDE8F88F4846694602F0C9
:20F6100063FD0546FF2DF5D09DF80000012806D0A06B05EB8501401880F804A004E0606B06
:20F6300000EB451080F81FA009490A6808EBC900026049684160074E7068804794F88C10F3
:20F65000491E84F88C10B16888472846BDE8F88F680D0000F4120020000F002038B504F0EE
:20F67000C9FF02F019FE224D05F13C00007820B1214808380168012088472048007810B914
:20F690001F48007808B108F0B5FC1E4C606880471D4AA1681378022B20D10123154C1370FF
:20F6B000A378022B12BF032B832313708847A17831F0010008D0042906D0052907D10020BF
:20F6D000607108F00FFD01E0F9F71AF9A178022918BF032903D103F04DF800E0884795F8D2
:20F6F0003C0020B1286D10B1102008F0E3FC38BD5412002054180020581400201431002098
:20F7100016310020F41200201831002010F47C1F70B51CD110F00F0F1CD00146002401229A
:20F7300002EA010091435200401E0BD0401E07D0801E03D0001F07D1093404E0241D02E08C
:20F75000E41D00E0641DA4B20029E9D133E010F00F0F01D0002070BD064602244FF4803545
:20F7700005EA0600AE436D00B0F5803018D0B0F5803013D0B0F500300ED0B0F5802009D0E0
:20F79000B0F5002004D0B0F580100FD1072008E0062006E0052004E0042002E0022000E07F
:20F7B0000120FFF794FD2418A41CA4B2002ED7D1022CD8BF0024204670BD704790B50446A7
:20F7D00000214022ADF1440D684602F0A2FAA0788DF80000E0788DF801009DF8000000BBA0
:20F7F000616811B101A805F073FB217A01F007028DF82820E0689DF82870C1F302118DF83F
:20F81000301027B19DF828100B9000EB41009DF8307007B10D90207C8DF8380067690F97D3
:20F8300019E0616811B101A805F052FB677A8DF82970A37A8DF82A30207A8DF82800E27AAB
:20F850008DF82B20217B8DF82C10677B8DF82D70E389ADF82E30034800680169684688475E
:20F8700011B090BD08190020F0B5012904460546ADF1140D04D0022941D142F2030001E0DD
:20F8900042F20200694604F0D1FD04B16D1C07F087FAC01DC010C0B2002830D00023064645
:20F8B000ADF1010C1F4618461CF801EF00224EFA02F101F00101884211D028B97F1CBFB2DE
:20F8D0005CB102EBC30103E03CB102EBC301491E05F8011B091205F8011B80F00100521C46
:20F8F000082AE4DB761E03F10103DDD130B12CB1D800401E05F8010B001228700FB900203E
:20F9100005E004B12770012000EB870080B205B0F0BD70472DE9F843254C804660688047B1
:20F9300081466946722007F00FF93225FF27002600994046091D07F0B1FF012808D0009888
:20F950006D1E06F1010600F118000090F0D100E03746A16848468847FF2F18BF381C22D1A5
:20F97000144DD4F804900A2700263C3512492846082207F039FB30B17F1E05F1080506F158
:20F990000106F3D10DE040460168296040686860C847064A92F88C10491C82F88C10A168AE
:20F9B00088476436F0B2BDE8F883C046000F0020F4120020000F0020680D000070B504469E
:20F9D000E820ADF1280D09A904F062FF9DF82400694607F065FD00280CBF00981E480DF185
:20F9F00025016060E82004F053FF9DF8250004A907F056FD58B90599C8200322B1FBF0F0CA
:20FA1000401EB0FBF2F15143401AC0B200E00020207207F0C5F900216081656821700F4B89
:20FA300061700A4608925968A9420CD1197A267AB14208D15989814205D1187820705E7802
:20FA50006670104606E008990C33491C06290891E9D901200AB070BD38C40D0098140020D8
:20FA70002DE9F047254C01258246984691460E46C4F87C570320C4F8805708AFC4F884077E
:20FA9000D4F88C0710F0030FFAD1387858B14FF08057D7F8B001016A27208847D7F8B001CA
:20FAB0000169272088470220C4F8FC06C4F80894284608F09DFCD4F808040008F8D2D4F809
:20FAD0008C07800F28BF281C15D2B8F1010F14BF08200C20C4F84C051021C4F85015002083
:20FAF000C4F85405064A1560C4F800A0A160C2F800542662A162BDE8F087C046044002407E
:20FB100000004842B0B50546264CE968E06888423FD1A86803F09CF9A0B1E9684968A06CBF
:20FB30000978022900D168B9012005F07DF8832835D1E068783008F08BFC04F1C80008F0B7
:20FB500085FCB0BD16492869A1F10802136805F110071843106097E80C0051F8102C181C84
:20FB7000104341F8100C00270F60A86841F81C0C0F68002FFCD004F13C0008F0B2F82564F8
:20FB9000206CC06840680078022808D14FF4004101E04FF4806104F1EC0008F081FCB0BD32
:20FBB0001C100440A820002070B52248204D4FF080562865D6F8D8011F4C036801210A4650
:20FBD000ADF1400D20469847D6F8D80142680121204690471948012606601948F9F7B2FF45
:20FBF00005F058FB284607F039FF05F118044FF4E13029462060002005F06CFB11493C2287
:20FC1000082308600021684608F010FDF0344FF46170002307940C4908906A46069605F148
:20FC3000580008F0FFFC08F0F9FC10B070BDC04608020020318401000040034004011CE223
:20FC5000980A000098060020A53600002DE9F041DFF8948006460C4636F07F0014D1002ED1
:20FC70003DD1224D686880471E49096831F81620144321F81640A968884741461431086847
:20FC900007F0DEFABDE8F081042007F09BF9071C25D04FF6FF7038807C8008F0EFFA4146D8
:20FCB0008C78A7F10C05FF2802D0C96A40184478FF2C06D1384608F05BF907F067FCBDE87C
:20FCD000F081304607F0B2FD01463A46FF20A872204606F0BDF810B1384608F049F9BDE858
:20FCF000F081C0460831002034170020F412002070B50025ADF1200D07A8ADF81C5008F0C6
:20FD100051F9234CBDF81C10208F884237D194F85300032811D004280DD0022810D104AE07
:20FD30006946304605F056FBE06820B1026812B1304669469047042000E0032006F028FAC7
:20FD5000A06D06F0ABFB5220294607F0F7FD07F0E9FF044607F0E6FF00EB042407F0E2FF2E
:20FD70004FF47A7200EB0420B0FBF2F15143401A0A3006F0ABFB284606F0C0FB05E00320BC
:20FD900008F0A2F8052006F003FA08B070BDC046B011002025483EB50078002843D042F296
:20FDB0000100694604F042FB42F2050002A904F03DFB1D4D95F8540010B39DF80800002473
:20FDD0009DF80810009B2864642285F85440581A02FB00F1E96705F1780003F057FF01A898
:20FDF00005F0B4FB124801992E300078B1FBF0F2451E4243891A01918D4214D9204610E0C8
:20FE10009DF8081064204843E86705F1780003F03DFF288F401C288700242C64012085F816
:20FE3000540004F011FD3EBD402D0020890C0020FC2D00202DE9F041224C064604F1580088
:20FE500005780F46002D04BF0020011C1CD0204D1D49281D0B780068D3B91C480568E06CFB
:20FE700008F050F8228FB0FBF5F1B0FBF5F3891889B203FB05F2236C3980801AC018306042
:20FE900085421CD8401B491C30603980BDE8F08180475FFA80F804F1780008F04BF9226CA9
:20FEB0004FF47A73410001EBC001B1FBF3F0238F3060A9683B808018306040468847BDE855
:20FED000F081C046402D0020890C0020042E0020F4120020F8B50546DFF890C06B68297A4C
:20FEF0002C681A680CF106070801A0EB4100C1194E88B1F804E0395A40F2011048401C49FD
:20FF10000143D0680140D160D1684E20B0408143D160297A04270801A0EB410000216044EF
:20FF30000C3030F8026B7F1E46EA0101F9D19069884390610EEB020751624FF0FF31B96253
:20FF500039630026BE633E649879FEF7EBFF08F089FA2178002904BF6670A67002D0297ABB
:20FF70006418667008F072FBF8BDC046580B0000FEFEFFFFF8B50F46002302B90123DFF8C7
:20FF900090C00021EFB13D6ADDB1C669CEB1FC68C768A74207D0DCF854110CF5AA77A142CC
:20FFB00014BFF968B968B4086FF05047A4EB9504641AA74225DDB4F1704F01DB002C20DD30
:20FFD00001210AB3D769FFB1066AEEB1D268C068824208D0DCF854310CF5AA70934214BF19
:10FFF000C068806800E00020C0EB97006FF05042BE
:020000040001F9
:20000000A0EB9600824204DDB0F1704F03DB002801DC0020F8BD012301EA0300F8BDC04635
:20002000A82000202DE9F043254C0746283CA06AADF1240D00283ED0002F3CD0387A002849
:2000400039D004F081FE5FEA000834D0062000250323A1468DF808002E46ADF80A30B5F5ED
:20006000FA7F28DAD9F82800ADF80C5004AB02AA0469009392E803000A230022A047B0B994
:20008000387A9DF81810814210D1022804D1BDF810103A88914207D0032807D104A93846DF
:2000A000082206F0A9FF08B9284606E0761CB04505F10105D3DC4FF0FF3009B0BDE8F083F2
:2000C000200E0020F0B520480127F84201D004F0E5FA204D204F214EBD4206D203CD047851
:2000E000A4003459401CA047F6E71D48002800D08047164D164FBD4202D210CDA047FAE74B
:20010000F0BD03251BE0416808300A1C2A400BD11A1C2A40AB4305D0046804300C6004311E
:20012000043BF9D1131C05D0047801300C700131013BF9D1021C2A4001D0A843043003686E
:20014000002BE0D17047C046FFFFFFFF0000000000000000E894010048950100A894010072
:2001600055C5011070B504466068254E4078ADF1480DC00921D3B4F842003546E63DB5F809
:20018000BA10884219D11D480078A0B995F8C40098B104F1280006F093FD70B90120009094
:2001A0001C340194B5F8BA3005F1AA0203210620F6F7D6FC1FE007F0DFFA0BA8002118223B
:2001C00001F0AFFD02A821460C900BA8FFF740F92C208DF82C000BA803F05AFC3546503DF2
:2001E000287810B19DF83C0028B105208DF82C000BA8FDF73FFF12B070BDC04655120020BD
:20020000B20C002003B426482DE9F041058806AF1446ADF1080D98464FF6FF70ADF800000E
:200220000222ADF802006946ADF8040044F40040ADF80600601986B2304602F0FDF9BDF8B4
:200240000600022269466FF3DF30ADF80600304602F0F2F9A1102846CAB2414602F0ECF95D
:20026000387840F40040ADF800007888ADF80200B88802226946ADF80400304602F0DCF915
:20028000BDF80000022269466FF3DF30ADF80000304602F0D1F902B0BDE8F04102B070479D
:2002A0005E1900202DE9F843002A894607464CBF47F6FF75151C002F08BF002033D038884A
:2002C000002808BF002403D02A4600F0D7FB0446281B002826DD388828B1291B484613A22E
:2002E00004F0DCFD0419B868E0B1D7F804802E1BB8F1000F0DD0404607F0C6FD401DB042A3
:2003000007DC291B48460AA2434604F0C7FD04192E1B122E06DBBB68291B484606A204F023
:20032000BDFD04192046BDE8F883C0463A2000C0222573222C2000C06C696E652025643ACD
:2003400020007047F8B5044608F094F8234D064605F5C4710878A04305F5AA7408702068E5
:20036000002808BF002706D020689C3007F042FE002700B10127606838B19C3007F03AFE5A
:200380000024384318BF0124274695F8880100BB012F1ED0D5F87C01F0B1016A89080ED29F
:2003A0004469304608F05AF9D5F87C0100214FF400030A46A0470020C5F87C01F8BDC469AB
:2003C000304608F04BF9D5F87C0102210022A047F1E7304608F042F9F8BDC046A8200020D1
:2003E00070B50546234C287800283CD16078012839D0281DFFF716FEB0F1FF3F33D1298A5A
:20040000C81330D001F00F010F292CD12046018F4FF6FF728A4203D0EA898A4204D101E08B
:20042000E989018701218170A97C80F83A10AE888687298A01F00F020F2A05D080F85020DA
:20044000C1F3031180F8511090F850100F290AD1012141700848064607F004FE012802D19C
:20046000304608F02DF86C34216809B12846884770BDC046B0110020B80E0020BFB507F064
:20048000D1FA0446214D2249286981422FD1214905F17000002207F0F5FF0120287007F08D
:2004A000FBF8B5F8C47000204FF6FF712871B94209D10220ADF80000684606F075FBBDF895
:2004C0000800A5F8C400286C60B905F13C0007F0E3FF071C06D005F05BFB40B93846FFF74A
:2004E00019FB04E005F1EC00022107F0E1FF04F0804104F00200084305D005F1EC004FF03C
:20050000005107F0D5FF0090BFBDC046A8200020152E000051C50000F8B5244D01200146E6
:200520002870F6F753FF6FF001001F4C1D4927690870381C28D0A1684268914203DA07F005
:2005400061FD27693846C8B105F0AEFB7968884224BF2769381C11D201F016F814E0266941
:200560007068002802D507F04DFD2669304603F0A3FEB168307B88472769384620B105F063
:2005800093FB79688842EAD2094C606880470646FDF710FFA1683046884707F033F90020A2
:2005A0002870F8BD3919002014190020E8190020F4120020002A4AD05FEA000C8B071CD1D0
:2005C000830722D1102A08D370B4103A78C978C0103AFBD270BC103238D0042A2CD3082AB6
:2005E00005D30C2A24BF08C908C008C908C008C908C092072AD0920F22E00B780370491CAE
:20060000401C521E22D08B07F7D1C30714D18307D8D0121F12D308C903801B0C4380001D70
:20062000121FF8D20AE008C903701B0A43701B0A83701B0AC370001D121FF4D2121D05D031
:200640000B780370491C401C521EF9D160467047F8B507F00FFF234C0746D4F8C00010F44E
:20066000602F33D0D4F8C000400CC6B2700807D2B00803D2F00828BF022602E0012600E0CA
:200680000026751D002168B203F044F8D4F8C03006F111010120884023EA00013846C4F842
:2006A000C01007F0DBFFB00004F1A8010A18D7682FB1085800224FF000632946B8470A4826
:2006C000006830B9022004F0B7FA02E0384607F0C5FFD4F8C00020B104F59070002107F079
:2006E000E7FEF8BDA82000200C1004401CB51F4C04F1780006F0F4F904F15C0006F0F0F95C
:2007000004F1940006F0ECF90021882204F1340007F0E0FE07F018FB06F04AFB84F85A0091
:20072000134984F85B001348086001200DF1010184F8B30042F2040003F080FE42F2050091
:20074000694603F07BFE0C489DF80110A0666420414321660949C4F884109DF8001048431D
:20076000E0670748C4F8A0001CBDC046402D0020501400209D620100A5430100A5FD00000C
:20078000D7830100D0B5244C04F124010F68002F3FD0002215280AD13B7D0126022B08D01C
:2007A000032B06D0052B04D0042B02D000E03B7D0026984200D016B17B7E5B0905D23A464D
:2007C00057F80C7C002FE5D123E00846394605F069F8F88A2760000A03D397F91C0007F0AB
:2007E0002BFB387D022818BF052802D1012006F0CFFD2068407E30F07F0005D194F82F00C4
:20080000401E84F82F0004E094F82E00401E84F82E003846D0BDC0469C0A00202DE9F84301
:20082000234D884606464FF0FF3105F12400814607F094FB00200CE0FF2909D02A688A42ED
:2008400004D905EB8101D1F894700FB1002627E0401CB8F1000F03D018F82010FE29EBD185
:200860000024346074600127B46011E0FF280ED005EB80000B787268C0F8946007FA03F04D
:20088000104370600A680949304605F051FB641CB8F1000F04D008EB84010878FE28E5D1DA
:2008A000484607F0FDFD3046BDE8F883007FC767C4270020B0B5456884682349607DA27D05
:2008C000ADF1180D40F000400090207D0027FF2A41EA000001904FF0020002D0E27DFF2A11
:2008E00000D13FB1E37DA07D1943039140F0004002900420FE214DF8201005F15800694613
:20090000FFF78CFF6866002808BF381C1AD0617D0F2205F089FF686E217D102205F084FFB1
:20092000A17D3846FF2902D0E27DFF2A00D140B1686E112205F078FF686EE17D122205F005
:2009400073FF012006B0B0BD0000C0A038B5054695F83000032839D195F83A00032835D15F
:2009600005F128044A202146F6F734FE8A202146F7F718FD6C686178207800EB0120ADF85B
:20098000000069465020F6F725FEA41C6178207800EB0120ADF8000069464B20F6F71AFE27
:2009A0008B206946F7F7FEFCA41CE1202146F6F711FE641C6178207800EB0120ADF800002F
:2009C00069465320F6F706FE002000E0E82004492A24087028462C7003F05AF838BDC0469F
:2009E000952F00202DE9F8432020EFF3118780F31188214CA068012107F014FE4FF0010913
:200A00004FF0000865692168A4F81C906A1A2168A4F81E80461B401A904227D387F311880F
:200A200040464519361A4846294607F0F7FDB042F7D92021EFF3118781F31188E18B01297A
:200A400003D14046294607F0E9FDB0F1FF3F06D0A169801B814238BF081C411901E0A06974
:200A6000291807F0D7FDA4F820902560A4F81C8087F31188BDE8F883780100207FB5034618
:200A80001F480D4601881F480088144614A6984205DB32462146284604F000FA1DE0994243
:200AA00006DB184606F0F4FC0028F2D04268F1E715480088002808BF0CA2EBD00095002CA7
:200AC00048BF47F6FF74114E0020114901946A46346802901846A047029800907FBDC04662
:200AE0007B6D6F64756C652325647D007B6D6F64756C652D726F70653A25787D00C046C0CE
:200B0000D20C00004E0D00008E140000D00D0000ED66010090B50C46214A0178575CADF1FD
:200B20001C0D0B2F8DF8007035D0002F36D00C2F04D0112F29D107F023FA26E01A2C22D088
:200B400090F899100190C7688DF80210038A0297C28AADF80C30510905D21249827EC83135
:200B60000978891A00E000218DF80E10877F8DF8107090F91F308DF81130826A0592417FC1
:200B80008DF80F1001E0002001908DF801406846FDF770FA02E04470FCF782FF07B090BD3F
:200BA00094030000CC0B00202DE9F04107467868BE68044600F5847007F052FC30681C4998
:200BC00080690968C0F3C00008BB07F053FC194D8046287820B1022005F0C4F90020287016
:200BE000404607F03BFD3168134D886B20F020008863286820F480702860606A216A091AA5
:200C000021622369626A38469847BDE8F0814FF4FA70B0FBF1F1012998BF012104F58474B8
:200C2000204607F019FC204607F018FCBDE8F081043100200D310020301000402DE9F04141
:200C400007467E68D6F8BC00C8B307F013FC1D4D00248046042305F10C00046002202B60C8
:200C600007F0CEFB7368D6F8A810384622469847022005F077F90BE08069C6F8BC007368DE
:200C8000D6F8BC10224638469847022005F06AF9D6F8BC00D6F8C0108142EDD134722046C6
:200CA000C6F8A800C6F8BC00C6F8C000064B2C6038461C6003F00EFC404607F0CFFCBDE815
:200CC000F081C04604280040100405422DE9F04180461E4800680D464169272088470124C3
:200CE00004FA05F61A4DC5F80064C5F87C470327C5F8807717480460C5F88477D5F80404C5
:200D0000012818BFC5F80444C5F8FC6312480460C5F800801023AB60204607F071FBD5F8E3
:200D20008C074008F8D3D5F88C17204611F0404F09D1C5F884770021C5F8FC16D5F8002434
:200D4000164218BF081CBDE8F081C046B00100100440024000E04842000048422248F8B5D2
:200D60000C460178012904D0017A012918BF012034D190F8C710CA080AD390F8C620A242A8
:200D800006D101F0FB0180F8C710002780F8C67007F070FB074607F087FB0646012120466F
:200DA00002F0B8FC0E48210201F47F41084305F0FBFE0C4A1168054604F10C03012098400F
:200DC00081433046116007F045FC384607F046FC05F0FF05012D0CBF81200220F8BDC04609
:200DE0000100080408100440A82000207CB515460E46044600E004192046694605F0EAF98E
:200E000000282ED014F8021F8E42F4D1491E04F1010420D0491E12D0491E08D0491E18BFD3
:200E2000622029D102281CD12078287023E0032817D114F8010B2870207868701BE007288F
:200E40000FD161782078A41C40EA0120288020682E1D30600FE0052803D1207806282870DD
:200E600001DD67207CBD2D1D0020641C2860A678AE702088288000207CBDFEE7D0B5ADF175
:200E8000180D04F0AFF9684606F090FF0020039001248DF8084069468DF8004040F61E7081
:200EA0000190022004F0BEF9061C00D1FEE707F034FA022730466FF0004107F029FA0E4828
:200EC00007F09EFA30464FF0FF3107F021FA0B4807F096FA7F1EEDD1304607F023FA304657
:200EE00007F011FA0648074904604FF480570F6006B041F8107CD0BDE03F1200A0BF360097
:200F0000301A4442A020024098B54368C3F8A8100868C3F8AC004868C3F8B0008868D3F8E7
:200F2000B070C3F8B400C8681949C3F8B80017488FB9D3F8A820127C520042F0010202606C
:200F4000022018720A68D20916D2D3F8B820022A16D30B2215E0D3F8A820127C012752003B
:200F60000260D3F8AC201F72541CC3F8AC40127882600868C00902D34FF0FF3098BD022071
:200F800003220A6007F03CFA002098BD00280040042800402DE9F0411E4615460F460446A7
:200FA00007F082FA8046384605F0ACFC071C04D097F8270030F07F0003D1404607F04AFBFB
:200FC00028E097F8270010F00F0F1BD113487968884202D07968A166786004F1600080E8F4
:200FE0006000404607F036FB04F140004FF0FF3106F0B4FF04F170070020A06697E8030082
:20100000BDE8F081404607F025FB97F8270010F00F0FFAD102200021BDE8F08147320100AB
:2010200070B506467468B568606E06F050FA29681C488A6B10408863304600F037F8304608
:2010400001F0DAFC2968C86A20F01000C862296815480A6B104008636868FDF76BFF04F17B
:20106000800007F005FA04F19C0007F01BFAA07818B904F1D00007F011FA607818B904F10F
:20108000EC0007F00BFA04F5847007F0DFF907F0F1F90021217007F0E1FA04F16C0006F0F0
:2010A00037F970BD0DF8FFFFFEFCFFFF2DE9F04106467568B46807F0DDF9A96A39B92168F1
:2010C0008969090903D207F0C9FABDE8F0810027AF6207F0C3FAA17D3846FF2902D0E17D87
:2010E000FF2900D118B12846214600F043FF2168886B20F0200088630D49086820F48070C6
:20110000086007F0B7F90B4C8046207818B1022004F028FF2770404607F0A0FA686A296AF2
:20112000091A29622B696A6A30469847BDE8F081301000400D31002038B50C464422054660
:20114000002100F0EEFD04F12801284606F0B2FC04F1320105F10A0006F0ACFCE06B686189
:20116000B4F840002883B4F842006883B4F84400A88394F84600A87794F84700E87794F934
:20118000480085F8200094F8490085F82100B4F850006884E06C6862A07B85F8280094F8AD
:2011A000520085F82900606D0B2204F11C01E86205F13000FFF7FEF92089A5F84000606880
:2011C000E86338BD70B5214C06460E220D4604F13800FFF7EFF9687B28B9022084F82800D9
:2011E0006B88238409E003202B1D84F828001A6804F120010A6058684860206B05F06EF90C
:2012000030462946FBF79CF8207801280BD0687B48B9288869882A1D02F096F9011C02D08B
:2012200006A007F0F0F8256905F0B2FF6421401B2061B0FBF1F0A4F87C0070BD4175746831
:20124000204572726F723A20307800C0E810002010B5204CE8B904F174010022087894F820
:201260003C30A26300F0F000087003F0F00094F8403084F83C0004F1410143F0080000F0AC
:20128000EF0084F84000F42003F00AFB44F6206015E094F8400040F0080000F0EF0084F889
:2012A000400003F05FFE0A2280B24FF4FA6390FBF2F1514344F62062401A03FB0020064A1A
:2012C000A06492F83C1019B1D2F89C1001B1884710BDC04608100020541200202DE9F84391
:2012E000814600261B481E4D06701B48DFF86C80067098F83C00E8B1D8F880702C68CFB1E8
:20130000207D352809D16068218900F009FA60680088000901D304F0A7FAD8F880104846E4
:2013200088471048007801280BD030460146F6F74DF806E003F066F900F0B6FF4846F8F7C1
:2013400075FA286810B1007D352801D006F02AFCBDE8F88310310020183100205412002096
:201360009C0A0020E819002070B51E4DAC68064606F034FB4FF47A71001B4843030C05F099
:20138000FFFB2969401A48BF404240F6B8319B19994210D306280EDAE9688C420BD82868A5
:2013A00048B1114A091B51438A0C02EB1141884288BF011C08E00D49486840080ED2086898
:2013C0007D2100F0FF004143C82905D3B1F57A6F88BF4FF47A6103E0C82101E04FF4FA61F4
:2013E000084670BDC030002040420F00AC3F00502DE9F8431F4C00264FF001084FF0020922
:201400003746A51E15F8020F03280FD0022824D168786368022820D0304606F092FF01463C
:20142000384606F00FFF85F8019011E0304606F088FF014663686878012805D0384606F0D4
:2014400001FF85F8018003E0404606F0FBFE6F700246C9B2184604F063FB761C022ED1DB76
:2014600005F0DEFB18B104F1200007F027F8BDE8F883C046781600207CB5042005F0A8F9EB
:20148000022818D0032816D019480068C0F38150032814BF41F288324FF47A721649174C00
:2014A00009684C342046B2FBF1F106F0D5FF204606F0D4FF7CBD4FF08056D6F8A4010D4D32
:2014C000446800214FF040521C23032000902846A047D6F8A40100214FF40072092301268B
:2014E000446800962846A047022004F03BFD7CBDB43F005000A00C4004310020EC0C002032
:2015000003B42048F0B505AF3E787D880088BF88ADF10C0D001F84B2082C2CDB201F694694
:20152000082280B204F002FFBDF8000086420FD1BDF8020085420BD1BDF80400874207D149
:20154000BDF806006FF3DF30241A241FA0B213E0BDF80600C10BCB0309D100F108018C42A2
:2015600002DA06F04FFD06E0241A083C00E0241FA4B2082CD2DA002003B0BDE8F04002B032
:201580007047C0465E190020F8B51E4C002528462268A168256190420CD05268914209DD13
:2015A00004F082FB0146206842689142C8BF41602061A168676837B118B142687B689A42D3
:2015C00001DD38462061C8B14068814216DD0F4D044605F108000068A04201D806F012FD8B
:2015E000094E706880470746EC60204600F0E8FDFCF7E0FEB16838468847F8BD05F088FBBD
:201600002561F8BD14190020F4120020B81800202DE9F8431F481C4D07786868804781462E
:201620001A4883680026344680469C4212D013F8020C874208D134B163B138464FF4004181
:20164000FEF70CFB13E01C4604B91E4653F80C3C002BECD15FB9686880470D49096831F8FE
:2016600017206FF3DF3221F81720A96888472CB108F108002146324604F014F9A968484633
:2016800088472046BDE8F883F412002034170020083100207C13002010B504461D4920784F
:2016A000F0B98A7808466178012913D0022908D0032928D10021C1704021083006F024F826
:2016C00021E090F83A00FF280CBF0120022006F003FC18E0012A18BF011C0AD12021ECE717
:2016E0006278032A08BFEA2806D0012A0BD10020887041F2883000E0074891F8542081F885
:20170000552004F003FF05487430016809B12046884710BDB0110020E0930400B01100200F
:201720000829C8B50BDA00293BD00278491E92FAA2F24FEA226200F8012BF6D1C8BD46422C
:2017400006F00306891B37188AB2361802F00301864209D9361A0378761E93FAA3F34FEAB2
:20176000236300F8013BF6D122F00302D71987420AD93A1AD21C96100268761E92FAA2F22F
:2017800012BA40F8042BF7D1CF19874209D93F1A01787F1E91FAA1F14FEA216100F8011B60
:2017A000F6D1C8BDF8B50546012004F021F81D4C04F1140002F080FD04F1240002F07CFD52
:2017C00069684A78087800EB0220ADF800008F7804F114066FB953206946F5F7FBFE05F109
:2017E00028014A20F5F7F6FE05F128018A20F6F7D9FD06F1200005F11C010B2206F00EFA95
:20180000BDF80010384604F0FBFB94F83F00800803D36878002106F089F9002084F83F001E
:20182000F8BDC046042F00201C491B4898B5FF220F7890F83B301A4980F83820012B15D0A6
:2018400091F8A10091F8C010884224D015480024047005F08DFD01F02FFC134800780128BB
:2018600019D020460146F5F7B1FD98BD002380F83B3087B18DF8032091F8D7008DF8000018
:2018800091F8E6708DF8017091F8E7408DF80240684606F074FD98BDBC160020CB0A0020AB
:2018A000CC0B002015310020E81900202DE9B84106F0E0FD1C4C1B4D804604F1E0000078E5
:2018C00048B92C46A168022088470746102003F0C3FA17B31EE001F02DFA78B9134800689A
:2018E0003221B1FBF0F101B9012104F1300006F0B3FD04F1300006F0B1FD0EE0002084F80E
:20190000E0002C46A168022088470746102003F0A3FA17B1A16803208847404606F09EFE93
:20192000BDE8B881E40C0000E40C002004310020BCB5446867780D46684606F089FD381CA7
:2019400007D0401E18BF281C0BD10198B0FBF5F006E00198154A0023A5FB0001F6F73AFB6E
:20196000401E07466FF07F40B8420CD35FB1217B226901290AD051EA020007D002290DD06E
:201980006069B8420AD96FF00200BCBD384602F0C7FD01466161E06906F0E5FC6560A7609E
:2019A000E069394606F0DBFC0020BCBD40420F00F8B500201C4D1D4E1A4C85F83D0096F819
:2019C000A17094F84000401CC0B2042884F8400022D0202003F00CFF96F8E3200F2A0AD0A0
:2019E00095F83E0096F8A110814204DD174686F8A10004F003FE94F8401096F8A13035F860
:201A000017504FF4707204F11000491C9A4001FB152105F091F9F8BD04F00CFBFDF7BCFCE9
:201A2000F8BDC046E82F0020BC160020CC0B00201D491E482DE9F041352751F8048B51F83B
:201A400004EB51F804CB51F8046B51F8045B40F8048B51F8044B40F804EB51F8043B40F8D9
:201A600004CB51F8042B40F8046B40F8045B40F8044B40F8043B7F1E40F8042BDDD151F8E8
:201A8000045B51F8044B40F8045B51F8043B40F8044B51F8042B40F8043B40F8042B0968E2
:201AA0000160BDE8F081C0461489010000C0002170B51B4C05461022ADF1200D04F17101EF
:201AC0006846FEF777FD0026049509208DF8146004F10D018DF8160001258DF815500A68EE
:201AE0000DF1170002604A684260097A01720D496A4618200DF074FB0B4918208922631DC4
:201B00000DF06EFB7120314606F06CFAD520214606F068FA5D20294605F018FF08B070BD6A
:201B2000C406000035B30000A58300002DE9F0431C4E044600271D468846A2EB0409ADF13E
:201B4000140DC6F8B071012006F05AFC3068C00FF9D3306A0090706A0190B06A0290F06A4A
:201B6000039044B128462346694611F8012B5B1E00F8012BF9D10320C6F838026CB108EB90
:201B800009016D1E491E11F8010F15F8012F904218BF042002D1641EF5D1384605B0BDE833
:201BA000F083C04650450240F8B51A4E1A4D0120002414EA030730704FF0020000EA02003F
:201BC00008BF00280CD14FF0E04004EA0201184008BF002904D11249088C401C088403E012
:201BE00095F90000401E287005F0F0FD05F0DAFF0A48047095F9000030B195F900000028C6
:201C000006DC06F0FFF903E020460146F5F7DEFB3470F8BDE8190020421900203B19002036
:201C2000541800202DE918410446DFF870802078E02828D140464278C178012A0AD049B97F
:201C400090F85220012A05D190F8540001281AD001200CE0104BB3F87220521CA3F872205A
:201C600041B9491CC9B2C17000234370022006F033F908E0002004F019FC032006F02CF9F0
:201C8000052004F08DFA40467C30016809B120468847BDE81881C046E8100020B0110020DD
:201CA000F8B500680E4617464FF0FF310446483006F054F94FF0FF35092E08D0217A0120AC
:201CC000B040084211D108433546207210E0227A0721012303FA01F0104202D0491EF9D571
:201CE00003E0227A0D4610432072B5F1FF3F0ED06FB129463846FEF7E9FF40B1217A0120D4
:201D0000A8404FF0FF3580F0FF000840207204F1480006F0C5FB2846F8BD002213460A463E
:201D2000194671B510F0030F0BD0002A82BF00F8011BB2F1010210F0030FF6D1002A08BF42
:201D400071BD11F0FF0141EA0121042A18D341EA0141082A0FD30E46102A08D30C460D465F
:201D6000B2F10F0312F00F0272C0103BFCD812F0080F18BF42C012F0040F18BF40F8041B15
:201D800012F0020F18BF20F8021B12F0010F18BF017071BDF8B5054606F06CFB1A4C0126BA
:201DA000074605F19C00A67006F05AFB2078012811D094F8880170B1B4F95000B4F95210FF
:201DC000884208D1384606F049FC0720FEF7BAFA06F050FB0746B4F95200B4F95010884273
:201DE00018BF85F8C2600AD105F1780006F038FB304602F021FFA17920780843A0713846E7
:201E000006F02CFCF8BDC046A820002038B51B4D95F8A1000F2824D0194C3B3C94F83810A3
:201E2000FF291ED094F83A0068B102290BD103F03BFF216B0F4C95F89820401A2178083121
:201E400001FB12010BE003F02FFF616B0A4B95F8C020081A1988401A34F81210411A0029EA
:201E600001D5002038BD4FF6FF708842C8BF88B238BDC04665170020C80A0020CC0B0020B8
:201E8000F71600201749B0B50546154C0F7820780FBB154A8100B2FBF1F1A94202D206F097
:201EA000B1F820786168134F800005FB00143868C06B8047211AA1F54871090806D30B4AC7
:201EC000011B891A090828BF00F548740A482146FBF712F9B0BD064901200870B0BDC0461C
:201EE000B8180020E9190020FFF6C2FF00093D001731002060140020E5E200001C4938B5BF
:201F000091F85C3001EBE304657F012203F0070302FA03F383F0FF032B4063778B7E01F12E
:201F20001800032B18D091F86030012B10D0022B08D0B1F856108A409102A1EB821101F5C8
:201F400070710EE0B1F856209101A1EB820108E0B1F856108A4001E004490A789102A1EB62
:201F600082111C3005F05CFC38BDC046950C00207C2F002038B50C4621680546886B20F098
:201F800020008863686E217D012202F0ADFC686E217D012203F0C4FD686E217D002204F02F
:201FA00043FC686EA17D002204F03EFCA878012806D005F1D0004FF0FF3105F0CFFF03E0A4
:201FC000216888690009FCD2686E217D102204F02BFCA17D0020FF2902D0E27DFF2A00D15E
:201FE00018B1686E112204F01FFC38BD2DE9F84F8346894617467120114604F0ADFD812092
:202000006946F8F755FE4FF0F308002507E0B8F1000F23D038686D1CEDB22C3038609DF88D
:202020000000A8421ADD3868066890F804A0002402E0641C0A36E4B2A245E8DD737A002B65
:202040000CBF052009208145F3D14A463046594605F0BEF90128ECD14FF000084046BDE834
:20206000F88F70471A487CB5007880B342F2050001A902F0E3F942F20100694602F0DEF986
:20208000144C9DF80400216C88420BD80098884203D806F0E9F901250DE00022012584F821
:2020A000542004E001259DF8040084F85450401A64214143E16704F1340606F1440004F0E0
:2020C0000FFD06F1440001F0E9FD84F858507CBD890C0020402D0020F8B50B461A4991F859
:2020E00031708D6B4C7A6430C2B25FB100206D1F6D1DEE7816B12E79B24207D07F1E00F106
:202100000100F5D1641CE0B2487204E0FF281CBF0021197016D10120187091F830704C6B2C
:202120004B7A5FB10020203C2034A67F16B1E57FAA4207D07F1E00F10100F5D15B1CD8B291
:202140004872FF20F8BDC046000F002038B5054601201A4C68712879B0B90DF016FC217872
:20216000002904BF6FF00704051C15D0491EC9B2217039B90DF033FC606804F0CFFA0020CD
:20218000687118E0054613E00DF0FFFB05462078FF2805D16FF0060428460DF020FC0BE07E
:2021A000401CC0B20128207002D1606804F0CDFA28460DF014FC0024204638BD64190020AB
:2021C000154998B50F7817BB19490A784968930000FB0314114B9700B3FBF7F1814201D2A2
:2021E00005F010FF0E480068C06B8047211AA1F54871090806D30B4A011B891A090828BFAB
:2022000000F5487408482146FAF776FF98BD07490120087098BDC046E9190020FFF6C2FF7F
:202220006014002000093D001905010017310020B818002038B517481749007818B908460A
:20224000007828B906E00846007830F07F0001D005F0D8FE114D68688047114C0C3C21780B
:20226000A278914207D10F4AA9681278D20803D28847012038BDA968884705F079F8A078B3
:20228000FCF77EFC012804BFA078207005F08AFC38BDC0469012002018310020F412002076
:2022A00070170020153100209EB5164C606880472146154C2289E388934220D0134B1F7835
:2022C000EFB9134B89681F7837F07F0718D1E28088471027E088ADF8007001A9ADF80400A2
:2022E00009880DF1020319800A49BDF804000A4A08801068426AE068694690479EBD89688B
:2023000088479EBDF4120020641700201631002018310020AA100020601400202DE9F84343
:2023200080461848077817B9174D287810B90120BDE8F883154E706880478146688801243C
:20234000B8F1000F0ED1214603464FF6FF72B9404A40104068807BB170B9002004F0E8FB79
:20236000044609E018B9204604F0E2FB68882146B940084380B26880B16848468847204691
:20238000BDE8F8837C1300203C140020F412002000B500212022ADF1240D6846FFF7C1FC90
:2023A0001748018FADF8181090F83A108DF80B10808FADF80E0002218DF8161009208DF8B1
:2023C0000C0001218DF80D108DF81F1000208DF808008DF81B006A468DF81A0006498DF809
:2023E0001D0018200CF0FCFE0449B1F85800401CA1F8580009B000BDFD820100E8100020E9
:20240000B01100202DE9F8438146EFF31188202080F31188174D154C134F012605F11C009C
:202420000660A4F114000660F86A016A14208847D9F81000810C14BF000C042020603868C6
:2024400002682321002090470948066054F8180C20F4C02040F4803044F8180C2E6088F36F
:202460001188BDE8F883C0468401001018200940800224430000244330B504460D4642F281
:202480000900ADF12C0D09A901F0D8FF9DF8240008B342F20B000DF10E0101F0CFFF002340
:2024A0000094BDF80E00029300040190684602F039FD044604A942F2030001F0BFFF04F0F4
:2024C00077FC024604A9B4FBF5F06843241AE0B202F02FF906E042F20D0003A901F0AEFFFA
:2024E0009DF80C000BB030BD2DE9F843194D064628780C469846012805D0287A012818BF20
:202500006FF0010024D162600A20208001F044FB071C1CD4A77005F0ADFF8146204604F0BE
:2025200043FB0446484606F099F804F0FF04012C06D03846012101F0EDF86FF0010706E041
:2025400005EB8705A83545F8088C45F8146C3846BDE8F883A8200020F0B50546194C287819
:20256000ADF11C0DE9281CD028BB002694F8520084F8566002281ED104AF6946384602F093
:2025800031FF5220314605F0E1F92046C06820B1026812B1384669469047042003F000FEAE
:2025A00009E094F85600401C84F85600C0B2032801D104F05DFB8C34216809B12846884727
:2025C00007B0F0BDB01100202DE9F04107461748174CC01F06786068804780461549A26846
:2025E000087886281CD1104D05F11E021088401C10808720087005F03DFEA168404688471C
:20260000082004F0D5FCE879B04207D127B90020FEF764FEBDE8F0811B20F9E7E920F7E733
:2026200040469047BDE8F081541800208C300020F4120020183100202DE9FC4716460C4629
:20264000054604F065FD164F814678688047804603F0BCFC8246B2002146484605F03AFEF9
:20266000504605F06DF802E02D1D241DADB23046411ECEB278B128466946042203F056FE96
:2026800068462146042204F0B7FC0028ECD00549012048700870B96840468847BDE8FC8737
:2026A000F41200205C1900202DE9F8430024002B16460F468046254606D5002FC3F100031C
:2026C00002D57F42761E2D2599463846494602F0A9FE0CA0405CB7FBF9F7002F04F10104E4
:2026E00008F8010DF1D1A64205DD3021301B401E08F8011DFBD10DB108F8015D4046BDE815
:20270000F883C046303132333435363738396162636465660000704798B5164C94F8E10003
:20272000002710B91448007860B105F0A3FE94F8E310002906BF012184F8E310012705F013
:202740008DFF0FB1002098BD022003F07FFE0E20FCF7DAFE094A106848B909494020C86087
:2027600008600127D761002084F8E20098BD012098BDC046E40C0020F20C000004800C4064
:202780002C500C40154880B50078022822D0052805D001281FD9C11E01291ED81BE005F039
:2027A000ADF948B10F490E4A097812688900B2FBF1F1401A48BF00200B490F7847B10B490F
:2027C00009780F2904D018B91C20FEF787FD80BD052000E00220F2F7C7F980BD561800200E
:2027E00050100020B8180020541200206D0C002038B5042903462BDA05F0A3FD05460846B4
:2028000005F020FD134C5B0002460229195503EB040012BF0329002141706068E9B203F0F4
:202820007FF904F0FDF950B904F12000044605F019FC01280CD1204605F042FE38BD04F139
:202840002000044605F00EFC10B9204605F036FE38BDC046781600202DE9F843174C04F165
:20286000240108688846074628B300261D25387D35281BD140463946324603F013F8787EF6
:2028800030F07F0005D194F82F00401E84F82F0004E094F82E00401E84F82E007D7057F81D
:2028A0000C9C384600F072FB4F4602E03E4657F80C7C002FDBD1BDE8F883C0469C0A0020FC
:2028C00070B544688668D4F8A40004F000FE154800250C30056040F80C5C1148056070687E
:2028E000FCF728FB04F1100005F0C2FD04F12C0005F0D8FD04F1600005F0D0FD207818B99E
:2029000004F17C0005F0CAFD04F1C80004F000FD05F0B0FD84F8DC5005F0A0FE70BDC046CC
:202920001004054204280040164880B507683FB315498B6803EA5300C00E21D2134A1068B5
:2029400080081DD2486880081AD21068096810F0050F4FEA114101F0F00101F5E0710AD150
:20296000B9420DD2190F38BF40F00100D90E38BF40F0040003E0B94202D920F005001060DD
:2029800080BDC04628500940AC3F0050000009402DE9F04180461748283007680E46ADF18A
:2029A000300DBFB13869A8B1B8F1000F12D08EB106208DF828000125ADF82A500022ADF8B8
:2029C0002C2002AC00943C690AAB93E803001A23A04708B100200AE002A940460C22FDF757
:2029E000E9FD05A930460E22FDF7E4FD28460CB0BDE8F081F80D0020F8B50646B0680168E9
:202A00007568886B20F4FA6088631349086820F40070086005F02EFD104C0746207820B1A3
:202A2000022003F09FFA00202070384605F016FE05F020FDA96B11B905F010FEF8BD0021E8
:202A4000A96305F00BFE686B296BEB68091A29636A6B30469847F8BD301000400C31002047
:202A6000F8B5844640F6FF741CF8013B002210E0481B401E10F8015B7F1E01F8015BF9D1F3
:202A800003E01CF8010B01F8010B521C5B08082AEADA5808F5D21CF8010B1CF8015B05F0BB
:202AA0000F07FF1CC5F30315122F45EA001508D11CF8016B300A24BF1CF8010B60F3DF16B2
:202AC000F719AC42D4D1F8BDB0B5184C05460F46101C28D00DE03868E06397F8270039460C
:202AE00040F0040087F8270004F14C0003F054FAE76BD7B1F8688542EDD014E0386888B1EF
:202B00003868C06885420DD139680868386091F8270040F0040081F8270004F14C0003F0E7
:202B20003BFA00E03F68002FE8D1B0BDA8200020084610B500F0005100F00400084321D018
:202B4000012003F045FE114C012813D00E4801683220B0FBF1F2012A8CBFB0FBF1F10121F1
:202B60002046A0F12404204605F076FC204605F075FC10BD064805F023FB06492046D838AA
:202B80000839086010BDC0460431002094210020152E0000081004402DE9F843DFF85880F0
:202BA000044608EB440000F11805008B894604F011FA074611480678AFB12A883846002158
:202BC00005F088FC00253C7041467D700A5D381D494605F023F83046394600F085FC40B97D
:202BE0002846BDE8F8838DF8004068461A21FDF791FF1A20BDE8F883880300007C13002081
:202C000010B5164A144C92F83D0094F8401048B91348006860B9012082F83D00202005F0A2
:202C200049FA05E0481CC0B2042884F840000DD00C49A1310A784FF4707304F1200003FAF0
:202C400002F101F2636104F0EBFD10BD202002F0CFFDFCF7A1FB10BDE82F0020BC1600209E
:202C60009C0A0020CC0B002010B5044600212822ADF1280D6846FFF754F81349112268461D
:202C8000FDF798FCFF228DF8182005208DF812008DF8114000218DF815108DF8161009229B
:202CA0008DF8132001208DF817008DF814000B220DF11900FFF735F8044918206A460CF06E
:202CC0008FFA0AB010BDC046DB06000025F20000C8B50146164AC87AB8B992F83170906BE9
:202CE0002FB3401F401DC6781EB1CA7F03799A4202D07F1EF6D1C8BD8A7FC270CA880280BE
:202D0000CA7F0271097B8170C8BD92F83070506B6FB120382030867F3EB1CA7FC37F9A42F5
:202D200003D12022FDF746FCC8BD7F1EF2D1C8BD000F002038B5012003F04AFD012820D04D
:202D4000114DD5F82401C4681048342101220023A047002808BF002014D0286803F04CFF5C
:202D600004F03CFE0B4A0A4D93681168D060C01AA1EB910105FB00F3180C884228BF011CF8
:202D80001160012038BDC0468000001000A00C4040420F00C03000202DE9F041071C0E46CB
:202DA00004D0154C2068F5B2A84202D80220BDE8F08104F124004FF0FF31804605F0CEF8AA
:202DC00004EB85049434206860B979680120A84027603246084307497860384603F0A8F8A5
:202DE000002400E00124404605F05AFB2046BDE8F081C046007FC767C4270020012898B52A
:202E000025D1012003F0E4FC012820D004F0FEFD124C012104F1D800017005F0FBF9800990
:202E200017D20D4800683222B2FBF0F707B90F46083C04F1300005F013FB04F130003946DF
:202E400005F00AFB04F1300005F008FB01E003F055F8002098BDC04604310020EC0C002052
:202E600098B50446207B00F00F00022824D100F03FFFA168081A8108114800F10C02176849
:202E8000002F14BFFB6840F6C41303F57A728A4212D20A4A12686FF050448C420CD3C91ADB
:202EA000B1FBF2F3012B8CBFB1FBF2F10121C83005F0D2FA012098BD002098BD0431002060
:202EC000A8200020001F06B480B290B5082803AFADF10C0D22DB3A78B0F5805F1EDA00F105
:202EE0008851091F0C686B461C6049685960BDF800108A420BD17988BDF80230994206D1BF
:202F0000B988BDF80430994208BF012007D0BDF80610401A083880B20828DDDA002003B09C
:202F2000BDE8904002B0704710B50446012002F05FFC208900280CBFEB2000201249607044
:202F400091F83F00C20824BF20F0040081F83F00820809D2400813D32B202070EB236370E1
:202F6000204600F095FD0BE091F83F0000F0FD0081F83F00217C6078C1F3001104F0D6FD10
:202F8000204605F08FF810BD042F002080B501460A7D012A05D0152A03D0252A18BF352A95
:202FA00002D1087E000919D3087EC3091BD2012A18BF152A01D1000909D24F781B2F04D0A8
:202FC000094807B10E30805C02E0232000E0312008700648007800F087FA80BD4A7808467C
:202FE0001146FDF797FD80BD630700007C13002030B5174C054605F12801ADF1140D04F136
:20300000AA0003F003FD08B3EF2309208DF801306B688DF800005A781978181D01EB022168
:20302000ADF802102A890178082A8DF8041014BF94F8E600C07805F11C018DF805000DF1CA
:20304000070005F0F8F96846FBF714F805B030BDCC0B002010B504460320ADF1180D04F154
:2030600028018DF8020000208DF8030001A805F0E5F96068007804F11C018DF80C000DF19B
:203080000D0005F0D8F904F1280003F019FE58B14FF6FF7453206946ADF80040F4F79AFAEF
:2030A000044920460A3108800DF10200FAF7E2FF06B010BD760C002070B5164D286808B1D2
:2030C00005F0CCF8144C606880470C3DE9690A68002616710968E961A16888470A4A0B4953
:2030E000107810B90846007860B1167008460670FCF7BCFA06480078012803D03046014636
:20310000F4F764F970BDC0461431002016310020E81900208C300020F4120020B0B5124C82
:203120004FF470000025E0601348A56000686560C06B80470D49C0F1FF3008600C48C768D7
:2031400065700FB90B49C1600C480570012001F0A9FF08B104F056FF0F2003F04FFAE06825
:20316000FFF72EF8B0BDC046B81800200830044034170020B93601006014002017310020FD
:2031800070B5164604460D1C08BF052426D034F07F0001D004F002FA002C18BF032407D1EF
:2031A00055F80C0C18B915F8020CFF2804D00524284604F0E5FE11E0012E094805F8024C99
:2031C00003D0294602F09EFF02E0294604F010F920464FF40041FCF741FD0024204670BDFE
:2031E0003C17002030B50446606800252062ADF1140DA5657820A4F84C0094F82C00256533
:203200000F2807D004F12C0120460122F6F72EFE08B116E0284694F83C10FF2901D1A16DDF
:2032200021B104F13C012046FBF75EFA48B92B4601208DF80C30032101AA00902046F0F7DA
:2032400041FC05B030BD2DE998430446A76E9946904607B1B8470020022110EA090701EA9B
:20326000080108BF002915D104F1600106C919EA020708EA010108BF00290BD16168097834
:2032800002290FD1082110EA090001EA080108BF002907D004F1700080E8000304F1400037
:2032A00005F0FEF8BDE898832DE9FC41144C154F06468846700809D3206845680021012265
:2032C0000B461FFA88F000903846A847B00809D3206845680021022201231FFA88F00090BC
:2032E0003846A847F00809D320681FFA88F600210C220223446800963846A047BDE8FC8131
:20330000A401001000A00C400246F8B5084611464C68203821D0401E1CD0401E18BF6FF097
:2033200001001ED18D6805F0A5F80E4E07463068016928688847B0F1FF3FF8D10025A56436
:20334000606C401EE06425653846A56305F086F92846F8BD0021084601E00121002084F84A
:203360002D10F8BDD001001038B504460D46E920694601F095FA13483D300078812801DBF3
:2033800084280FDB04F10D0081B2680824BF04F1260081B2122CCCBF05200220401880B227
:2033A000C0000DE0600100F5967081B2680824BF01F21E2081B2122CCCBF28200C20401885
:2033C00080B238BD760C0020F8B51549154A134D36395B320B681778E91C0978002F0CBFDC
:2033E0001C695C6901EB810164182679002101E0491CC9B28E42D8BF4FF6FF700DDD236888
:203400000A4602EB42029B1893F900209042EFD1B3F801002881B3F80100F8BD64170020E9
:2034200092140020860C002038B5154C04F1180005461C3000F040FF03F096FD042003F056
:20344000B7FDA07E032801D1607EA0B105F14501E120F4F7BFF805F14601E720F4F7BAF8AE
:20346000084894F85F100078884204D005F14701E820F4F7AFF82846FAF7FCFD38BDC046C0
:203480007C2F0020B30C002038B50120124C114D94F8A11085F83D000F2917D00F490870D2
:2034A000202004F007FE94F8A1200D490D4835F81220886201F1200091F84010491C5143AE
:2034C000490001F2A32103F037FC38BD02F0B2FD38BDC046BC160020CC0B002054120020C6
:2034E000E82F0020B119010070B502460D4632F07F0004D110460022FFF742FE70BD04F0C5
:20350000C5FE104908398C78A5F10C06FF2802D0C96A40184478FF2C02D104F03FF80DE04C
:20352000104604F08BF901462A46FF20B072204602F096FC20B1284604F022FD012070BD3B
:20354000002070BD3C17002000B5ADF1240DADF80000ADF80210116801A8016051684160EE
:20356000002002460D490690887D8DF80C200D318DF80D000B680DF10E0003604B68436039
:20358000097A017218208DF81C2005498DF81D206A460BF025FEC0B209B000BDC4060000AC
:2035A0001959000098B5154B1B1D18680004070C21D003F0E5FA104991F90720824205DDAA
:2035C00010F1800FB8BF6FF07F00C8718C88BC4210D80A68D3F8D40F801A801C1F2888BFEF
:2035E0001F203F1B4008C7404FF6FF70E719B84238BF071C8F8098BDFC30002030100940E2
:203600001348144A14490078801E0A2807D8DFE800F019140F06140F06140F0607C0FEE776
:2036200010688008FCD250688008FCD2F6F7CAB908688008FCD3F6F7C5B908688008FCD246
:20364000F6F7C0B910688008FCD3F6F7BBB9C046C80D002034600C4038600C403EB5401EC4
:203660004FF000040AD0401E04D0401E1CD1F6F7A9F919E0FFF750F8044615E0684604F009
:203680009EFE01940B4D8DF800400849029401226B4605F1780001F0BBF8054A2C2123460A
:2036A00005F19C0001F07EFC20463EBD013601005D480000E40C002070B5134C60688047AC
:2036C00012490025064648784D70A168820808D2C00816D33046884728460146F3F776FE2B
:2036E00070BD304688470A480078012803D001202946F3F76BFE606880470646FAF75AFE8B
:20370000A1683046884770BDF4120020B8180020E8190020B0B50F46044604F0ABFE05460B
:203720001148EC3890F8C710C90803D390F8C610A14215D0B0F8C430012101FA04F21A43D4
:203740000A4BA0F8C420181D026804F10C0399408A430260006818B917B1022001F06CFA73
:20376000284604F07BFFB0BD94210020081004401549096821280ADC212819D00C380FD07C
:203780000D380FD0001F0FD0C01E0FD01AE0253810D0001F10D0401E10D0401E10D011E0A7
:2037A000086870474868704788687047C8687047086970474869704788697047C8697047CD
:2037C000086A704700207047F0010020F8B50646B08815460F46FDF751F90446002D02D46C
:2037E000281B0A2806DB3368291B38460BA201F055FB0419B08978B1002D06D4B06804F096
:2038000043FB291B401D884206DCB368291B384603A201F043FB04192046F8BD257000C0DF
:203820002827257327290000F8B50746C81D01F00705C610002F4FF0010000FA05F0A0F1B0
:20384000010C14BF0029002019D00020BEB17F1E33460246941B17F8011FB4F1FF3F08D1CF
:203860000DB10CEA010104E001F1FF04401C2140C0B20029F8D15B1E02F10102EAD1F8BDB9
:2038800038B505466868297A02680801A0EB41001049095A40F2011048400D490143D068E5
:2038A0000140D1602C6804F0E5FD2A7AA11891F8441011B904F0D2FE38BDA418002184F816
:2038C000441004F0CBFE022002F04CFB38BDC046FEFEFFFF5E0B000038B505466C68D4F846
:2038E000A810237A002203B9012263689847D4F8BC00D4F8C010814211D08069C4F8BC009F
:20390000D4F8BC102846FDF7FFFAB0F1FF3F0ED10320207204F12C0004F0CCFD38BD00204E
:20392000C4F8A800C4F8BC00022002F01BFB38BD70B5F0F741FC124D68688047064604F00D
:2039400025F9104C94F9D60004F076FA03F006F804F068FA04F00EF904F000F9A968304670
:20396000884794F8D70000F07FFC04F1BD015220F3F730FE04F078FC08B9FFF7CFFB70BD57
:20398000F4120020CC0B002038B50C4620B141680122A240114201D1022038BD914341609B
:2039A0000E480025231800EB8401C1F8945003F140010978FF291ABF406850F8211044F038
:2039C00020410548F9F7B8FE20464FF0FF3103F02BFE284638BDC046007FC767C427002081
:2039E0001248134908B54FF42C72FCF7E3FD4FF00451002081F89003012081F879030220A8
:203A000081F87503032081F87703042081F8AE03052081F8AB03062081F88103072081F842
:203A20004D030448C1F8C00308BDC0461C04002164860100CD05002198B5124CE2685168D6
:203A4000496839B110B102F0D9FEE268506840688047E2685268906808B9D7688FB10A4941
:203A60001C310F68002FFCD000230B6010B18047E0684268D06800B180470448503803F008
:203A800093F898BDA82000200010044051000706144BB0B5997B03EB81010A69017801F087
:203AA0007F014D000170AC185219527803EB82052F6907B19A732278141103EB84031F6C3E
:203AC0002FB90C290CDA1821FDF724F8B0BD02F00F0257F8221011B904F094FAB0BD884721
:203AE000B0BDC0467C13002038B50546012001F07FFE124C2046143000F0DEFB2889002833
:203B00000CBFEB200020687094F83F00C10824BF00F0FB0084F83F0080080BD394F83F0089
:203B200000F0FD0084F83F00297C6878C1F3001103F0FCFF284604F0B5FA38BD042F00204C
:203B40002DE9F041054612480E46002100782960012802D00120F3F739FC0E4C60688047DF
:203B60003768804630463FB16A687968914203DC38463F68002FF8D1056030682F608542A5
:203B800001D1FDF701FDA16840468847BDE8F081E8190020F4120020134A38B5B2F8C4509E
:203BA0004FF6FF71A9421BD00024012000FA04F32B4212D05940B2F8C4300C4D1940A2F872
:203BC000C410291D0A6804F10C03984010430860022003F061FD204638BD641C0F2CE5DB79
:203BE0006FF0010038BDC046A82000200810044038B5044642F209000DF1020100F01EFCA7
:203C00009DF8020050B19DF8020002281AD1A08894F82710FEF730FC054606E042F20D00E2
:203C2000694600F00BFC9DF80050284600F01CFB0020A4F87C5094F82130607013B110205B
:203C400004F040FA38BD38B5046845682068002808BF4FF0FF301FD004F00CFC21680029B9
:203C600054BF491E0021216004F0F8FC206890B904F12C0004F0FCFB04F1480004F00EFC28
:203C800004F1640004F00AFC6868FBF753F904F1180003F03DFB002038BDFEE72DE9B84182
:203CA000124C0546201D00688047804603F0A0FA6F7E002F08BF6B6807D069682A69AF6894
:203CC000091A5218B9180B466960E968286105F11402184602F0DEF8012768686F76A1687A
:203CE000A86040468847BDE8B881C046F412002010B504F0BFFB104C217829B10F490C684F
:203D000004F0ACFC204610BD04F0A8FC04F03AF80B4A002303F0A6FF626A002314001B18D0
:203D20004FF07A024FF0905044EB0104C11842EB04021046001C10BDA820002004300440CA
:203D400000093D00B0B5134C6068628800B325880021AA42C8BF01210B46AA42C6BFA91A0C
:203D600001F58061A91A8FB28FB1012B03D0A1183A46083109E0A118C2F58062083104F04F
:203D8000D6FA606804F108012A4604F0D0FA6580B0BDC0469406002038B51248104C016841
:203DA000114D0C40E1430160A10907D34068800904D328464FF4005104F07AFB14F4602F46
:203DC0000DD02846EC3800F1C0010A6804F4602400F5907014430C60002104F069FB38BDAE
:203DE00020000E000810044094210020134910B5044691F83F00ADF1180D40F0020081F8C3
:203E00003F00012003F0C4FA607890B9211D02A803F075FD03F07EFE01460120009004F1C7
:203E200010030193E38902AA0520F2F799FE607010B1002103F07AFE06B010BD042F00202B
:203E40001FB5014604208DF8000048788DF80100B1F896000DF10203ADF80C008C3118464A
:203E600003F04DFD02F02CFF60B14FF6FF7453200DF10E01ADF80E40F3F7ACFB0449204668
:203E80000A3108806846FAF7F5F800901FBDC046760C00202DE9F0410120104E104D3070FC
:203EA00028781F469046022801D004F0ABF80024022114EA070001EA080108BF002902D192
:203EC00004F0A0F807E0074991F90000401E08702C7003F07FFE3470BDE8F081E8190020D8
:203EE000E9190020421900201048F8B50668114800680F4CC06B80476168401A217889005F
:203F0000B0FBF1F0B04201D304F07CF80A4D243D686880470746A6603046FDF7B3FFFAF738
:203F200049FAA96838468847F8BDC0461C190020B81800206014002018130020C8B5071C61
:203F400001D104F05FF879684878C6111FD03B89F96400204A78C2F3C3020F2A09D00A78CC
:203F60001018801C80B25218834202F10201F1DC01E0801C80B2834206DB79683E89411803
:203F80007960311A398100E00020A7F85000C8BD10B5044600211C22ADF1200D6846FDF7F4
:203FA000C0FE60788DF80000A0788DF80100E0788DF8020020791122611D8DF8030001A8EE
:203FC000FCF7F8FAA07D8DF8150008B1A06906900348006881696846884708B010BDC04648
:203FE00008190020F8B504460D46084611220021FDF797FE94F800C0BCF1000F1AD0641C99
:2040000000214FF0010EE078A37843EA0023207809E0C610AF5D00F00702401C0EFA02F2BA
:20402000C0B23A43AA558342F3DA491C241DC9B28C45E8DCF8BD80B502465378107840EA9B
:204040000320C7130F7007BFC0F3062300F0FF00C0F3C323C0F30A004B70802848800DDAEB
:2040600002280BDB012B0CD0022B0AD0042B08D0052B06D0062B04D0072B02D00022104693
:2040800000E0921C4A6080BD70B5114C2068E8B1104D686880470646216894F82F0002285A
:2040A00006DBA96830468847F120F5F7BFFB70BD04F1240003F09CF9002394F82F00A96855
:2040C0002360401C84F82F003046884770BDC0469C0A0020F412002038B5044642F208007F
:2040E0000DF1020100F0AAF99DF8020040B19DF80200022817D1204601F04CFC054606E02B
:2041000042F20C00694600F099F99DF8005094F8200030B9284600F0A7F8A4F87C5000202F
:2041200000E00120207038BDF0B5124D00260C460746ADF1140DC5F8B061012004F060F935
:204140002868C00FF9D3286A0090686A0190A86A0290E86A03903FB13846694611F8012BD4
:20416000401E04F8012BF9D1032005B0C5F838023046F0BD5045024010B50446012001F005
:2041800037FB2078212804BFEB2060700D4991F83F00C20824BF20F0040081F83F0080084F
:2041A00005D22B2020702046FFF772FC10BD91F83F0000F0FD0081F83F006078002103F05D
:2041C000B5FC10BD042F002070B5114D95F8A100B5F8C6400F2810D00E483430066801F07A
:2041E00063FD2018864208D895F8A1104FF4707088402418A41B04F57074044D284600F0CF
:204200005BF82146284603F00BFB70BD182F0020CC0B0020BC160020114898B501210170C7
:20422000022111400F4A4FF0E0471F4008BF002903D092F90010491E1170044692F90000D1
:2042400030B192F90000002806DC03F0DBFE03E000200146F3F7BAF80020207098BDC0462B
:20426000E819002042190020B0B50546802D01DD03F0C8FE0D4C606880470D4B0D490A4AC4
:204280001F780A390D701FB91778A1682FB907E01778A16837F07F0702D088470120B0BD14
:2042A0008847FDF7C7FFB0BD18310020F4120020901200207017002070B505460F480078D1
:2042C000012803D001200021F3F780F80C4C201D006880470B49064628460B4603F033F9FC
:2042E00018B9191D284603F02EF91869A84201D1FDF74AF9A1683046884770BDE81900201F
:20430000F41200201419002070B540680C46054600F5847004F0A4F80D482A7F0168687FF9
:204320008018AA69C01D80B244430A4805F584766043B0FBF2F008186330B0FBF1F1491C21
:20434000304604F089F8304604F088F870BDC0460431002040420F000146104808B500789B
:204360004FF4C852812803DB8428B8BF4FF41642052909D002F02AF90949407B09880228B7
:2043800014BF02F57A720A4402F57A624FF47A6002F5FA62B2FBF0F008BDC046B30C00209F
:2043A000F62D00200F4838B50078C8B10E4D0F4C95F82E106420503C4843206604F15C0092
:2043C000FFF76CFCE08EE26B95F82E10401C80B28918E08600B900210020E16300F03CFA00
:2043E00038BDC046890C0020FC2D0020902D0020F8B5114C60680D4680470E4BA16893F80E
:2044000030705A6B97B10024203A2032967F4EB1D37F9D4206D100239377FF23D37788479B
:204420002046F8BD7F1E04F10104EED18847FF20F8BDC046000F0020F4120020F8B50E460C
:2044400003F09EF805464FF6FF70A84208BF682013D00B4C6068804708490A4B0746680077
:2044600000EBC50008180278991842783046FCF7A1F8A168384688470020F8BDC400000096
:20448000F4120020FC2D002038B505466868297A02680801A0EB41000D49095A40F20110C7
:2044A0000840D1680843D0602C6803F0E3FF297A64184434217839B90121217004F0CEF808
:2044C000022001F0C3FF38BD04F0C8F838BDC0465E0B00003EB545688468684603F0B8FF16
:2044E0000C480068E96803682068094C54F82110002201B1012201999847074901200860A1
:20450000064A106041F8180C41F80C0C3EBDC046900D0000AC0100101C28004010040542F3
:20452000BCB5054614460F46684603F091FF27F00100204316D00199381C0BD0401E18BF80
:20454000201C10D1A5FB04014FF0FF320023F3F741FDBCBD044AA4FB01010023F3F73AFD32
:20456000401EBCBD681CBCBD40420F00042838B51CD1104CEC3C04F1C800054603F03AFD1A
:20458000A0B1284603F066FF09490968484364280CD2284603F064FF052001F057FF2046B6
:2045A000012141720421EC3003F082FF002038BD043100209421002038B5EB2003F0ACF9A2
:2045C0000D48002505700B480078862802D1284600F03EF8094C6068804709490C39CA695E
:2045E00013681D711268CA61A168884703F050F938BDC0461831002016310020F412002008
:204600008C30002038B50D4C6068804705460C48007870B90B48007830F07F0009D10A4813
:20462000007830B90948007830F07F0001D102F09FFEA1682846884738BDC046F4120020E9
:204640001531002014310020163100201831002038B50F49104C888B401C88836068804715
:2046600005460C480178862903D0A1682846884738BD8721017003F0FDFDA1682846884719
:20468000082002F095FCE920FCF728FE38BDC0465418002018310020F4120020F8B506463E
:2046A0000F4D104F7388002417E0A00000EBC400321851689068D26852B9AF420BD00A784C
:2046C00055F822200346491C08461946904701E0FBF770FF7388641CA4B2A342E5DCF8BDAB
:2046E000A8940100B494010070B50D4600220646142101F015FA002430460A21002201F041
:204700000FFAC4F10700092145FA00F2304602F0010201F005FA30460A21012201F000FA6F
:20472000641C082CE8DB30461421012201F0F8F970BDF8B5034600208C460446074613E0B3
:204740001CF8015B082685F0010101F001014018C0B2411E994206D0641C761E4FEA6505C0
:20476000E4B2F0D100E00127A24203DC27B903F07BFE01E0002FE3D02046F8BD3EB50546AF
:2047800015F8060C03281DD12B681869009058690190986902906C6859689A681868DB68FE
:2047A000A0472968086015F8080C01F03FFF0446012002F00FFC011C04D042200870204630
:2047C000FEF792FE3EBDFEE72DE9F04117468846064603F059FB0D4C0546002128222046FA
:2047E000FDF79FFA31462A462046FBF7E3FE40463A46291900F0E4F8204603F09AF802A06B
:2048000003F097F8BDE8F0810D0A00C058300020F0B515460E4604461F1CADF1240D08BF12
:20482000002308D0684600212422082303F0EEFEB8686B460690204631462A4603F0E2FED7
:204840000348044F0168204609B03960F0BDC046BC0D00000431002070B50F4C0546217963
:20486000E079814217DD6179A94214DDA3680B4E23B1294632469847E0796179A07101FB34
:204880000050216800EB800009180878E071D1F801103046884770BD90150020742D002010
:2048A000F8B502F032FE0D4607463B2F08BFF42012D00B4C606880470646BA0007480949D5
:2048C000835C801842784E39C918284603F0A6F9A168304688470020F8BDC0469C02000078
:2048E000F4120020AE0C002038B50D460E49144660390A68AA4205D901EB8501D1F8941013
:20490000884201D0022038BD03F0B4FD074B103B1A68AC400121A9408A4314431C6003F098
:204920009DFE002038BDC04624280020E02002401049D0B50F68ADF1180DCFB17E69BEB125
